:020000040800F2
:10000000F8FF0120190102088BF7040879F70408AA
:100010008DF7040899F70408A5F70408000000000C
:10002000000000000000000000000000B1F704081C
:10003000B3F7040800000000D90C0508F10C05080E
:100040000100020831F8040843F8040849F80408DC
:100050003B70050801000208056405080B640508EB
:1000600011640508176405081D640508FD2B0508C3
:100070000D2C05081D2C05082D2C05083D2C050808
:100080004D2C05085D2C0508010002087D5005086F
:100090005150050861500508715005082364050892
:1000A0005DF8040863F8040875F804087BF8040890
:1000B00081F8040887F804088DF804085D32050803
:1000C0007932050895320508B132050801000208A9
:1000D00001000208DDF80408E3F80408E9F8040860
:1000E0004764050837F80408C1F70408B9F804089C
:1000F000BFF80408D7F80408D1F804086D2C0508E7
:10010000010002080100020895F804080100020835
:10011000EFF80408F5F80408ADF80408B3F804088B
:100120007D2C05088D2C05089D2C0508AD2C050897
:10013000BD2C0508010002083DF80408BD50050863
:1001400091500508A1500508B1500508B5F70408FD
:10015000CD2C0508DD2C0508ED2C0508FBF804085E
:100160000100020801000208010002080100020863
:10017000010002080100020801000208000000005E
:08018000010002080100020861
:10018800006870470B0A017043700B0C090E8370EE
:10019800C1707047036A0239023B8B4283BFC3892F
:1001A800406B01FB030000207047034600F10B0180
:1001B8000020C20142EA500213F8010B50FA82F201
:1001C8008B42D0B2F5D1704737B50D46044620B9F9
:1001D800092000232B6003B030BD0368002BF7D043
:1001E8005A79002AF4D081885A899142F0D1186846
:1001F8000DF10702062102F0E9FA9DF8073003F035
:100208000103034313F0FF00E2D12368E2E738B5A6
:10021800C3790446C3B100F13C05826B0068012331
:10022800294602F0BEFA88B9A16BE36A626AE071F6
:10023800CB1A934208D2A379022B05D10A4420682D
:100248000123294602F0ADFA002038BD0120FCE761
:10025800F8B50446FFF7DBFF0546002842D163796D
:10026800032B37D1277A012F34D104F13C060146FC
:100278004FF40072304646F07DFD552384F83A323B
:10028800AA2384F83B3252234122722184F83C305D
:1002980084F83D30612384F83E3084F8233284F8B2
:1002A8003F2084F8201284F8211284F82222A169C0
:1002B80004F50970FFF766FF616904F50A70FFF736
:1002C80061FFA26A20680132A2633B46314602F010
:1002D80068FA257200222068114602F077FA003881
:1002E80018BF0120F8BD2DE9F0470026D0F800908E
:1002F8008E75836907460C46002B7DD0C36A01338F
:100308005FD1F96900234D1E184615F8012F202AE0
:1003180000F101000DD0052A08BFE522092805D102
:100328000B2B9FBFE6182E2777720133E61801338F
:1003380072720B28E9D1E21800205072A27D002ABF
:100348004FD1002B44D004F1080308255A78581CD3
:10035800002A53D11B1B083B3DE0B8F1000F05D123
:1003680000F520539BB2B3F5006F13D340F2B511DB
:1003780040EA084043F0AEFCFF28C5F1FF0A18D94F
:10038800BAF1010F20D96319020A9A75D8750223A8
:100398001D44002002368046D9F81030985B0028AA
:1003A800DBD1B8F1000F18BF002525440023AB7539
:1003B800A7E748B1BAF1000F08D06319987501236F
:1003C800E6E7B0463546E7E70025EAE75546E8E7B9
:1003D8003F23A3750123234400229A750B7B03B99D
:1003E8006372CB7A237201F11C00FFF7C9FE20600B
:1003F800CB8AE3800B8BA380BDE8F0872E2A1346B7
:1004080009D0413A192A03D80A7B154200D0203373
:10041800437303469AE71025FAE7C2F307238A765F
:10042800CB764379032B01BF120C0A75120A4A7561
:10043800704738B5836B8B4204460D460FD0FFF7E3
:10044800E6FE58B9206801232A4604F13C0102F06F
:1004580099F910B101204FF0FF35A56338BD002090
:10046800FCE7000038B50023C3714FF0FF33836306
:100478000546FFF7DEFF044608BBB5F83A224AF600
:1004880055239A421DD195F83C2002F11803DBB29E
:10049800012B01D9EB2A16D10C49032205F1720070
:1004A80046F094FC48B10A49052205F18E0046F051
:1004B8008DFC041E18BF01246400204638BD0424A6
:1004C800FBE70324F9E70224F7E700BFECD10508AE
:1004D800F0D10508F0B5437987B0044601F0FE0570
:1004E8008BB100680DF10702062102F06FF99DF843
:1004F8000730DE0707D40DB15C0702D4002007B02F
:10050800F0BD0A20FBE70023637120680DF10702A4
:10051800052102F05BF99DF80730D80700F1ED805E
:100528000DB15907EDD400212046FFF79BFF0228A3
:10053800034603D0012824D8257975B302AA04F20A
:10054800022304F24221174613F8040C10B118468E
:10055800FFF716FE10338B4242F8040BF4D12679CC
:1005680006B1013E57F826507DB129462046FFF7CF
:1005780079FF0346227952B9012B0ED90136032E91
:10058800F0D9042B07D10120B9E70323F2E7042BA4
:10059800F9D0012B01D90D20B1E7B4F84730B3F5F4
:1005A800007FF8D1B4F8521021B904F16000FFF7C8
:1005B800E7FD014694F84C3061625A1E012AA37186
:1005C800E9D894F84960E681002EE4D0721E3242E0
:1005D800E1D1B4F84D70A7813A07DCD1B4F84F00E7
:1005E80018B904F15C00FFF7CBFDB4F84A20002AE3
:1005F800D1D001FB03FE02EB171CF4446045CAD3BB
:10060800A0EB0C00B042B0FBF6F3C4D33C488342E5
:10061800C1D84FF6F57083425DD840F6F576B342FF
:100628008CBF0226012602332A4405EB0C00032E58
:100638002362A562E26260634FD1B4F866203A4350
:10064800A9D104F16800FFF79BFD9B0003F2FF139B
:10065800B1EB532F20639ED34FF0FF33C4E905332A
:10066800032E4FF0800323722BD1B4F86C30012B8A
:1006780027D1691C2046FFF7DCFE10BBB4F83A22EC
:1006880020724AF655239A421BD104F13C00FFF729
:1006980077FD1C4B984214D104F50870FFF770FDE4
:1006A80003F1FF5303F500532033984209D104F5B1
:1006B8000970FFF765FDA06104F50A70FFF760FD9A
:1006C8006061114A6671138801339BB2138063819C
:1006D8000023E36112E70326A5E7002F3FF45BAF91
:1006E800022E02EB0E004FEA43021BBFD21803F0A2
:1006F8000103134603EB5203A8E70320FFE600BFFC
:10070800F5FFFF0F525261418005002001292DE9B4
:10071800F84305460C4616466ED9036A8B426BD9D8
:100728004379022B3FD0032B4FD0012B64D101EB2F
:100738005107C16A01EB5721FFF77BFE10B1012079
:10074800BDE8F88305F13C0807F10109C7F308077C
:1007580014F0010418BF18F80720F3B21EBF02F006
:100768000F0242EA0313DBB208F80730E96A0123F3
:10077800EB7101EB59212846FFF75BFE0028DED11B
:10078800C9F308023CB1C6F3071608F80260012352
:10079800EB710020D4E718F80230C6F3032623F0E3
:1007A8000F031E43F1E7C16A01EB1421FFF741FE75
:1007B8000028C4D1640005F13C0304F4FF741A193D
:1007C8001E55C6F307265670E1E7C16A01EBD4113E
:1007D800FFF72FFE0028B2D1A40005F13C0304F472
:1007E800FE7423441846FFF7CBFC014666F31B0151
:1007F8001846FFF7C7FCCAE70220A1E7F8B5054687
:100808000E46FFF704FD0446A0B931462846FFF717
:10081800C1FC05F13C070646A8634FF40072214667
:10082800384646F0A7FAEB899C4205D3EB891C1B96
:1008380018BF01242046F8BD28680123321939461B
:1008480001F0AFFF0028F1D10134ECE703284B8B0E
:1008580004BF8A8A43EA0243184670470129F8B55B
:1008680006460C464ED9036A99424BD24379022B6D
:1008780029D0032B34D0012B44D101EB5105C16A97
:1008880001EB5521FFF7D5FD10B14FF0FF30F8BD52
:100898006F1CF16AC5F30805354401EB5721304652
:1008A80095F83C50FFF7C5FD0028EED1C7F30807BF
:1008B800374497F83C3045EA0320E3074CBF00096A
:1008C800C0F30B00E3E7C16A01EB1421FFF7B1FDA8
:1008D8000028DAD1640004F4FF743444A08FD6E70A
:1008E800C16A01EBD411FFF7A4FD0028CDD1A40003
:1008F80006F13C0004F4FE742044FFF741FC20F0AC
:100908007040C4E70120C2E7F8B50C46012C056821
:10091800064611462BD92B6AA34228D92AB14FF093
:10092800FF322846FFF7F2FE38B921463068FFF754
:1009380095FF2746044608B90020F8BD012816D0BF
:10094800431C16D0002239462846FFF7DFFE002850
:10095800F3D12A6AAB69911E8B4205D20133AB6190
:100968002B7A43F001032B72A242DED8E4E702207F
:10097800E3E70120E1E72DE9F843056881460F46E2
:1009880049B96E69C6B12B6AB34298BF0126AB69F3
:10099800A3B9002406E02846FFF760FF01280446B3
:1009A80003D801242046BDE8F883421C54D02B6AA2
:1009B8008342F7D83E46EAE70126E8E7BE4216D169
:1009C8002B6AD9F80000741C9C4228BF02242146D7
:1009D800FFF744FF0128E4D0431C3DD0F0B1D5F81F
:1009E8001480B8F1010F02D92B6A434500D8B046EC
:1009F80044462B6A0134A34203D8B8F1010FC8D08A
:100A08000224D9F800002146FFF728FF40B1012849
:100A1800C7D0013020D04445EBD1BAE7002CE6D04E
:100A28004FF0FF3221462846FFF770FE90B957B9BC
:100A38002A6AAB696C61023A934210D92B7A43F067
:100A480001032B72AEE7224639462846FFF75EFEC1
:100A58000028EDD00128A4D14FF0FF34A2E7013BD4
:100A6800AB61EBE72DE9F843076906682037B7F56E
:100A7800001F24BF0023836183690446894673B13C
:100A8800C7F30808B8F1000F39D141690133836110
:100A980041B9B389B3EB571F31D80023A3610420B0
:100AA800BDE8F883F389013B13EA572327D1304681
:100AB800FFF7D4FE0128054601D80220F0E7421CC2
:100AC80001D10120ECE7336A834212D8B9F1000F53
:100AD800E3D061692046FFF74EFF0546A8B101281B
:100AE800EBD0431CEDD001463046FFF787FE0028C7
:100AF800E7D1656129463046FFF74CFBA0613C36DB
:100B080046442761E6610020CAE70720C8E70000DD
:100B18002DE9F047FF25076880460E46A9460424BC
:100B2800D8F8181019B9002C74D004245BE03846A2
:100B3800FFF77FFC0446002855D1D8F81C0001783F
:100B48000029F2D0C37AE52903F03F0388F806307C
:100B58004FD02E294DD023F02002A2F1080CDCF151
:100B6800000242EB0C02B24243D10F2B47D14C0694
:100B78003DD5D8F81030457BC8F82C3001F0BF01BE
:100B8800437BAB4235D1428B9ABB0378D7F810C070
:100B9800DFF8889023F040030D24013B63434FF6B0
:100BA800FF7A012419F801EB30F80EE024B3FF2B8B
:100BB8001FD82CF813E07446013301320D2AF1D105
:100BC8000278520605D524B1FF2B12D800222CF842
:100BD80013204B1E5FFA83F900214046FFF742FFBE
:100BE800044600289CD00023C8F8183012E0894534
:100BF800C6D04FF0FF09EFE7D645DED0F9E7B9F1E7
:100C0800000F03D1FFF7D1FAA84203D04FF0FF330A
:100C1800C8F82C302046BDE8F08700BF16800608CB
:100C2800B1F5001FF8B506460C4601D30220F8BD01
:100C3800CA06FBD1826805680161BAB96B79022BD3
:100C480001D92B6B9BB9AB89B3EB541FEED9286B39
:100C5800C6E905200028E9D000EB54203C35C4F350
:100C680008042544B061F5610020E0E71346EF89E8
:100C78001A467F02BC42114603D22846FFF78AFA79
:100C8800E6E73068FFF7EAFD431C024606D0012874
:100C9800CCD92B6A8342C9D9E41BEBE70120C6E70C
:100CA800F8B50E46002107680446FFF7B9FF68B992
:100CB8000546A1693846FFF7BCFB38B9E3691B78DC
:100CC800E52B00D01BB90135B54201D1F8BD054669
:100CD80001212046FFF7C6FE0028EAD0042808BFF5
:100CE8000720F3E7C16A4B1C2DE9F0410568066946
:100CF800044618D1E5274FF00108A1692846FFF7F7
:100D080098FBA0B9E3691F7085F807802369B3428F
:100D18000DD201462046FFF7A5FE0028EDD0042895
:100D280008BF022003E0FFF77BFF0028E2D0BDE800
:100D3800F08100002DE9F04F002187B0D0F800A025
:100D48000446FFF76DFF0546002840F08A804FF003
:100D5800FF394FF0FF0804F12003C4F82C90C34674
:100D68000293A1695046FFF764FB0546002878D135
:100D7800E6693778002F78D0F27AE52F02F03F0342
:100D8800A37103D0100758D50F2B02D0C4F82C90AC
:100D98004BE094F82B3059063DD47A0643D52369A5
:100DA80096F80D80E36207F0BF07737B43453CD19B
:100DB800738B002B39D13578DAF810B005F03F0580
:100DC8000D23013D5D432A4B012113F8012BB25A33
:100DD80071B3FF2D059328D81046049242F0ACFF5A
:100DE8006B1C03903BF81500019342F0A5FF039993
:100DF80081421AD1049A019D059B11461D4A9A42C7
:100E0800E3D133785B0603D511B13BF8153063B9EC
:100E1800013F5FFA87FB00212046FFF723FE0546C6
:100E280000289ED01DE0BB45BFD04FF0FF0BF2E776
:100E38004FF6FF708242E1D0F7E7BBF1000F04D113
:100E48003046FFF7B2F940450BD094F82B5015F017
:100E580001059BD102990B22304645F0B7FF0028C7
:100E680094D1284607B0BDE8F08F0425F9E700BF04
:100E780016800608238006082DE9F04F90F82B30DD
:100E880013F0A00889B0054640F0E6800768396984
:100E980031F81820002A70D105F1200696E80700DD
:100EA8000DF1140A8AE80700DA0740F1DC804022D5
:100EB800864C85F82B204FF0010B9AE80700B446C2
:100EC800D7F810E0ACE803002CF8022BBBF1050FB3
:100ED8004FEA12428CF8002062D9AEF102005A465D
:100EE80030F8021F00294BD1D446072102F00F0E1B
:100EF8000EF13000392888BF0EF137000F2A0CF8A0
:100F0800010D01F1FF314FEA12104BD801F1200217
:100F18006A447E2002F8140C05F11F008446002262
:100F2800914206D01CF801EFBEF1200F02F1010931
:100F38003AD107299CBF01F1200CEC4402F10102CF
:100F480096BF1CF814CC4FF0200C0131072A00F88A
:100F580002C0EED928460193FFF7ECFE019B8146BB
:100F680000287CD10BF1010BBBF1640FA5D14FF028
:100F78000709484609B0BDE8F08F08F1010887E77E
:100F88004FF0100C01F0010E0EEB420212F4803FFC
:100F980018BF6240BCF1010C4FEA5101F2D19FE742
:100FA8005A46A1E70246A1E74A46B9E72969284611
:100FB800A1EB4411FFF734FE81460028D9D1304611
:100FC800FFF7F3F84FF6FF780190A9693846FFF765
:100FD80030FA81460028CCD1EB69019AD7F810E0A5
:100FE8005A73E1B24FF00F024FF00D0CDA72DFF8CE
:100FF800E0A018734A1E0CFB02F29876D876844655
:101008001AF8019B404518BF3EF8120003F8090082
:1010180003EB090B0CF1010C18BF01324FEA102940
:10102800002808BF4046BCF10D0F8BF80190E7D1AE
:10103800404502D03EF812200AB941F0400119702B
:101048000123FB7100212846FFF70CFD814600288B
:101058008FD1013CB9D11AE04FF0060989E704287D
:1010680087D185F82B309B0745BF08F10C040D2369
:101078000124B4FBF3F448BF013421462846FFF7A6
:101088000FFE814600287FF474AF013C8ED1A96918
:101098003846FFF7CEF9814600287FF46AAF01464B
:1010A8002022E86945F066FE03CEEB6918605960B6
:1010B800B278318819819A7295F82B30EA6903F071
:1010C800180313730123FB7153E700BF21100100BC
:1010D800168006082DE9F04F85B0036801930B7858
:1010E8002F2B0646884601D05C2B0AD1424613783E
:1010F8002F2B904602F10102F9D05C2BF7D0002388
:1011080001E0019BDB69B36098F800301F2B00F207
:10111800FE8080230021304686F82B3005B0BDE8DC
:10112800F04FFFF77DBD2F2811D05C280FD07F2806
:1011380007D8AA4A12F8013B1BB19842FAD10620F7
:10114800D1E0FF2DFBD02AF815000135E3E0424637
:1011580013782F2B904602F10102F9D05C2BF7D0BF
:101168000024E6E0022D04D1BAF802302E2B00F05C
:10117800E3800AEB450306E033F8022D202A01D06C
:101188002E2A02D1013D002DF6D14FF000032AF896
:1011980015300AEB4502002DD1D000213AF8110094
:1011A80020280B4601F10101F8D00BB92E2802D1F5
:1011B80044F00304E4B232F8021D2E2901D0013DA7
:1011C800F9D14FF020324FF0000972623262C6F84E
:1011D80027204FF0080B4F463AF813005A1C0028F6
:1011E80000F0E480202804D02E2807D1AA4200F07D
:1011F800D18044F00304E4B21346EDE7D94580F00A
:10120800CC80AA4212D1BBF10B0F07D1C9E0AA4288
:1012180004D044F00304E4B200F2C880BF00FFB277
:101228002A464FF00B0B4FF00809E5E77F2837D91E
:1012380044F00203DBB240F2B5110392029342F08C
:1012480049FD10F0800FDDE902320FD0644900F04B
:101258007F00085C28B1634C14F8011B11B3884265
:10126800FAD143F00303DBB25F2011E0FF28F1D984
:101278000BF1FF31894504D344F00304E4B2D946A5
:10128800BAE706EB0901040A81F8204009F10109CF
:1012980006EB09011C4681F8200009F10109ABE7BA
:1012A8002346D8E7A0F1410189B2192902D847F0AD
:1012B8000207EDE7A0F1610189B219299EBF203824
:1012C80047F0010780B2E3E7A5074BD407F0010315
:1012D80044EA0313DCB2780748BF44F0080441E04D
:1012E800002A08BF052005B0BDE8F08F5A074DD485
:1012F800B379DB064CD5019B03F13C013369C3F399
:1013080008031944019B5879FFF7A0FAB0603368C5
:10131800D3F810A0002518F8010B48B140F2B51118
:1013280042F0F6FC00283FF40AAF1F283FF6FBAE58
:101338000424012D7FF416AFBAF800302E2B7FF469
:1013480018AF00232AF8153006F11F029D4294BFFA
:1013580020212E2101330B2B02F8011FF6D144F076
:101368002004E4B286F82B403046FFF7E3FC96F8F9
:101378002B300028BAD00428B5D1990603F004020E
:10138800AED5002AC3D0802386F82B300020AAE7E8
:101398000520A8E7D945FFF436AFBBF10B0F7FF462
:1013A80036AF44F00304E4B24FF00B0B96F820304C
:1013B800E52B04BF052386F82030BBF1080F04BFD6
:1013C800BF00FFB207F00C030C2B04D007F0030397
:1013D800032B7FF479AF44F00204C2E7F6D1050885
:1013E800967F0608FFD1050800214171FFF772B802
:1013F8002DE9F0470546ADF50C7D924699460C4619
:10140800002900F0C18003F03F084146FFF762F869
:101418000746002840F0B0800CAB2B615146684667
:101428006E460095FFF756FE20B99DF92B30002B2C
:10143800B8BF062019F01C0F00F0838000283FD0A9
:10144800042840F099803046FFF716FD002840F048
:10145800938048F00808D6F81CA068795146FFF731
:10146800F5F9814655F0DEFF01460AF10E00FEF758
:1014780089FEF3692022DA72F16900222846FEF714
:10148800CCFFF36900221A775A779A77DA77012323
:10149800EB71B9F1000F10D049463046D5F838A0A5
:1014A800FFF732FA002867D151462846FEF7C1FFF8
:1014B80009F1FF336B6100285ED148F0400809E06C
:1014C800B37913F0110F45D119F0040F53D119F066
:1014D800080FC0D1AB6BF169236261626879FFF7CD
:1014E800B5F9A060034601F11C00FEF749FE6A89C0
:1014F800A28018F0200F4FF000020646E060256039
:1015080084F810806274E261626115D0A0B1B5F808
:101518000E8060614FEA4828B0451DD30020A361C2
:1015280050BBC6F308023AB119462846FEF732FE08
:1015380040B300EB5620E06138460DF50C7DBDE860
:10154800F087C8B9B379D8061AD419F0020FC1D0F8
:10155800D907BFD507200FE019462068FFF77EF9A5
:1015680001280346A6EB080603D9421CD4D1012062
:10157800D5E70220D3E70820002323600746DBE7EE
:101588000420F9E70220F7E70927D5E72DE9F04F0E
:101598009A4685B000238946CAF8003003A9044654
:1015A8001546FEF711FE002840F0868094F8118059
:1015B800B8F1000F1FD194F810B01BF0010300938D
:1015C8007DD0E6686369F61AAE4228BF2E4696B10A
:1015D8006269039FC2F30803002B55D1FB89013BC5
:1015E80013EA522B18D152B9A06801280CD84FF031
:1015F800020884F81180404605B0BDE8F08FA16963
:101608002068FFF72BF9F0E7431C04D10123DDF82C
:1016180000806374EFE7A061A1693846FEF7BAFD60
:101628000028E4D0B6F5007F0BEB00022BD3F98934
:1016380001920BEB562088424FEA562588BFA1EB52
:101648000B0538682B46494601F09CF80028DDD187
:10165800FB7963B1B86B019A801AA84207D24FF49C
:10166800007207F13C0109EB402045F03FFB6D0299
:10167800DAF800302B44CAF8003063692B44761B33
:10168800A9446361A3E7E2616569E169C5F30805F7
:10169800C5F50075B542384628BF3546FEF7C9FE80
:1016A8000028B3D161693C37C1F308012A4639449F
:1016B800484645F01BFBDBE74FF009089BE74FF076
:1016C800070898E72DE9F04F9A4685B00023894628
:1016D800CAF8003003A904469046FEF775FD0028B5
:1016E80040F0A980677C1FBB237C9A0740F1A58046
:1016F800636913EB080F01D36FEA0308B8F1000F11
:1017080012D06369039EC3F30802002A77D1F589D2
:10171800013D15EA53251ED173B9A16871B9204658
:10172800FFF729F9014648B9237C43F040032374A5
:10173800384605B0BDE8F08FA169F0E7012902D16C
:1017480002276774F4E74B1C01D10127F9E7A36866
:10175800A16103B9A160B26BE3699A4204D1304632
:10176800FEF755FD0028F0D1A1693046FEF712FDBD
:101778000028E5D0B8F5007F05EB000B32D3F189DE
:1017880005EB582088424FEA5823306888BF4B1B26
:101798005A464946019301F004F805460028D4D179
:1017A800B16B019BA1EB0B01994209D24FF4007276
:1017B80009EB412106F13C0045F098FA019BF571CF
:1017C8005D02DAF800302B44CAF800306369A8EBF0
:1017D8000508A9441D44E3686561AB422CBFE3607A
:1017E800E5608BE76169E368994206D33046FEF706
:1017F8000EFD0028A9D1C6F838B0C4F81CB0656938
:10180800E169C5F30805C5F500754545304628BFAB
:101818004546FEF70EFE002897D1636906F13C00A5
:10182800C3F3080318442A46494645F05FFA4FF0C7
:101838000103F371C5E709277AE7072778E72DE958
:10184800F34101A90546FEF7BFFC88BB2C7C14F0C8
:10185800400429D055F0E6FD019F296A80463846A4
:10186800FEF7E7FD0446F8B96E6AF37A43F0200301
:10187800F372AA6828683146FEF7CFFDE96806F1D9
:101888001C00FEF77FFC414606F11600FEF77AFCC5
:101898000123B474F4743846FB71FEF7D9FC2B7C31
:1018A80023F0400304462B74204602B0BDE8F081C3
:1018B8000924F9E713B50446FFF7C1FF28B901A9C0
:1018C8002046FEF781FC10B9206002B010BD092047
:1018D800FBE7F0B50F46ADF50D7D00210546FEF797
:1018E800F9FD044670B90CAB2B6139466846009582
:1018F800FFF7F0FB044698B99DF92B30002B05DA69
:10190800029BEB6120460DF50D7DF0BD9DF806307C
:10191800DB0609D507996879FEF798FFE861F1E7D2
:10192800042808BF0524EDE70524EBE72DE9F04F6F
:101938000D460021ADF5557D297006461746FEF780
:10194800C9FD019000BB54ABD6F81C9033610DF172
:1019580008083C46C8F80060B9F1000F1BD1BC422A
:1019680002D1013C2F232B552B46611B1A5D03F82E
:10197800012B5A189742F9D87B1E1B1B0134A7422A
:1019880038BF002301351D44019800232B700DF545
:10199800557DBDE8F08F20214046C8F81CB0C8F836
:1019A8000890FFF73DF9D8F81CB08246C0BBD8F8BC
:1019B80018103046FEF73DFD824688BB70795946BF
:1019C800FEF744FF5146C8F808004046FFF728F9DB
:1019D800D8F80830D8F81C10824608BBC8F81C1084
:1019E80040460021C8F80830FFF792F8D8F81CB034
:1019F800824680B970795946FEF728FF48451ED0BF
:101A080051464046FFF72EF8D8F80830D8F81C1091
:101A180082460028E2D0BAF1040F08BF4FF0020A4C
:101A2800CDF804A0B0E7013B0EAA02EB030C9CF82A
:101A380016C000F801CD15E04FF0110AF0E7404656
:101A48000EA9D8F80890FEF74EFC0DF14D0053464C
:101A580010F8012F19460133002AF9D19C42EBD323
:101A680028190B46002BDED1631E5C1A2B445B1A27
:101A78002F21197070E72DE9F7430D4601A9044697
:101A8800FEF7A2FB00287DD1667C002E51D1E368C9
:101A9800AB4204D2227C12F0020F08BF1D4600227E
:101AA800636962619DB90020E2686369934282BFFD
:101AB800227CE36042F04002C3F3080388BF22742B
:101AC800002B36D0E369834233D0E06131E0DDF8A2
:101AD8000480B8F80E707F027BB1013B6A1EB3FB2D
:101AE800F7F1B2FBF7F28A4207D37A421340A169B1
:101AF8006361ED1A0029D6D002E0A16889B1A1611D
:101B0800BD42636920D863692B446361C5F3080348
:101B1800002BC8D04046FEF73DFB40B100EB5520F6
:101B2800C2E72046FEF727FF0128014605D1022615
:101B38006674304603B0BDE8F083481C01D1012625
:101B4800F6E7A160A161D5E73B446361237C9A076E
:101B5800A5EB070906D52046FEF70DFF054628B96F
:101B68000146D0E72068FEF779FE05466B1CE6D0F3
:101B7800012DDCD9D8F82030AB42D8D9A561294647
:101B88004D46BDE70926D4E770B50546ADF5007D9D
:101B980016460C4649B30021FEF79CFCD0B92560D7
:101BA8003146C5F810D02046FFF794FAB8B994F931
:101BB8002B30002B07DBA379DB0614D56879E169A4
:101BC800FEF744FEA0606B89A38000212046FFF742
:101BD80027F808B1002323600DF5007D70BD0428A7
:101BE80008BF0520F6E70520F4E70920F4E713B558
:101BF80001A90446FEF7E8FA00B9206002B010BD5A
:101C080070B5ADF5027D01AE0D4631460446FEF7CE
:101C1800DBFA0146F8B93DB9294620460DF5027DA3
:101C2800BDE87040FEF7FCBF336802AA1A6120467F
:101C3800FEF76EFF10F0FB060AD129462046FEF794
:101C480052FB31462046FEF70DFF042808BF00204E
:101C58000DF5027D70BD0920FAE72DE9F0418846AF
:101C6800ADF50C7D002107461646FEF733FC0097BC
:101C7800044680B90CAB3B6141466846FFF72AFA37
:101C8800044640B99DF92B30002B09DB1EB13146C3
:101C98006846FEF728FB20460DF50C7DBDE8F0816F
:101CA8000624F8E72DE9F84F884600210446FEF798
:101CB80011FC054640B9D4F820A0A369AAF1020294
:101CC800934204D8C8F800302846BDE8F88F6379F5
:101CD800012B17D10227064639462046FEF7BEFDDE
:101CE800431C34D0012834D000B90136236A0137A7
:101CF800BB42F1D8C8F80060237AA66143F001031B
:101D08002372E1E7E16A0746064604F13C0937B960
:101D1800204601F1010BFEF78CFBE0B959466379C7
:101D2800022B0AD1E3199B8F03B901360237BAF1A6
:101D3800010AC7F30807EAD1DCE709EB0700FEF759
:101D48001FFA30F0704308BF01360437EFE701256A
:101D5800D0E70225CEE70546CCE72DE9F0410F464E
:101D6800ADF5187D02210546FEF7B4FB0446A8B977
:101D780018AB2B61394668460095FFF7ABF96E46FC
:101D8800044658B99DF82B309A0641D41B063FD417
:101D98009DF8068018F0010F05D0072420460DF5A0
:101DA800187DBDE8F08107996879FEF74FFD18F0B6
:101DB800100F07460BD13046FEF794FF0446002863
:101DC800ECD1E7B92846FEF743FA0446E6E7EB69A3
:101DD8008342E2D00DF130080E90214640460C9522
:101DE800FEF71EFF04460028D8D101464046FEF7FC
:101DF8008FFE04460028D0D00428CFD1DBE7024666
:101E080039463046FEF780FD04460028C6D1D9E79A
:101E18000624C3E72DE9F0470E46ADF5107D0221F3
:101E28000546FEF757FB044600286FD104AF10ABF8
:101E38002B61314638463D60FFF74CF904460028CF
:101E480073D0042862D197F82B1011F020016ED1BD
:101E580068460095FEF78FFDE946064600285AD0E9
:101E680001285AD0431C5C425C4155F0DBFA80469D
:101E7800002C54D131462846FEF7C0FC0446002801
:101E88004DD14FF02033C5F83D30C5F84130A5F8A5
:101E980045302E2385F83C30102385F847304146DD
:101EA80005F1520005F13C04FEF76CF93246214673
:101EB8002846FEF7B2FA05F15C031A4651F8040BFE
:101EC80042F8040B9942F9D12E23BA6885F85D309F
:101ED80028464FF0010AFEF7A0FA85F807A0384611
:101EE800FEF7CAFF0446D0B9F86941461630FEF736
:101EF80049F93246F9692846FEF78FFAFB6910223C
:101F0800DA7285F807A0FEF7A3F9044620460DF516
:101F1800107DBDE8F0870724A7E70224A5E7002283
:101F280031464846FEF7F0FCF0E70824EEE70624C1
:101F3800ECE72DE9F0430E46ADF5217D022104467C
:101F48009146FEF7C7FA002840F0828008AD20AB22
:101F58002361314600232846AB602C60FFF7BAF8AE
:101F6800002875D195F82B3013F0A00F74D1EE69C5
:101F7800D5F8088033466F4606F1200C1868596872
:101F88003A4603C2083363451746F7D1AE46BEE862
:101F98000F00F77A14AEB446ACE80F00BEE80F00A5
:101FA800ACE80F009EE80F008CE80F004946304669
:101FB800FFF790F840B9B368434503D132692B69FC
:101FC8009A4203D0082043E0042841D13046FEF766
:101FD80053FF00283CD1F1690DF10D0301F10D0209
:101FE8000DF11D0053F804CB42F804CB8342F9D11C
:101FF800188810809B789370FA0658BF47F020071E
:10200800CF720127E771CB7ADB061AD5B36843454F
:1020180017D06079FEF71AFC01462046FEF7BAF899
:102028000146D8B12046FEF704FA88B994F85D3025
:102038002E2B06D1B26804F15C012046FEF7EDF9BB
:10204800E7712846FEF74EFE10B92046FEF700F964
:102058000DF5217DBDE8F0830620F9E70220F7E7BA
:102068002DE9F041884692B002210746FEF732FA80
:10207800044698BB4FF0203301936D460093CDF88A
:10208800073008F1FF38064618F8010F1F281FD837
:102098009DF80030E52B20D01EB1731EEA5C202A83
:1020A80034D0002106A806970891FEF7B9FD04462A
:1020B800A0B9012106A8FEF72BFD90BB0D9B3EB3EE
:1020C80003CD186059602988AA789A72198121E08D
:1020D80040F2B51141F01CFE20B90624204612B08A
:1020E800BDE8F08141F028FE40F2B51141F0F2FD63
:1020F8000028F2D01D4A12F8013B13B19842FAD1D8
:10210800EBE7FF2822D80B2E29D1E6E71E46C3E7C6
:10211800E5221A700123FB713846FEF799F8044648
:10212800DCE70428FBD1002ED8D0012106A8FEF751
:10213800B7FD04460028D1D1202201460D9844F06D
:1021480019FE0D9B0822DA720D9BB9E7092EC4D837
:1021580006F148036B44020A03F8482C013606F1DD
:1021680048036B44013603F8480C8DE7847F060862
:102178002DE9F04FD0F800908BB01C460023437136
:10218800039103790293154605210DF11F02484674
:1021980000F01CFB9DF81F30DE0700F15182580744
:1021A80000F1508208AA0321484600F00FFB30B91D
:1021B800089A531EB3F5004F01D21A4201D00123E9
:1021C80008935DB19F4BA5F500729A4203D913207D
:1021D8000BB0BDE8F08F6B1E2B42F8D1002C00F03D
:1021E8003382149BB3F5007FC0F02E82029B002B34
:1021F80000F09D80012300222146484600F0C2FAE3
:10220800002840F0B782B4F8FE214AF655239A42D6
:1022180001D00E20DCE7029B04EB031202F5D77312
:1022280092F8B221002AF4D003F10800FDF7A8FFC4
:10223800804603F10C00FDF7A3FF8246BAF1150FA3
:10224800CDF824A0E5D9B5F5813FC0D2039B13F0A2
:1022580002030593039B00F0818003F00703022B20
:1022680000F08180039B03F00103C3F10303DBB299
:10227800089A032B4FEA552502F1FF3CC2F1000EE4
:1022880040F08980002D50D16F4A4FEA5A4101250C
:1022980032F8023B13B18B4267D90023BAFBF5F23F
:1022A8006A499600A2F57F42F63A06F207268A4264
:1022B8004FEA5626ADD8002201924FF0200B032793
:1022C80008EB0B020092019AB11808EB0B021144BB
:1022D800032F01EB0C0208BF009802EA0E02A2EBE2
:1022E800010206BF80189344B618C8EB05120A44C9
:1022F80008BF009052458CD8019AAAEB0202A2EBC3
:102308000B02032FA2EB0602B2FBF5F2049232D1C4
:1023180004994FF6F572914200F2AE81002B7FF4DA
:1023280078AF012D7FF675AF6D082B46B6E709AA81
:102338000121484600F04AFA002840F01B82039A1F
:10234800099B110707D43E2B7FF663AF4FF03F0878
:10235800A3EB080A72E7DDF80880F9E7DA077FF5EA
:1023680036AF022384E7032382E76D0090E752002B
:1023780017E02A461AE0022F40F0778104994FF6B9
:10238800F57291422ED9002B40F069816A00402AEB
:1023980000F25C811546002DEBD12D494FEA1A3623
:1023A800012231F8023B0BB1B342E0D940F6F57394
:1023B800BAFBF2F69E429BBF06EB46060136023692
:1023C80076088CBF7600033606F2FF162B461546B4
:1023D8004FF020028CBF02270127760A01924FF0A6
:1023E800010B6DE7049940F6F572914200F24481C1
:1023F800002B7FF40EAF6D00802DCCD909E7514634
:1024080004F12000FDF7BEFE5FE155F00BF8014630
:1024180004F12700FDF7B6FEC6F30723E375802312
:1024280084F82430292384F826300A4BA67504F151
:102438002B0203F1100153F8040B42F8040B8B42F2
:10244800F9D181E100FEFF00767F0608FFFFFE0F4D
:10245800687F060826D20508032F37D1012308F123
:1024680006022146484600F09CF905994FF400728F
:10247800204644F07FFC5223237063706123A370CD
:1024880084F8E731049B41227221E27084F8E41158
:1024980084F8E51184F8E621591E04F5F470FDF777
:1024A80071FE022384F8EC3108F10702012321466A
:1024B80084F8FEB184F8FFA1484600F072F90123C0
:1024C80008EB03022146484600F06BF9149A0021F4
:1024D8006FF30802204644F04DFC032F6FD1F82318
:1024E8002370FF236370A370E37023716371A3717A
:1024F800E37123726372A3720F23E372149B4FEA92
:10250800532A5645B34628BFD3462146009A5B4610
:10251800484600F046F90146002840F02B814FF468
:102528000072204644F026FC009BB6EB0B065B4489
:102538000093E6D1019B032F08BF2B460193019D11
:10254800009A554528BF55462B462146484600F077
:1025580028F9002840F00E81009B2B440093019B32
:102568005B1B0193EBD1032F32D0099BB3F5803F5E
:1025780030D2022F14BF01250425029B63B3002229
:1025880001232146484600F0FDF80246002840F0A5
:10259800F180029B04EB031383F8B2510123214617
:1025A800484600F0FEF8002840F0E480002211467A
:1025B800484600F00BF9003818BF012008E6012F43
:1025C8006D49204618BF6FF00701FDF7DBFD95E761
:1025D8000C25D2E70625D0E7039B1B07E6D4029912
:1025E8004FF40072204644F0C5FB552384F8C251CD
:1025F800099D84F8FE31AA2384F8FF3105EB08020F
:1026080043F6C163B2FBF3F2FE2384F8C3319308A7
:1026180043F03F03012684F8C43184F8C5214146BC
:1026280004F5E37084F8BF6184F8C061FDF7AAFD82
:10263800294604F5E570FDF7A5FD029A3346AEE795
:102648000320C5E50A20C3E51120C1E5059B002B41
:102658007FF41AAE802A3FF6DCAD1546A6E6059A49
:10266800002A3FF4D6AD1D4618E6049A40F6F573E5
:102678009A423FF6CEAD01274FF400720021204662
:1026880044F078FB3D4B84F80EB01A6822605A6813
:1026980062601A899B7AA37202232373012323742D
:1026A800FB1E18BF0123CBF3072B5B00BAF5803F55
:1026B8002281657384F80FB0A374BFF4A0AE84F8C8
:1026C80013A0CAF3072A84F814A0F82363753F23DC
:1026D8002376FF23A376414604F11C00FDF752FD43
:1026E800032F7FF492AE54F09DFE014604F143009F
:1026F800FDF748FD314604F12400FDF743FD0223B0
:1027080084F82C30002384F82D3084F82E3084F897
:102718002F3084F8313084F83330802384F8403007
:102728002923012284F84230154B84F830200622F0
:1027380084F8322003F1100104F1470253F8040B26
:1027480042F8040B8B42F9D119889B7811804FF01D
:10275800550B4FF0AA0A9370214684F8FEB184F80D
:10276800FFA101234246484600F01BF805900028C7
:102778003FF472AE01202BE5F8FFFF0006D20508F2
:1027880012D2050810B50C4611461A4638B1234630
:10279800043040F015FF003818BF012010BD042098
:1027A800FCE710B50C4611461A4650B123460430D2
:1027B80040F01FFF10F11E0F05D0003818BF012090
:1027C80010BD0420FCE70220FAE7000070B50C46B3
:1027D80015460646002831D0234A01F00703D15C8C
:1027E80071B30022043040F022FF062C26D8DFE81F
:1027F80004F008050A152518180006202BF01CFB04
:102808002860002070BD062804D14FF4007028808D
:10281800B060F6E72BF010FB80B2F8E701232B60DD
:10282800EFE7062801D0430806D1336AB3FA83F3E9
:102838005B099B002B70E4E70123FBE70420E1E739
:10284800062CFBD801A353F824F000BF0B2800087E
:102858000328000813280008252800084528000830
:102868003328000833280008747E0608022970B54A
:10287800044615461E4613D15368012B0AD0022B75
:102888000CD01BB91168201DFFF7F5F8A3692B6060
:10289800002070BD81692B681944F4E70169FAE7E3
:1028A80001290AD10430FEF7CAFF0028F0D0084BEE
:1028B8001B5C33604FF0FF30EBE7042906D1436817
:1028C800002BE5D00430FEF7F5FFEEE71623F0E71E
:1028D800547F060837B51D46043001AB1446FEF791
:1028E800F1FE38B1064B1B5C2B604FF0FF342046DD
:1028F80003B030BD019BA342F9D01C23F4E700BF0D
:10290800547F060813B51C46043001ABFEF73EFEA3
:1029180030B1044B1B5C23604FF0FF3002B010BD98
:102928000198FBE7547F060870B5054608460C4633
:102938002BF098F92346024602492846BDE8704024
:1029480001F016B9E1D10508F8B5064610460F465C
:1029580031F036FC2B49421E2B48002412F8013F67
:10296800BBB92C202BF06CF90546384631F028FC11
:102978002F1D0246E3B206F144003946FEF738FD42
:102988000646B8B328461DF097FC204B985D2AF000
:10299800A7FB782BE2D8712B08D8612B25D0622BA6
:1029A80026D02B2BDAD144F00304D7E7723B062B51
:1029B800D4D801A555F823F0E129000865290008B5
:1029C800DD2900086529000865290008E7290008AD
:1029D800ED2900080B49C1E744F00104BEE744F0C3
:1029E8000A04BBE744F00604B8E744F01204B5E76C
:1029F8000146B3E7E30603D529693846FFF73BF8F4
:102A08002846F8BD847E0608B47E0608547F06086A
:102A18002DE9F04F099FDDE90BC4DDE90D5650B1F2
:102A2800884208D3710747BF0137013401350A21AD
:102A380058BFB0FBF1F016F0020E39D0002D37D098
:102A48000BDB0A998D4233DA2C44A74203DC07F1E9
:102A5800FF3CA4EB0C0C00252AE0291D28DB694269
:102A68004FF000084FF00A0AB0FBFAF90AFB190404
:102A78001CB108EB0504414604E008F1010888454B
:102A88004846F1D11D464FF0300905F8029B7F1AE0
:102A9800091B4FF02E084C1E83F801802346A846D8
:102AA800002B5DDC002908BF00242B190025FF241A
:102AB80007F1FF3841464FF00A09002954DA611C32
:102AC800B94260DBFE2CD4BF002101213B44BCF19C
:102AD800000F07D0A4EB0804A4EB0C0C2E20302721
:102AE800644555D1BEF1000F09D041B119460B46D6
:102AF80011F8010D3028FAD02E2808BF0B4606F031
:102B08000101294327D0710725D4002DBABF6D4292
:102B18002D212B2106F02004632D597044F0450423
:102B2800C8BF64211C704FF00A00C9BFB5FBF1F1A2
:102B38009C1CDC1C3031C8BF9970B5FBF0F62346ED
:102B4800B6FBF0F100FB1161303103F8021B00FB0A
:102B580016513031617000211970981ABDE8F08F54
:102B680008F8019B013B9BE78C42B4BF01F1010BC4
:102B78008B46B0FBF9FA09FB1A00303003F80B005A
:102B88000139504699E701332E21195501219DE756
:102B980014B903F8010B012103F8017B013C9FE7FD
:102BA8002DE9F04F2DED028B884610EE101A97B0E4
:102BB80000291C46B0EE408A9DF888300E902ADA2B
:102BC800B4EE400AF1EE10FA25D6B1EE408A2D2374
:102BD8000E9F07F8013B08F1FF389FED7D7AF0EE74
:102BE800C87AF4EE477AF1EE10FA02F0200316DD07
:102BF80043F0490443F04E00FA1C43F04601002319
:102C080078703C70B97013700E9BD01A17B0BDEC79
:102C1800028BBDE8F08F002BDAD10E9FDDE7B4EE12
:102C2800488AF1EE10FA06D743F04E0143F041000E
:102C3800FA1C0C46E3E742F02002662A4FD143F023
:102C4800040B002CA8F1030650DA0624A6423346EA
:102C5800A8BF23460C9318EE103A002B099353D0C3
:102C6800C3F3C7537F3B07EE903A9FED5A7AF8EECD
:102C7800E77A18EE103A67EE877AB3F17E5FFDEED9
:102C8800E77A38BF4FF0000917EE905A28BF4FF087
:102C9800010909EB0500B7EE000A00F01BFA099BD1
:102CA800B3F17E5F2CBF4FF0010A4FF0FF3AB4EE4C
:102CB800C80AF1EE10FA94BF012300234B451BD03C
:102CC8001BF0040F4CD0002D20DD6319023398450A
:102CD8001CDA8BF0040343F0020B013444E0672A4A
:102CE8000CBF43F0020B43F0010BAAE7632CADD1F4
:102CF80010230C930924AEE7554405EB0900B7EE01
:102D0800000A00F0E7F9D2E7099DD9E7A8F1020225
:102D1800A242D4BF33462346002D1EDA022B15DD0E
:102D2800AA1C17DA6E429E42A8BF1E46023E9C1B92
:102D3800092C0DDD1BF00403A4F1090207934FF0E1
:102D480009041CD004230793032319E05C1C002604
:102D58000022F7E75C1C0026EAE76C1C1C44FAE733
:102D68001BF0020FB9D034B1092C4FF00006E1DC9A
:102D78003246079603E02646224607940124072395
:102D8800062CA146A8EB0408A8BF4FF00609A8EB3B
:102D98000308A9EB0503013B0D939045D4BF04EB51
:102DA8000803A3181193119BA3EB09030F93099B25
:102DB800002B00F0CB80079B002B00F0C380002D78
:102DC80080F2BD8046B909F1FF3008963B4613E012
:102DD800FFFF7F7F9B209A3E3B46302103F8021B72
:102DE8002E227A701846324643F0C4FFFF2203466B
:102DF800334409EB060008920A214FF0010C0A91AE
:102E0800E14500F3A880B9F1060F40F3AF8001282F
:102E180040F3AC80B9F1070F00F0A480022800F05D
:102E2800A18002384FF06408B0EE480A0B9300F016
:102E380051F9F6EE007A30EE270A0A99BCEEC00A7C
:102E48003A4610EE103A08FB03F8089B03930F9BD1
:102E580002930C9BCDE9045BCDE9009340460B9BA4
:102E68001093FFF7D5FD15AA01460B90384600F0E0
:102E780061F9DDED157A0B9977EEC87A17EE902A8D
:102E8800002A58D0B9F1060FC4BF09EB4902123A1B
:102E98004FF0010AC8BF0AFA02FA0C22109BCDF8BB
:102EA8002C80F0EE678A109217EE902A002A089A72
:102EB80003920F9A02920C9A0A991393B4BFD044C2
:102EC800A8EB0A08CDE90092CDE9045B3A464046F2
:102ED800FFF79EFD15AA01461290384600F02AF920
:102EE800DDED157A129977EEC87A17EE902A12B3AB
:102EF800B0EEE77AF0EEE86A37EE667A139B17EEE3
:102F0800102A002A35DB4FF00A0CB8FBFCF00CFB4A
:102F180010800243002A0B9A08BF42460B9208BF52
:102F2800F0EE678ABAF1010F28D0109A013A4FEAF9
:102F38005A0A1092B8D10E9B3944C81A66E60D9801
:102F4800089543E7079B0D9808933FE7099A08926D
:102F58003B46104650E70A990A2251430A910CF160
:102F6800010C4DE701384FF00A085DE74FF0010802
:102F78005AE7CDF82C80F0EE678AD3E70D9AA14581
:102F880002F101020D9202DA09F101090BE70B9A2D
:102F98009045D0D0089A03920F9A02920C9ADDE9D4
:102FA8000A10CDE90092CDE9045B3A46FFF730FDFF
:102FB8000146C0E708B5044631B1054B4A6B0360CA
:102FC800096800232DF086F820461DF025F900BF7A
:102FD800681706082DE9FF41044601921F46461866
:102FE8002AB1023A222A02D9374829F083FEB4428C
:102FF800254626D34FF00008711B284601AA28F061
:10300800CCFB019B054428460024B04201462AD344
:10301800B8F1000F00D06442640044F00104A942F2
:1030280004D00D46B5422B4642D348D0019A2749D1
:103038002748012A08BF00222DF000F83946FFF77B
:10304800B9FF14F8010B1EF051FA80460028CED1C2
:103058002B782B2B01D12546CEE72D2BCAD125461F
:103068004FF00108C8E710F801CBACF13002092A8B
:103078000AD9BCF15F0FC8D04CF02002A2F1610C54
:10308800BCF1190FC4D8573A9342C1D983FB044104
:10309800B1EBE47F03D1144494EA4402B5D5711B23
:1030A800424603A803952EF0E4F903990446B6E7CF
:1030B800187801351EF01AFA0028B3D1B6E7204671
:1030C80004B0BDE8F08100BF76BA05088BBA0508E0
:1030D800D816060808B52DED028BE8B1B5EE400A02
:1030E800F1EE10FA18D010EE103AC3F3C7520244AA
:1030F80062F3DE5310F10A0F08EE103A0FD3434281
:1031080000EE903AB1EE040AF8EEE00A42F0CEFA88
:10311800F0EE407A88EE270ABDEC028B08BD07EE78
:10312800900AB1EE040AF8EEE70A42F0BFFA28EE78
:10313800000AF1E700232DE9F047014404469046D0
:103148009E461D4618461F469A461E468C4257D232
:10315800A4461CF8012BA2F13009B9F1090F38D89F
:10316800022E07D1354A904202DC0A2202FB009067
:103178006446EBE7B9F1000F14D0314A974211D8F1
:103188000A24B5B975460A24CDB997421ED8012E2E
:103198004FF00A0208BF03F1FF3302FB07974FF015
:1031A800000EE5E70EB90135E2E70EF1010E012642
:1031B800DEE7974294BF67430133013DE1E7974259
:1031C8009CBF03F1FF336743013DDDE77EBB01335D
:1031D800E5E78EB92E2AEAD042F02009B9F1650F49
:1031E8000CD1614504D962782B2A19D104F1020C5B
:1031F8008C4520D00226BBE7022EEDD15F2AB7D03E
:10320800BAF1000F15D107EE907A1D44B8EE670A9F
:103218002844FFF75FFF88ED000A2046BDE8F087E5
:103228002D2AE7D104F1020C4FF0010AE0E7AE467F
:10323800BDE74042E7E70024EFE700BF64666606A3
:10324800979999192DE9F04F2DED048B83B09FEDD7
:10325800658ADDF840909FED649A054690461F46C2
:1032680046184FF0000AF0EE488ACDED018AB542C3
:103278002C466CD34FF0000BA31C9E4240F2898071
:10328800237843F02003692B73D1637843F020033C
:103298006E2B7ED1A37843F02003662B79D14FF0B3
:1032A800FF430193E31D9E4204F103001AD9E3781A
:1032B80043F02003692B15D1237943F020036E2BAB
:1032C80010D1637943F02003692B0BD1A37943F024
:1032D8002003742B06D1E37943F02003792B01D125
:1032E80004F10800B8F1000F0ED0B0420CD20378F8
:1032F80043F020036A2B07D1844204BF4FF07E536A
:10330800019301304AF0020ABBF1000F05D0DDED50
:10331800017AF1EE677ACDED017A844240D0044615
:10332800B442254643D348D1BAF1010F38D09DEDB8
:10333800010ABAF1000F4AD0F0EE400AB0EE480A8E
:1033480003B0BDEC048BBDE8F04F2BF0B7BD15F80A
:10335800010B1EF0CBF88346002888D123782B2B4D
:1033680001D12C4688E72D2B84D12C464FF0010B38
:1033780082E76E2B0DD1637843F02003612B08D1CF
:10338800A37843F020036E2B03D1E01C8DED019A46
:10339800A8E701AA311B2046FFF7CCFE0028A1D1DF
:1033A800124913482CF0B4FD4946FFF703FE28786C
:1033B80001341EF09BF80028B2D1002FF0D0BAF1EA
:1033C800000FEDD19DED018A4FF0010A4DE717B1CD
:1033D800DFED040AB4E703B0BDEC048BBDE8F04FA1
:1033E8002CF06CBF000000000000C07F97BA0508F1
:1033F800D81606080846114644F044BC70B5054680
:1034080008460E4643F0F4FC044620B102466B68B9
:10341800286831469847204670BD00002DE9F74FCF
:103428008A469DF8301091460D9A11F0DF0F074635
:10343800A2EB090552D0302954D1C3F34721002902
:1034480054D05F290CBF0526042692FBF6F106FB33
:1034580011210CBF2A482B4809B901350132711EC8
:1034680092FBF6F406FB14228A1A00EB020813F00A
:1034780020023ED005EBD573A5EB63045D10002D4B
:103488003BDDAB465E4532467B683868A8BF5A4686
:10349800414601929847019AABEB020BBBF1000F32
:1034A800F0DCB9F1000F05D07B6838684A46514610
:1034B80098474D44002C0DDD2544A642B146A8BFCF
:1034C800A1467B6838684A464146A4EB09049847F8
:1034D800002CF2DC284603B0BDE8F08FDFF8288026
:1034E8001026C4E70DF130080126C0E7DFF81C807C
:1034F800F6E713F00104C2D02C460025D1E700BF3F
:1035080030060608350606083B060608240606089F
:103518002DE9F04F93B09246CA07DDE91E761C9C50
:103528009DF87490059380460D460BD48B0703D104
:1035380009687C4B994205D028462AF07DFC450055
:1035480045F0010514F0210306D1B9F1300F03D17C
:10355800B742B8BF37461E4628462DF098FE0028C9
:103568000DF1280B1CDBA00716D52B238DF828306E
:103578000DF1290322079DF814101FD5BAF1020F87
:1035880010D118464FF0300C00F802CB01F1010CB5
:1035980083F801C0034611E0610701D52023E5E760
:1035A8005B46E7E7BAF1080F5BD1302018702006B8
:1035B80045BF01F10E0058700133023300200EAAF6
:1035C8001870012EA3EB0B030B924FF01002069319
:1035D800C4F34723C8BF1443CDE90C2014F01002EC
:1035E800CDE902138DF82700059245D0CDE900A05A
:1035F8002B460DAA0CA90BA82DF00CFD03782D2B3A
:10360800824606D18DF827300D9B013B00F1010A57
:103618000D93012E7ADD0D9D059BB542B8BF354649
:103628002BB19DF8273003B10135069B1D4424F0CA
:103638000103AF42079371DD14F00109A7EB0505FB
:103648006DD120230195009337494B464A464046A1
:10365800FFF7E4FE4D460446059B4FF03009C3B919
:1036680036E0BAF1100FA9D118464FF0300C00F827
:1036780002CB01F1170C8BE70AABCDE900A30DAA29
:103688002B460CA90BA82DF0C5FC8246C1E70025E6
:103698002C469DF8273053B100230122CDE9003292
:1036A8000DF127014046FFF7B9FE013F0444069B90
:1036B8005BB100230122CDE900325946069A404603
:1036C800FFF7ACFE069B0444FF1A012ED8BF3E4606
:1036D800CDE90096079B0D9A51464046FFF79EFE9E
:1036E80004444DB12023009300230F4901951A4645
:1036F8004046FFF793FE04440B980EAB984201D066
:103708001CF0DAFD204613B0BDE8F08F059B079446
:10371800002BBCD11D461C463E46D9E70025002497
:103728009AE700BF141D0608AFD205082DE9F0433B
:1037380007469007984658BFC2F380038DB05ABF1A
:103748005B01DBB22B23164600930A46159BDDF876
:103758005090212103A8FFF723FAF20504461FD54C
:103768002E2103A843F08AFBD0B9652103A843F0B2
:1037780085FBA8B96E2103A843F080FB80B9631CC0
:1037880004F130026A4430336B442E2102F8241CC1
:103798000234302203F8242CA3186B4403F8240CB9
:1037A80073060ED504F13002631C0DEB02042522CA
:1037B80004F8242C03F130026A44002102F8241C86
:1037C8001C4616F010051DD09DF80C302F2B4FF01D
:1037D800000319D8012203A9CDE900323846FFF7C2
:1037E8001DFE09F1FF390546013C0DF10D01CDE93A
:1037F8000089334622463846FFF710FE28440DB0AC
:10380800BDE8F08303A9F2E703A91D46EFE700002E
:103818002DE9F04F81468BB014464FF000080B4657
:103828001D4613F8012B0AB1252AF9D1A94208D25D
:103838006E1AD9F80430D9F8000032469847B044D7
:1038480029460B78002B00F08B8120234A1C039318
:103858000027134613F8016B3EB12D2E25D01ED834
:10386800202E29D02B2E24D00026154612F8013BF5
:10387800A3F13001092922D92E2B4CD16B782A2BA0
:1038880023D00023154612F8011BA1F130000928A6
:103898001ED80A2000FB031BABF13003F2E7302EE1
:1038A800E2D147F01007039601E047F001071A46F6
:1038B800CFE747F00207FAE747F00407F7E70A21DE
:1038C80001FB0633A3F13006CFE754F8043B023579
:1038D80023EAE37B2B786C2B08BF013595F800A011
:1038E800BAF1000F00F03C81BAF1780F09D8BAF1AB
:1038F800570F13D8BAF1470F5AD8BAF1440F00F24C
:103908001D81D9F80430D9F80000012229469847CA
:1039180008F1010885E04FF0FF3BDBE7AAF1580307
:10392800202BEED801A252F823F000BFBF390008BF
:103938000B3900080B3900080B3900080B3900084F
:103948000B3900080B3900080B3900080B3900083F
:103958000B390008113A00083B3A0008BF39000843
:10396800453B0008453B0008453B00080B3900086B
:103978000B3900080B3900080B3900080B3900080F
:103988000B3900080B3900080B390008BF3900084B
:10399800513A00080B390008793A00080B39000839
:1039A800BF3900080B3900080B390008BF39000877
:1039B800BAF1500FA5D154F8040B0AF0DF03502BCD
:1039C800014667D1BAF1640F6AD1002880F29D8060
:1039D8002D238DF8173041420A2251230DF1280A70
:1039E8000A3B0DF1180BB1FBF2FC02FB1C10092875
:1039F8008CBFC01830300AF8010DDA458E46614692
:103A08005DD07245EFD95AE054F8043B019653B1A2
:103A1800039B5549009304223B464846FFF7FEFCAA
:103A28008044691CFBE6039B009350493B460522F2
:103A3800F3E754F8043B8DF81830039B0093019684
:103A48003B46012206A9E8E706A954F8040B1DF035
:103A58003AFBBBF1FF3F014604D0069B9B4538BFAC
:103A6800CDF818B0039B0093069A01963B46D4E71D
:103A780054F804AB504643F0BBF9BBF1FF3F024694
:103A880002D0584528BF5A46039B009301963B46EF
:103A98005146C2E7BAF1640F97D0BAF1750F2ED02C
:103AA8002AF00F0300220F3B8DF81720DBB21022FB
:103AB800002893D130238DF827300DF1270A17F00D
:103AC800100B9DF817302DD0002B35D0039B009399
:103AD800012201923B460DF117014846FFF79EFC73
:103AE800013E8346039B00930AAA01963B46A2EB3C
:103AF8000A0251464846FFF791FC584490E70023D4
:103B08008DF817300A226123D2E7BB0705D52B238E
:103B18008DF817300A225123CAE7C7F380035B01E7
:103B2800DBB2F5E7002BDDD006AA9245DAD90AF810
:103B3800013C0AF1FF3AD5E79B46D3E7073424F066
:103B48000704F4E8020154F0B3FDCDE9006B00EE80
:103B5800100A039B3A4651464846FFF7E7FD5FE7E0
:103B680040460BB0BDE8F08F1DB5050822B5050825
:103B78000EB403B503AA52F8041B0192FFF748FEDE
:0C3B880002B05DF804EB03B070470000D1
:020000040802F0
:10000000FEE700000F49D1F8883043F47003C1F8CF
:1000100088300D4B1A68002042F001021A60986087
:100020001A6822F0847222F480321A60074A5A60F9
:100030001A6822F480221A60D8604FF000638B6047
:10004000704700BF00ED00E000380240103000248F
:1000500030B5002495B010252A4621460AA80494FC
:1000600026F08CFE284B01941A6C42F080521A64E0
:100070001B6C03F080530193019B244B029419687D
:1000800041F4804119601B68059403F48043029396
:100090000122029B4FF48033CDE908234FF4800105
:1000A00002230F22CDE90E3112930723CDE90B4530
:1000B000039208254FF4A87213934FF4A05C4FF4F9
:1000C000805308A8CDE91052CDE906C32AF014FAEE
:1000D00010B10F482FF01AF8119B109A3021DB0055
:1000E000B3FBF2F3B3FBF1F201FB1232003A1299C7
:1000F000B3FBF1F118BF012203A830F0DBFE08B119
:100100000448E7E715B030BD0038024000700040F9
:10011000008B0508128B05080446DFF82CD00B492C
:100120000B4A0C4B03E051F8040B42F8040B9A42C3
:10013000F9D300200849094A01E041F8040B914233
:10014000FBD320462FF036B9F8FF012074DA0608F9
:100150000000002034000020340000209C220020F9
:1001600040F8044B40F8045B40F8046B40F8047B13
:1001700040F8048B40F8049B40F804AB40F804BB03
:1001800040F804CB40F804DB68467047024B5A69DC
:10019000026058610020704734000020024B5A6909
:1001A00012685A61704700BF34000020024B9A6900
:1001B000C0E900219861704734000020044A936927
:1001C0001968916110B15A6818461047704700BF0E
:1001D0003400002038B5054D0446AB690BB1A3428D
:1001E00000D338BD0120FFF7E9FFF6E73400002017
:1001F000C460056146618761C0F81C80C0F820902A
:10020000C0F824A0C0F828B0C0F82CD080ED0C8B2A
:1002100080ED0E9B80ED10ABC0F808E0FFF7B6BF95
:10022000124D6C6908B50CB92FF0B0F8606020462B
:10023000FFF7D0FF23686B612046C46805694669F3
:100240008769D0F81C80D0F82090D0F824A0D0F88E
:1002500028B0D0F82CD090ED0C8B90ED0E9B90ED4B
:1002600010ABD0F808E00120704700BF3400002038
:1002700010B50021044600F0F9FA18B914B120466F
:100280000CF028FD10BD002100F0F0BA10B50121DE
:10029000044600F0EBFA18B914B120460CF01AFD30
:1002A00010BDFFF7E5BF10B501220C4600F002FCBF
:1002B00018B914B120460CF00DFD10BD00F0FABBCA
:1002C00000F0BABB2DE9F0432B4C864600254FF0D9
:1002D000030CD4F8B402002101310EEB01039A089B
:1002E00003F00303825C5B0042FA03F303F00303B1
:1002F000022BF1D0D4F8C002090100EB0E108E08D9
:1003000089B300EB860603681A0729D1D4F8C01216
:100310005A1AC2F3011E99424FEA92174FEA4E0E43
:100320004FEA12121CD8D4F8C412994218D9D4F842
:10033000B48218F8071041FA0EF303F003030CFA25
:100340000EF9012B41EA09010AD104EB450E3F2DBC
:1003500008F807109ABF0135AEF8D422C4F8D0329D
:100360000430B042CFD12DB1013D04EB4503B3F8C9
:10037000D4E2AEE7BDE8F0833400002030B51C4C79
:10038000D4E9AF53C01AC109C0F3021E6B5C01224D
:1003900002FA0EF223EA02036B54D4F8C82283094E
:1003A0004FEA101CB2EB901FD4F8B40288BFC4F817
:1003B000C832C15C4FEA9C0E0CF0030303255B00BE
:1003C00005FA03F321EA030100F80E100CF1010C09
:1003D000D4F8B4024FEA9C0E0CF0030310F80E1090
:1003E0005A0041FA02F202F00302022AE7D030BDBD
:1003F0003400002021F00F0138B50B1A134A144CB9
:10040000013BDB00A2FB03235B0A9A00C4E9AD03B6
:100410000546C4F8C4120732A1EB831101331D4411
:1004200003EBD202C4F8C0120021C4F8BC5226F07B
:10043000A5FC002301214FF0FF32C4E9B233C4E927
:10044000D6322381A4F8541338BD00BFF32C23FA0D
:1004500034000020024A138902331381704700BF21
:1004600034000020024A1389023B1381704700BF09
:1004700034000020024B1889003818BF0120704753
:1004800034000020F8B51C4D2B89002243F00103F5
:10049000C5F8D0222B81C5F8582305F1080405F5CD
:1004A000027654F8043F1A071AD1D5F8C022981AD8
:1004B000C0F3011193424FEA901C4FEA41014FEA09
:1004C00010100DD3D5F8C422934209D2D5F8B472D6
:1004D00017F80C2042FA01F303F00303012B02D0BA
:1004E000B442DED1F8BD03238B401A4307F80C2039
:1004F000FFF7E8FEF4E700BF3400002081B3F8B551
:10050000184E0F46051F002455F8043F1A071AD14C
:10051000D6F8C022981AC0F3011C9A424FEA9011F3
:100520004FEA4C0C4FEA10100DD8D6F8C4229A426C
:1005300009D9D6F8B4E21EF8012042FA0CF303F010
:100540000303012B03D00134A742DDD1F8BD0323FF
:1005500003FA0CF31A430EF80120FFF7B3FEF2E79B
:10056000704700BF340000202DE9F043614ED6F8FB
:10057000D032D6F8B41283B0C3B1D6F8B832002561
:100580009800C6F8D05288B10024A30804F00302F2
:10059000CB5C5200134103F00303032B1FD0013443
:1005A0008442F2D3D6F8D032002BEAD1D6F8CC323E
:1005B0004FF000094FEAD3080127D6F8BC3213F8F0
:1005C00009504FEAC9043DB304F00303E8074FEABA
:1005D00094024FEA430314D46D080134F4E7204633
:1005E000FFF770FED6F8B832D6F8B4120134B4EB87
:1005F000830F4FEA8300C8D3D6F8D032002BC0D186
:10060000D4E78A5C42FA03F303F00303012B09D019
:100610006D0804F10104D7D1C84509F1010326D0C2
:100620009946CAE7D6F8C0C223016A465CF803308F
:1006300040F297310CEB04105BB10BF0DBFC009B3C
:100640003BB10CF093FDDDE900010CF05FFD0CF017
:10065000A3FDD6F8BC02E30804F00701C25C07FA68
:1006600001F122EA0102C254D6F8B412D0E7002701
:10067000BE463A46032402250FE0012806D104FABB
:1006800003F32CEA03030B704FF0010ED6F8CC32C3
:1006900001329A421FD8D6F8B412900802F0030330
:1006A00011F800C05B004CFA03F000F003000228D0
:1006B00001EB920119D00328DFD105FA03F32CEAEC
:1006C000030C81F800C0D6F8CC32174601329A42AA
:1006D0004FF0000EDFD93389002223F00103C6E971
:1006E000B227338103B0BDE8F083BEF1000FEAD03A
:1006F000C5E700BF34000020044B1A89002142F0F6
:100700000102C3F8D0121A81FFF72EBF3400002077
:10071000554BD3E9B0122DE9F043521A0024D3E926
:10072000AD61C0E90144C0E90344C0E90544026089
:100730004FEA810C22462146A146A6462746254679
:1007400016F809304FEA4E0E43FA0EF303F0030396
:10075000012B02F1010255D0022B24D033BB01370B
:100760009445876004F101046DD04FEA920902F0CC
:10077000030E16F809804FEA4E0148FA01F818F006
:1007800002013BD108F0030894452DD0B8F1010FC8
:1007900004D1C3689C4288BFC46000244FEA920918
:1007A00002F0030ECCE7013545600131944541D09C
:1007B0004FEA920902F0030E16F809304FEA4E088C
:1007C00043FA08F303F003089B0718D401292CD03F
:1007D000022903D1436901334361022183698B42BA
:1007E000D2D294458161D1D1C3689C4200D9C46002
:1007F0002D013F01C0E90157BDE8F083194694453A
:100800009ED1F5E701359445456025D04FEA920920
:1008100002F0030E16F809804FEA4E0148FA01F87B
:1008200018F0020FEAD108F00308036901330361ED
:100830000121D3E701299846F7D00229CAD083695C
:100840009942CED8D0E7C368A342D0D32D013F014F
:10085000C0E90157BDE8F083026901320261826993
:10086000002AC1D18361BFE7340000202DE9F8439D
:1008700000F10F0636093FD06E4C2389E3BBB4F874
:1008800054230D46E2BBD4F8C802D4F8B872B8427B
:1008900032D24FF0010ED4F8B4C20138013F6044A7
:1008A00067440021CCF1010818E04A1C964255D952
:1008B00013F00C0F42D18A1C964240F2AA8013F02A
:1008C000300F41D10132964240F2A8803F2B2ED802
:1008D000511C8E4240F2A780B8420AD008EB0009B2
:1008E00010F8013F9A07E0D013F00C0F21D101223C
:1008F000E2E7BEF1000F0FD000231846BDE8F883F1
:10090000D4E9D612914226D2D4F8C802D4F8B872EB
:10091000874288BF9E46BED835F0DAF8D4F8C802C0
:10092000D4F8B872B8424FF0010EB4D3E4E7002116
:10093000D2E713F0300F0CD10122C4E703F03002EC
:10094000B2FA82F25209C1E73F2B8CBF002101218C
:10095000C2E70022BAE735F0BBF894E74FEA89090D
:10096000A9EB0201012A01F1010704D109F10103F8
:100970009B08C4F8C832D4F8CC324B4538BF4B463C
:10098000B808C4F8CC3207F0030E1CF800804FEA18
:100990004E0E0123023103FA0EF343EA08038945A0
:1009A0000CF8003012D34FF0020E8808D4F8B4C20D
:1009B00001F003031CF800805B000EFA03F3013121
:1009C00043EA080389450CF80030EED2D4F85833D6
:1009D000D4F8C0823344C4F8583308EB071312012B
:1009E0001846002126F0CAF9EA074FEA071603461F
:1009F00083D50022D4F8BC0248F80620F908012269
:100A0000445C07F00707BA40224342541846BDE849
:100A1000F8834FEA890909F10109A1E74FEA890939
:100A200009F102099CE74FEA890909F103090A461D
:100A300096E700BF34000020034B1A89012A02D830
:100A400008B1FFF79BBC704734000020034610F04C
:100A50000F001CD1164AD2F8C012994216D810B411
:100A6000D2F8C4429C420ED95B1AD2F8B4429A0919
:100A7000C3F30111A25C49000A4102F00302012AFA
:100A80004FEA131305D05DF8044B70477047002000
:100A9000704701301A18910802F00302615C52009D
:100AA00041FA02F202F00302022AF2D00001EAE760
:100AB000340000202DE9F84F0F460646002800F0CC
:100AC000CA80734D2C89002900F09180002C40F0E1
:100AD0009280D5F8C002D5F8B8C2301A030903F1E4
:100AE000010E0F31BEEB8C0F4FEA11114FEA8C0A49
:100AF00080F0B780D5F8B492A4464FF001084FEAD1
:100B00009E040EF0030B19F804404FEA4B0B44FA15
:100B10000BF404F00304022C2BD02CB90CF1010CC3
:100B20000CEB08048C4226D341455CD065D3C44409
:100B30008C4525D2002A5ED0C209D5F8BC12895C4A
:100B400003F007031941384601F00101FFF78EFE5B
:100B5000044600284FD04FEA0812314626F0CAF862
:100B60002B89012B02D83046FFF708FC2046BDE850
:100B7000F88F08F101080EF1010EF245BFD1D3E75D
:100B80005C1843449C421FD9980803F0030219F8EB
:100B9000007052004FF0020C01330CFA02F23A439B
:100BA0009C4209F800200FD99808D5F8B47203F0D8
:100BB000030217F800E052000CFA02F2013342EA95
:100BC0000E029C423A54EFD1D5F8CC32A1EB080288
:100BD0009C4238BF1C46120106EB08100021C5F8E4
:100BE000CC4226F0CBF834462046BDE8F88F012CE5
:100BF00001D8FFF7C3FB0024B8E75C18A00804F095
:100C0000030719F800E07F004FF0030CA8EB010187
:100C10000CFA07F72EEA0707012909F8007004F11A
:100C2000010410D003EB080EA708D5F8B43204F085
:100C30000302D95D52000CFA02F2013421EA0202E9
:100C40007445DA55F0D1D5F8C8328342CBD9C5F80E
:100C5000C8023446C8E701463846BDE8F84FFFF7FA
:100C600005BE0129BFD029B14FF00108002A7FF449
:100C700063AFC0E7D5F8B442800903F0030359001D
:100C80000322235C8A4023EA02032354DBE700BFEC
:100C90003400002010B58AB0044603A8FFF738FDE1
:100CA000DDE90430039A009007492046E2F764FF2B
:100CB000DDE9083206980549CDE90020079A20466B
:100CC000E2F75AFF0AB010BDF4DC050818DD05088C
:100CD0002DE9F843DFF858914749D9F8C022074673
:100CE000E2F74AFFD9F8B81289006DD0DFF84481E5
:100CF000002515F03F0633D005F003067600D9F83D
:100D0000B422AB08D35C334103F00303022B63D05E
:100D1000032B5FD0012B4AD1D9F8C0222B01D25826
:100D200042455BD0354B9A425AD0354B9A425BD004
:100D3000344B9A4256D0344B9A4253D0334B9A425A
:100D400054D0334B9A4251D0324B9A4252D0324B0C
:100D50009A424DD0314B9A4214BF68224D2227E06F
:100D6000A9421ED9D9F8B4022C4602E001348C42C3
:100D700008D0A20804F00303825C5B0042FA03F38C
:100D80009B07F3D0621B7F2A0BD92549920938466D
:100D9000E2F7F2FED9F8B83224F03F05B5EB830F45
:100DA00012D220492A013846E2F7E6FEA7E72E22B2
:100DB0001D493846E2F7E0FED9F8B8320135B5EB07
:100DC000830F4FEA830194D338461849BDE8F843AE
:100DD000E2F718BB6D22EBE73D22E9E75422E7E793
:100DE0004C22E5E75322E3E74422E1E74122DFE733
:100DF0004222DDE74622DBE760DD05082C1E0608FF
:100E00001416060804270608D42606083C1306080C
:100E1000C8120608BC1A0608581B0608981F0608C0
:100E20007CDD050898DD0508A0DD05085CDD05080A
:100E3000340000204C280608064A0346506A1A6807
:100E40004168C1F31E018A4202D3521A1A607047E8
:100E50000068F5E734000020014441F20553884260
:100E600004D398B2012838BF0120704710F8012B35
:100E700003EB43135340F2E7034B044A5A62002248
:100E8000C3F80C22704700BF340000203C5706080E
:100E90002DE9F04781460F46002943D0FFF7DCFFDC
:100EA000214B5C6A82460CB9204637E094F9073042
:100EB000E668002B06F1FF364FF0000516DB013621
:100EC00004F11808B54215D32468ECE705EB0608D1
:100ED0004FEA580808F106033A4654F823104846EA
:100EE00025F0B0FF0028CCBF45464646731B012BBA
:100EF000ECD8E4E7236933F815309A4510D16369DB
:100F00005B5D9F420CD158F825003A46494625F0D2
:100F100061FF28B96068C0F31E002844BDE8F0876F
:100F20000135CFE70120F9E7340000202DE9F8432F
:100F300080460F46FFF7ACFF002840F09280FF2F5D
:100F400003D9494949480BF0B9F8494DD5F80C3255
:100F50007E1CABB1D5E9841232448A422CD90246B8
:100F600031441846FFF7AAF9D5F80C320446E0B927
:100F70000246D5F814121846FFF7A0F9C5F80C423E
:100F8000802E344638BF80242046FFF77CF9034684
:100F9000C5F80C02B8BB3046FFF775F90346C5F833
:100FA0000C0278BB30460BF095FED5F81022324487
:100FB000C5F81022002BE3D0D5F814229C18324437
:100FC0004146C5F8142220463A464FF0000825F065
:100FD00091FE04F8078039462046FFF73DFF814621
:100FE000686AD0E90262B2422BD376000A2E38BF7B
:100FF0000A26C6EBC6001830FFF745F948B9C5F810
:101000000C02CFE734460022C5F81042C5F814227E
:10101000D2E700F1180202EB8602696A026102EB74
:10102000460242614A680160C968C0F80C80C2F398
:101030001E020A44416862F31E01C0E901164246DD
:1010400068620169436921F812909F54911D6B6A8F
:1010500043F82140D96858680131C0F31E00D960B7
:101060001044BDE8F88300BF268B0508B0170608BA
:101070003400002010B5044625F0BEFE014620468F
:10108000BDE81040FFF752BF07B5019001A8FFF778
:10109000D3FE019A036933F8120003B05DF804FB34
:1010A00007B5019001A8FFF7C7FE019B4269D05C1C
:1010B00003B05DF804FB07B5019001A8FFF7BCFE83
:1010C000019B063350F8230003B05DF804FB13B511
:1010D000019001A80C46FFF7AFFE019B4269D25C6C
:1010E0002260063350F8230002B010BD2DE9F8430A
:1010F0001D46002303600B6013602B60164BDFF866
:101100005C905C6A07468846164664B92B6832686C
:1011100013442B60BDE8F883336812F8010B0133E8
:10112000034433600DE04C45F0D03B6801333B6035
:10113000E268D8F800301344C8F800306269E36808
:10114000D1188A42E8D32046FFF780FC2B68246838
:1011500003442B60D9E700BF340000203C57060849
:10116000F8B50B4B0B4F5C6A0CB1BC4200D1F8BD1B
:10117000E36804F1180505EB8306B54201D3246842
:10118000F2E755F8042B04490448E2F7F5FCF4E7CC
:10119000340000203C5706082B8B05081C06060867
:1011A00030B50023202511F8012F0AB9027030BD97
:1011B000120600F1010420D513B12023037020464C
:1011C0000B78124A03F07F036BB9013A12F8013F22
:1011D00013F0800F044600F101000BD003F07F03F1
:1011E00023700123DFE712F9014B002CFBDA013BEE
:1011F000DBB2E9E700F8013CE8E7012B04BF05702A
:1012000020460B7800F8013B0223CCE7328B05081F
:1012100038B54368194403689942054610D9037BE1
:101220001BB1084800210AF049FF01F1100424F025
:101230000704083480682146FFF735F82C60A86061
:1012400038BD00BFB017060870B504460E461146FB
:101250001546FFF7DDFFD4E901302A461844314630
:1012600025F078FD63682B44636070BD38B50129B3
:10127000044638BF01210025084621606560FEF75D
:10128000F7FF2573A06038BD38B505460C4601311F
:10129000FFF7ECFF6C6038BD0023C0E90132012389
:1012A000016003737047000038B514460546FFF728
:1012B000DDFF024B2560636038BD00BF49120208A4
:1012C000037B10B5044613B98068FEF7F9FF0023CD
:1012D000A36010BD38B505461020FEF7C9FF2946AA
:1012E0000446FFF7C3FF204638BD10B5044648B199
:1012F000037B13B98068FEF7E3FF2046BDE810408A
:10130000FEF7DEBF10BD000038B5037B04460D4676
:101310001BB1074800210AF0D1FE0168806829440A
:10132000FEF7C1FF2368A0601D442560184438BD46
:10133000B017060838B504460D46FFF769FFD4E933
:1013400001301D446560184438BDD0E900239A423D
:1013500010B5044602D10121FFF7D6FFD4E90132CE
:101360000021D154A06810BD10B50C460121FFF733
:10137000E1FF047010BD7F29F8B50C46CEB204D849
:101380000121FFF7D7FF0670F8BD06F03F06B1F563
:10139000006FC1F3871546F0800607D20221FFF7E0
:1013A000C9FF65F03F0505704670EDE705F03F05A4
:1013B000B1F5803FC1F3073745F0800508D203211E
:1013C000FFF7B8FF67F01F07077045708670DBE70F
:1013D0000421FFF7AFFFA40C07F03F0764F00F04F0
:1013E00067F07F07047047708570C670CCE738B52A
:1013F000054608460C4625F0FFFC214602462846D5
:10140000BDE83840FFF720BFF8B54768B942044649
:1014100028BF39460D4611461646FFF7F9FEA36868
:10142000A81959197A1B184425F094FC6368A06820
:10143000334463602844F8BD43688B422CBF591A7B
:1014400000214160704738B50446154662688A42FB
:10145000084603D929448A4201D8606038BDA36890
:10146000521A1844194425F075FC63685B1B6360CD
:10147000F4E70346007893F90020002A0ADA00F026
:101480007F004022104206D113F8012F02F0C00164
:10149000802904D0704720EA02005208F2E702F0E7
:1014A0003F0242EA8010EFE7431C184601330278FE
:1014B00002F0C002802AF8D070470346002099420B
:1014C00000D8704711F8012D02F0C002802A18BF21
:1014D0000130F4E703460144002099421A4600D83F
:1014E0007047127802F0C002802A03F1010318BF8E
:1014F0000130F2E77F289DBF024B185CC0F340002B
:10150000002070474B0606087F289DBF024B185CE1
:10151000C0F3C000002070474B0606087F289DBF1F
:10152000024B185CC0F38000002070474B06060891
:101530007F289DBF024B185CC0F3801000207047CD
:101540004B0606087F2809D8064B1B5C13F00C0FCE
:1015500006D1A0F15F035842584170470020704700
:10156000012070474B0606087F289DBF024B185C80
:10157000C0F30010002070474B0606087F289DBF6F
:10158000024B185CC0F34010002070474B06060861
:1015900008B50246FFF7E8FF02EB401008BD08B5AA
:1015A0000246FFF7EBFF404220F01F00104408BD49
:1015B0003038092884BF20F020000738704710B564
:1015C00002460144E5240020914203D8B0FA80F09D
:1015D000400917E012F8013B30B103F0C003802B43
:1015E00011D10138C0B2EFE7BF2B09D9F72B09D8C9
:1015F000DB0803F0060344FA03F303F00300E3E718
:101600001B06E1D510BD0020FCE7023981420B46E4
:1016100003D31A880239002AF8D00233181A40106E
:101620007047B2EB131F70B504464FEA131019D977
:1016300001EB4001101A03F00F0302462646012A6F
:101640000CBF0D880D68013A25FA03F526F8025BF8
:1016500001F10201F3D104EB400434F8023C03B978
:10166000013870BD0020FCE7F0B5059C0025121B79
:101670002E46AC420FD101EB4403174600EB440465
:10168000411A9FB904EB420316B124F812600233E9
:10169000181A4010F0BD31F8157033F815C06744C2
:1016A0003E4420F81560360C0135E2E71D883544CC
:1016B0005D522E0C013F0233E3E7F0B4049F002695
:1016C0000D463446D11BB7420BD105EB47030A4602
:1016D00000EB4707451B7AB907EB4101F0BCFFF768
:1016E00094BF35F816C033F816206444A41A20F8C5
:1016F000164024140136E6E71E8834445C53013A50
:1017000024140233E7E72DE9F043079CDDF828E0D5
:10171000DDE908760239154684464FF6FF78A4EBDA
:10172000020955B900EB42011FB1012320F8123024
:101730000231BDE8F043FFF768BF31F8024F013DC9
:101740004444264405EB0904A5422ABF33F8024B62
:101750004FF6FF744444744486EA040E17FA8EF779
:101760002CF8027B4FEA144E360C3F0CD9E738B503
:1017700002290446806838BF02210D4618B123684B
:10178000B1EB930F07D96900FEF78DFD2368A060C8
:1017900065F39F03236038BD38B504460C20FEF77F
:1017A00067FD23682278054602F00102C3F39D001D
:1017B00023F0030313432B6063686B604000FEF764
:1017C00057FDA8602268A168C2F39D02520025F06F
:1017D00091FA284638BD994210B511D313D800EBC1
:1017E000410002EB410209B9084610BD30F8023D44
:1017F00032F8024D1B1B002B02DB04D10139F2E74A
:101800004FF0FF30F1E70120EFE710B5044638B1A3
:101810008068FEF755FD2046BDE81040FEF750BD3C
:1018200010BD70B505460C460221FFF7A0FF002C45
:101830002B78B4BF0122002262F30003AA682B7048
:10184000B4BF61422146012388B2090C14461E46EA
:1018500022F8020B03F10103F6D16E60208070BD07
:101860000023C0E900338360704728B103789B07E9
:1018700002D48068FEF724BD704738B504460D4693
:101880004968FFF774FF2A782378A06862F30003A1
:1018900023706A686260A9685200BDE8384025F08C
:1018A00029BA0A4629B90178426062F30001017041
:1018B0007047FFF7B6BF08B5FFF7D2FFBDE8084095
:1018C000FFF7EFBF920042F0020210B40260002264
:1018D000C0E901215DF8044B1946FFF7E2BFF8B5F6
:1018E0009DF8187014461D4604210646FFF73FFF79
:1018F00022462B4627B1002D0CDA624265EB4503E8
:10190000317867F3000131700021716052EA030100
:1019100002D1F8BD0027F3E7D6E901104C1C746032
:1019200020F81120120C42EA03421B0CEEE72DE9CD
:10193000F3418DED010A019D0378EA0F62F3000384
:101940000370C5F30F4313F4FF4380460BD198F89F
:10195000003023F0010388F800300023C8F8043079
:1019600002B0BDE8F081B3F5FF4FF0D0C5F3C75426
:10197000A4F17F06002EEADB05D1012102B0BDE80B
:10198000F041FFF74EBF162EC5F31605A4F16F0701
:10199000D8BFC6F1170645F400054FEA2717D5BF93
:1019A000F540963C00260936D4BF3446241139460A
:1019B000C8BF06F00F06FFF7DAFEC8F804702CB1B6
:1019C000D8F808006200002125F0D8F94EB1D8F807
:1019D000083005FA06F223F81420C6F11006F54087
:1019E0000134A742BCD0D8F8083023F814502D0C8D
:1019F000F6E72DE9F84304468F18C2F35B020D4663
:101A0000511C9846089EFFF7B2FE237868F3000346
:101A10002370AC4600221FFA86FEBC456046626019
:101A200002D3401BBDE8F8830178A1F13003092BF4
:101A30000CF1010C05D9A1F14103192B12D8A1F128
:101A40003703B342EDD2A06890468146B8F1000F4B
:101A50000FD100EB420113B120F812300231091A04
:101A60004A10DAE7A1F16103192BDAD8A1F1570383
:101A7000E7E7B9F800100EFB013329F8023B08F143
:101A8000FF381B0CE2E7F8B5044615461E46C1B107
:101A9000531E1E444FF0FF37E9000F31090920465D
:101AA000FFF765FE2378002123F0010323706160B6
:101AB0000B4645B9A06800EB4101FFF7A6FD606049
:101AC000F8BD0127E8E700220F2B08DC30789840AA
:101AD0000243013D92B203F108033E44F4D1A068F1
:101AE000013100EB41006160103B20F8022CE0E77F
:101AF00038B505780B7805F0010203F001030446C0
:101B0000981A08D1D1E90132D4E90110FFF763FE38
:101B1000EB0748BF404238BD884210B5044601D0AB
:101B2000FFF7ABFE237823F00103237010BD88423A
:101B300010B5044601D0FFF7A0FE63683BB12378DF
:101B4000C3F3000282F0010262F30003237010BDB0
:101B500088421FB5044601D0FFF78FFE626862B964
:101B600001212046FFF703FEA26801231380636072
:101B7000237843F00103237010E02378D9070FD5B1
:101B800023F00103237001230093A168ADF80E3008
:101B900008460DF10E03FFF790FD606004B010BD24
:101BA000511C2046FFF7E3FD01230093D4E90121F6
:101BB000ADF80E3008460DF10E03FFF755FD6060DD
:101BC000D6E74B682DE9F04705460E46144603B1AB
:101BD0002AB931462846BDE8F047FFF74EBE02F16C
:101BE0000F014FEA111803EB1111FFF7C0FDD6E901
:101BF000012308EB0207A96807F1004014F00F0465
:101C000000F1FF3008BF10244FEA400901EB40000B
:101C100003EB4203114686464FF0000CC4F110045A
:101C200009BB6FF001035A4383182CFA04FCC8F176
:101C3000010820F802C003EB48034FEA48021846A7
:101C4000524225F09BF809F1020903464B4417B1B3
:101C500033F8022D9AB16F6032782B7862F300036B
:101C60002B70BDE8F08733F802AD4AEA0C0C2CFA71
:101C700004FA2EF802A94FEA0C4C0139D0E7013FD3
:101C8000E5E72DE9FF410D4649680646144601B1D6
:101C900032B92946304604B0BDE8F041FFF7EDBD4A
:101CA000FFF765FDB768D5F808806A6823464146A6
:101CB0003846FFF7B6FC70602978337861F300038B
:101CC0003370DB0702460AD500236968ADF80E3091
:101CD0002009994201D0834204D181420AD804B03C
:101CE000BDE8F08138F813509DB101238142ADF871
:101CF0000E3012D904F00F04012338F8101003FA43
:101D000004F4013C214206D1BDF80E30002BE6D090
:101D100003E00133DDE7ADF80E30012312B93B805B
:101D20007360DCE7009339460DF10E033846FFF788
:101D30009BFC7060D3E72DE9F3410D465768D1F85D
:101D400004803B46144606469268A8684146FFF761
:101D500042FD01301EBF23462C461D4623782A78BB
:101D600083EA020318BF4746DB0719D4791C3046C3
:101D7000FFF7FDFC6B680093D4E90121AB68B06804
:101D8000FFF772FC70602378327800280CBF0023C4
:101D900003F0010363F30002327002B0BDE8F0818A
:101DA00039463046FFF7E3FC6B680093D4E9012124
:101DB000AB68B068FFF781FCE4E72DE9F3410F461B
:101DC0004E68D2F804801446434631469268054670
:101DD000B868FFF700FD01301EBF23463C461F4692
:101DE00023783A7883EA020316BFB046012600261C
:101DF000DB0719D508F101012846FFF7B8FC7B681D
:101E00000093D4E90121BB68A868FFF72DFC686046
:101E100018B1207800F0010070402B7860F30003C7
:101E20002B7002B0BDE8F08141462846FFF79FFCC9
:101E30007B680093D4E90121BB68A868FFF73DFCEB
:101E4000E5E74B682DE9F04F0C4651688B4215468B
:101E500021BF2546194613461C462B78DB0785B063
:101E6000064622D4237813F001071ED1FFF77FFC2A
:101E7000D4E9011CB068AD683B4699420CD100EB37
:101E80004101FFF7C2FB00237060327863F3000268
:101E9000327005B0BDE8F08F35F813203CF81340E0
:101EA000224020F813200133E7E701313046FFF7E5
:101EB0005EFC2F782378D5F804C0B068A26887EA62
:101EC0000301C94301F0010E41F3000189B207F09B
:101ED000010947F300070291B9B20191A968A1F184
:101EE0000208616803F0010A43F300039BB2A1EB0F
:101EF0000C0100936746834603918FB900EB4C01B8
:101F0000BEF1000F03D0012320F81C300231FFF78F
:101F10007CFB706022782B78C2F300021340B4E798
:101F200038F8021F019B5940039B013F8944D9198E
:101F30008F4225BF32F8021B009B009959408A440A
:101F4000029B09EA0A0159401EFA81F12BF8021B93
:101F50004FEA1A4A4FEA19494FEA114ECDE72DE9E7
:101F6000F84F4B680D4651688B42144621BF2C46F2
:101F7000194613461D462378DB07064631D42B78D5
:101F800013F001072DD1FFF7F2FBD5E9012EA06870
:101F90006468D6F808C0A41A3B469A4213D10CEBE9
:101FA0004203214600EB4202ACEB0000A1B903EB77
:101FB0004403A3EB0C0358103378706061F3000303
:101FC0003370BDE8F88F30F813103EF813502943F2
:101FD0002CF813100133E0E715881552013902324D
:101FE000E4E701313046FFF7C2FB27782B786168C0
:101FF000B068A468D5E901E203F0010947F30005E0
:1020000043F3000307F00108ADB29BB2A4F1020C48
:102010000F4683464FF0010AAEEB010E2FB900EBDD
:102020004101FFF7F2FA0121C6E73CF8024F013FF8
:102030006C40A0440EEB0704A7422ABF32F8024BC3
:102040001C465C40A14448EA0904E4431AFA84F4BB
:102050002BF8024B4FEA19494FEA18484FEA144A45
:10206000DCE74B68F0B50D4651688B4224BF19463A
:102070001346144624BF2C461D4627782B785F4014
:1020800017F0010785B0064636D1FFF770FBD4E99B
:1020900001212478B06814F00104D5E9015324D15A
:1020A000521BA54212D101EB4503144600EB450536
:1020B000411AACB905EB4201FFF7A7FA00273378C4
:1020C000706067F30003337005B0F0BD31F8147031
:1020D00033F814C087EA0C0720F814700134E0E7E5
:1020E0001F885F52013C0233E3E7CDE90277CDE977
:1020F0000057FFF708FBE1E70131FFF738FB2B78CA
:10210000DB4303F0010303932378DB4303F0010374
:102110000127029301976B680093D4E90121AB6812
:10212000B068FFF7F0FACAE72DE9F04F4B6885B0C9
:1021300004460E4615460BB1536843B9237823F085
:10214000010323700023636005B0BDE8F08F814276
:102150002DD1FFF721FBA542064607462ED06B681E
:10216000716820461944FFF702FB2268A068C2F399
:102170009D025200002124F001FEB368D4F808E06B
:10218000D6F804900193AB68029300226B68039326
:102190000EEB4908F4461146039B934233D0DDF819
:1021A00004B0CDF80090ACF1020000231AE08242A6
:1021B00006D1FFF7F1FA05460746D0E70546CEE718
:1021C0000027CCE730F802AF53441946029B3BF896
:1021D00002AB33F8123003FB0A1300990380013974
:1021E0001B0C009100990029ECD14146881C13B1C9
:1021F000A8F800300146A1EB0E0149100CF1020CC9
:1022000001328046C8E761602A78337853402278EB
:10221000384663F30002227005B0BDE8F04FFFF7C7
:10222000F4BA4B6870B50546144613B11378DA0753
:1022300006D52B7823F001032B7000236B6070BD53
:10224000636823B9BDE870400121FFF7EABA084688
:10225000FFF7A2FA06462046FFF79EFA0121044640
:102260002846FFF7DEFA636883B1A3681B88DB07A3
:1022700004D5324629462846FFF756FFD4E9012106
:1022800001230846FFF7CDF9606038B93046FFF703
:10229000BCFA2046BDE87040FFF7B7BA3246314677
:1022A0003046FFF741FFDEE72DE9F04F0C4651685D
:1022B0008FB09346013105460393FFF758FADBF8D8
:1022C0000420A86801325200002124F057FD2B7829
:1022D000002623F001032B706E60DBF8041020460B
:1022E0000131FFF744FA59462046FFF7C6FA039B2F
:1022F000D4F80890D4F80480D3E901370293AB688E
:1023000004933A46029B41464846FFF764FA002888
:1023100033D1049A6060012313806B602378626874
:10232000002A0CBF002103F0010161F300030399AF
:1023300023709BF8003009784B40DB0740F1FD80AB
:102340006B682978003B18BF012363F300012970F3
:10235000002A00F0F2800BA84FF0FF31FFF7ABFA34
:102360000BAA29462846FFF7E6FC039A2146204699
:102370000FB0BDE8F04FFFF7DEBC013001D16E6059
:10238000CCE7029B03F10042013A4FEA420A37F8D8
:10239000121033460E0403F101004ED59BB209EB37
:1023A00048014FF0000C08F10100C3F1100629F8B4
:1023B00018C0019160600231CE4605968E4540D32B
:1023C00037F812209A400592029A012A09D907EBA0
:1023D0000A02C3F1100132F8022CCA4005991143D8
:1023E0000591029A801A6860049A00F10040013851
:1023F00002EB400207920AF102020992BA1E089209
:10240000D4F804A0029A524529D30AF1004A0AF1ED
:10241000FF3A09EB4A0A0022C3F11000D14573D9F3
:102420006FF000416B682BB104985A1830F81220F5
:10243000002A73D06FF0004175E0490089B203466D
:10244000A8E7BEF8008008FA03F64CEA060C059EE1
:102450002EF802CB28FA06F81FFA88FCAEE7019A9C
:102460000198118832F8022C42EA01420599B2FB28
:10247000F1F20999411A06910899069F00200E462B
:1024800086460199B9420DD809880844A8BB079926
:1024900021F80229019A0791023A01920AF1FF32CA
:1024A0006260ADE736F8021FB7F80080994041EA54
:1024B0001E4E1FFA8EF1514318FA80F81FFA81FC64
:1024C000090CA8EB0C0CC1EB204127F802CB01EB67
:1024D0002C40D6E738F8021F994041EA1E4EBCF85E
:1024E0000010394411FA8EF12CF8021B0F0C0199DF
:1024F0006145EFD83844013AC8E70027DDF820806D
:10250000DDF818C0BE46F2E7BAF8001041FA03F64B
:10251000324381402AF802298AB27FE7013B6B608F
:1025200080E7013B63606368002B3FF4F7AE5A1805
:1025300039F81220002AF4D0F0E60FB0BDE8F08F91
:10254000F0B51F464B6885B004460D4616464BB1A4
:102550001378DA0706D47B68012B0BD1BB681B8884
:10256000012B07D1237823F001032370002363603C
:1025700005B0F0BD01212046FFF753F97368002B29
:10258000F6D02846FFF708F905463046FFF704F96C
:102590000023CDE90133064603937368B3B1B368F2
:1025A0001B88DB070AD52A4621462046FFF7BCFDDB
:1025B0003B462246214601A8FFF776FED6E90121D7
:1025C00001230846FFF72DF8706058B901A8FFF7FE
:1025D0004CF92846FFF719F9304605B0BDE8F04040
:1025E000FFF713B92A4629462846FFF79DFD3B46CB
:1025F0002A46294601A8FFF757FECEE710B5D0E9D5
:102600000121034601EB42020020914204D31B78D2
:10261000DB0748BF404210BD32F8024D44EA00409B
:10262000F3E730B5D0E90124002304EB42029442E1
:1026300006D30278D20748BF5B420B60012030BD51
:10264000B3F5004F04D232F8025D45EA0343EEE7EA
:102650000020F4E7037813F0010310B510D1D0E99E
:10266000012404EB4202944202D30B60012010BD0E
:10267000B3F5803F04D232F8020D40EA0343F2E79B
:102680000020F4E72DE9F74FDDF830C0019206464F
:102690000F4609B30CEB0300D6E9018901240021A0
:1026A0001A46A2468E46B8F1000F17D101990029AB
:1026B00045D0002A43D1002B41D0002F3BD09CF8BD
:1026C00000302CB13478DB4384EAD31404F00104E5
:1026D000204603B0BDE8F08F6046DDE739F8025BC5
:1026E0000EF1100E45EA0141BEF1070F02DC08F1C0
:1026F000FF38D8E796F800B08DB21BF0010F1FBF6E
:10270000ED435AFA85FA1FFA8AF5CAF3072A42B945
:102710001CB1EDB2B5FA85F46409AEF1080E090AF0
:10272000E2E7EDB227B100F8015C0138013AF4E7C5
:1027300000F8015BFAE7634413F8013CC1E7337822
:1027400013F0010F14BFFF210021002F18BF6046B6
:1027500024F014FBBCE70000D0E901329FED0C0A25
:102760009FED0C7A02EB43039A4205D30378DB0713
:1027700048BFB1EE400A704733F8021D07EE901AC9
:10278000F8EEE77AE0EE077AB0EE670AECE700BF12
:1027900000000000000080472DE9F74F0A29446837
:1027A0009DF830A00D9E154614BF042203228046DA
:1027B00089460092A4B98DB1013D324615F8011F3A
:1027C000134641B930221A70002203F8012F981BDA
:1027D00003B0BDE8F08F02F8011BEFE73346F1E7E5
:1027E000640020460193FDF743FDD8F80810224607
:1027F000074624F07FFA019B3046B34607EB040CF2
:102800003A3BACF102040021A742A6461DD9303163
:1028100039295C4688BFC91804F8011B39468C4524
:102820008E461DD83846FDF74BFD65BB98F8003045
:10283000DB0744BF2D2304F8013B3346621E9A4256
:1028400033D800232370A01BC2E7BEF800E04EEA95
:10285000014EBEFBF9F124F8021909FB11E1D3E79F
:10286000BEF800200231002AD9D0BAF1000F08D0FA
:10287000009A211A914204D10BF102048BF801A0B5
:102880002046A346BDE7284624F0B6FA29185A4642
:102890000B46AB4204D88D4288BF00200444C5E7F4
:1028A00013F8017D02F8017FF3E71978107803F837
:1028B000010B02F80119C2E7D0E9023293423DBF91
:1028C0005A1C826018784FF0FF3070470368013B54
:1028D000033310B5044602D84068FDF7F1FC2046EA
:1028E000BDE81040FDF7ECBCF8B5054610200C46DD
:1028F0001F461646FDF7BCFC054B8460C0E900741A
:102900003444C4606B60034B2860AB60F8BD00BF0B
:10291000B9280208CD28020802690A2AF8B5044637
:102920001BD18369013383610123E361237D23612B
:10293000637D237500260A27256EB5B16B1CA26D39
:102940002366555D626D934201D366652666237DDD
:102950000D2B14D0BDB16575F8BDC369092A04BF3C
:10296000073323F007030133DFE7D4E90103984776
:10297000431CECD0012838BF01200546E7E70A2DAB
:102980002775D9D0E6E7237D002BE4D00A2B18BFAA
:102990000A25E0E701692729024601D0222912D140
:1029A000012024E0137D272BFAD0222BF8D07229A6
:1029B00014D1662B16D1507D2728F1D0A0F1220327
:1029C000584258417047A1F16200132804D8084BBF
:1029D000034113F00100E5D000207047662904D1BF
:1029E000722B00E0622B02D1E5E76229F8D0704734
:1029F000EEFFF6FF38B504460D462069D0B10A282F
:102A000006D10DB1636AB3B12046FFF785FFF4E745
:102A1000FEF770FD0028F7D12369232B08D120464B
:102A2000FFF77AFF2369002BE7D00A2BF7D1E4E701
:102A30005C2B02D00025284638BD237D0A2BF9D116
:102A40002046FFF769FFDFE72DE9F04F002304463A
:102A500085B001214364FFF7CDFF276AA369636353
:102A6000002FE369A36307DA072384F83C300137BA
:102A7000276205B0BDE8F08F04D0062384F83C300F
:102A8000013FF5E7002835D039462046FFF7B2FF71
:102A9000052384F83C30D4E90B3003F10042013ABD
:102AA000E56930F81220013D9542E2D009D8013B9A
:102AB00030F81320954218D3DBD0022384F83C3041
:102AC000D7E7A16A8B4207D308314900FDF7EBFB3A
:102AD000A36A20630833A362E36A5A1CE26220F807
:102AE0001350236A01332362C3E7226AE362013A87
:102AF0002262DCE7256915B984F83C50B9E7204625
:102B0000FFF748FF0646002800F00C8284F83C706E
:102B10002369722B6CD008D8622B0CD0662B71D035
:102B2000B9460025A8460B230EE0753BD3F10009FA
:102B300049EB0309F5E7237D722B4FF0000569D0BF
:102B4000A8464FF001090C2394F83C20002A6AD1D2
:102B500084F83C30B9F1000F08D02046FFF7DCFEC6
:102B6000B9F1020F02D12046FFF7D6FE2369222BCE
:102B70000CBF2223272320460193FFF7CDFE2369B4
:102B8000019A934240F08680237D934240F08280F8
:102B90002046FFF7C1FE2046FFF7BEFE4FF00309B7
:102BA00035B1A36E23B9A64904F16400FEF71FFCFA
:102BB00004F140034FF0000B02932169002900F05B
:102BC000A881B9F1010F02D10A2900F0A281CB45F9
:102BD00063D3594604F14000FEF72EFC0121204644
:102BE000FFF708FF2046FFF7D5FE002890D11CE034
:102BF000237D622B0DD0662B10D00025B0464FF000
:102C0000010990E7237D722B354608D04FF000086C
:102C1000F5E70025B0464FF0020994E73546B04687
:102C20004FF002097FE79A4294D0A36E002B3FF445
:102C300020AF292104F16400FEF796FB236E04F116
:102C40005006002B40F06B8103213046FEF772FBEB
:102C500023690370237D4370637D8370D4E91A5721
:102C6000216E2A463046FEF7CFFB2A46394624F02D
:102C700041F80023A366236EA26D581C2066D15C28
:102C80002161991C2166105C207503332366535C17
:102C90006375EEE64FF0010982E7019B8B4209D193
:102CA000029819460BF1010BFEF765FB2046FFF772
:102CB00033FE82E7002D60D15C2940F02781204659
:102CC0000391FFF729FED4F810A00399B8F1000F83
:102CD0006CD00298FEF74FFBD346D2E004F1640BB0
:102CE00028215846FEF740FBD4F868A0002221694D
:102CF00079B172BB3A290CD07D290AD0212928D17B
:102D0000207D7238012829D8607D3A2801D07D289D
:102D100024D1D4E91A21881810F8010C3D2809D1D2
:102D2000A2EB0A02514404F14000FEF78DFAA26EB4
:102D3000013AA266924508BF0423584608BF84F8AA
:102D40003C302921FEF710FB2C215846FEF70CFBE6
:102D500024E021F020005B280AD10132C9B2584694
:102D60000392FEF701FB2046FFF7D6FD039ABEE76C
:102D70005D2808BF02F1FF32F0E77B299CD1204695
:102D80000391FFF7C9FD23697B2BA7D104F1400014
:102D90000399FEF7E9FA2046FFF7BEFD7B2104F117
:102DA0004000FEF7E1FA4FF0000B06E7BAF1780FAA
:102DB00009D8BAF15B0F0AD8BAF1220F53D029D83B
:102DC000BAF10A0F23D05C2104F1400082E7AAF196
:102DD0005C021C2A73D8DFE802F046727272728AB3
:102DE0002A7272723A727272727272723072727285
:102DF0000F722D3D37725C004FF00D0B94F83C3094
:102E00000B2B77D1594604F14000FEF7B4FA4FF08E
:102E1000000B4BE7BAF1550F1CD0D4D8BAF1270FED
:102E200021D0BAF14E0F4AD106480AF035F94FF0D9
:102E3000080BE3E74FF0090BE0E74FF00A0BDDE783
:102E40006DB5050876B505084FF00B0BD6E74FF0CA
:102E50000C0BD3E794F83C200C2A06D15C2104F13A
:102E60004000FEF788FAD346C8E7BAF1750F14BFE1
:102E70004FF0080A4FF0040A4FF0000BBAF1010AB4
:102E80000AD2BBF5881FB9D34FF0010384F83C3058
:102E9000BDE74FF0020AEFE72046FFF73DFD22694C
:102EA00003921046FEF744FB002800F05081039A7D
:102EB0001046FEF77DFB4FEA0B1B8344DEE7AAF1C9
:102EC000300BBBF1070F3FF67EAF4FF0030A06E071
:102ED0002046FFF721FD2269303A02EBCB0B227D21
:102EE000303A072ACDD8BAF1010AF1D1C9E74FF03B
:102EF000070B83E7BBF1FF0FC6D80C2BC4D15FFAD9
:102F00008BF104F14000FEF72FFA80E70298C9B276
:102F1000F9E7CB453CBF032384F83C3059E6033B3B
:102F200023669BE62846FEF7EFFA2169D8B95F29A8
:102F300019D07F2917D80846FEF7F0FA002855D196
:102F400023692E2B4DD0844D00262F781FB1236985
:102F5000BB4240F0A4802046FFF7DEFC002F40F08B
:102F6000A6800123AAE5082384F83C3004F140053B
:102F7000C9B22846FEF7F8F92046FFF7CDFC2069D4
:102F8000D8B92846FEF7E1F9744F0646002557F8F0
:102F9000041B304623F03EFF00281CD10E35EDB255
:102FA000112D84F83C507FF464AD6D4BD3F818328A
:102FB000002B14BF0E23102380E5FEF7A5FA40B9BD
:102FC00020695F2805D07F2803D8FEF7A7FA0028DC
:102FD000D7D0217CCDE7FFF64CAD0135242DD6D1DD
:102FE00047E5207DFEF79AFA0028ACD021692E290A
:102FF0002AD10A2384F83C30002504F140063046EB
:10300000FEF7B9F92046FFF787FC0A272069002858
:103010003FF42FAD55BB20F02003452B26D1652171
:10302000304684F83C70FEF7A6F92046FFF774FCA2
:1030300021692B2901D02D29E8D13046FEF79BF9D3
:103040002046FFF769FCE1E70923302984F83C308A
:10305000D2D1237D43F02003623BDBB2162BCBD8C9
:10306000404DDD4015F00105C7D1C5E7FEF74CFA2C
:1030700028B121692E290DD184F83C70DDE7206943
:10308000FEF74CFA0028F4D123692E2BF1D05F2BE8
:10309000D6D0EEE421F020034A2BCED1ECE7652F09
:1030A00001D0632F00D10135013601354DE7212FC5
:1030B00008D123693D2B7FF454AF2046FFF72CFC49
:1030C0003923FBE42E2F0FD123692E2B02D1237D30
:1030D0002E2B01D05C23F1E42046FFF71DFC204697
:1030E000FFF71AFC0D23E9E40335334615F8027C9B
:1030F000632F18D0652F16D01B4AD35C84F83C3060
:10310000543BDBB2052B3FF6B4AC012202FA03F3C9
:1031100013F02A0F18D113F0150F3FF4AAAC636A0D
:1031200013446362A5E415F8012C2169914206F16C
:10313000010607D12046FFF7EFFB3346652FDBD0B2
:103140000235D3E7632FFAE7636A013BE9E701231E
:1031500084F83C30834651E628B50508CC060608BD
:1031600034000020012040005C0706087FB50646B9
:1031700001AD742085E80E00FDF77AF80446034699
:1031800095E8070043F8046B83E8070001236FF01C
:1031900001020025C4E906320A22C4E90A23C4E96F
:1031A00008551420FDF764F82021206304F1400045
:1031B000FEF75CF8294604F15000FEF757F829465F
:1031C00004F164002566FEF751F8236B20461D804C
:1031D0002561A582FFF7A0FB2046FFF79DFB204657
:1031E000FFF79AFB2046FFF72FFCA36B012B06D0BD
:1031F00094F83C30052B1CBF062384F83C30204655
:1032000004B070BD30B585B001AC05462046FFF76F
:103210006BFB94E80E002846FFF7A8FF05B030BD11
:1032200030B585B001AD04460146284620F0A8FC23
:1032300095E80E002046FFF799FF05B030BD10B5A8
:103240000446B0B1C3684068984704F14000FEF7F7
:1032500037F804F15000FEF733F804F16400FEF78C
:103260002FF8206BFDF72CF82046BDE81040FDF745
:1032700027B810BDD0E90432013B036152F82300A6
:103280007047036942695B1A013B52F8230070479B
:10329000F8B5446A06460D46B4B1D4E900030B44C0
:1032A000834222D90831002201442046FDF706F866
:1032B0000246B8B9616820460831FCF7FFFF636831
:1032C0002360336A63603462802D2F4638BF8027C5
:1032D00007F10800FCF7CCFF0023076043600446B9
:1032E000706202E023682B442360606805446560D7
:1032F00008342044F8BD38B50D460C211446FFF7BC
:10330000C7FF4FF49D72C0E90124056038BD38B590
:10331000D0E903329A4204460D4608D3103399008F
:103320004069FCF7C0FFE36860611033E360D4E9F3
:103330000432591C216142F8235038BDF8B50446C7
:103340001D46D0E9000383420F46164608D31030CD
:10335000C100A068FCF7A7FF2368A06010332360BA
:10336000D4E90103421C626053F8301067F317017F
:1033700043F8301003EBC002D6705560F8BD10B4AE
:103380008469CAB20023616B5DF8044BFFF7D6BFB6
:10339000F0B593B0044668460E4617461D46FCF746
:1033A00027FF10B1002013B0F0BD3A463146204649
:1033B00009F0ACFC0446FCF7F1FEA30703D1226838
:1033C000024B9A42EED02C600120ECE7281406084C
:1033D00010F00102034604D040F001030B6001200D
:1033E0007047A8B110F0030013D11A793A2A11D10D
:1033F0009B680B6013F00100F1D19A070AD118689D
:10340000054B9842EBD0054BC31A584258417047C0
:1034100070471046704700BF141D0608BC1A060806
:1034200010F001021CD110F003030CD000F00F03C8
:10343000062B15D00A2B11D100090D3803288CBF9B
:1034400000200120704770B102793A2A08D02D2A55
:1034500008D18068B0FA80F0400970471046704784
:103460000120704718467047C20702D540F001009E
:103470007047830710D0030900F00F00062803D11E
:10348000D80040F002007047A3F10E00022809D8CE
:10349000064B53F82000704730B103793A2B03D123
:1034A00080687047024870470248704788070608DE
:1034B000DC2306081028060838B505460C46FFF739
:1034C000AFFF38B12846FFF7CFFF0AF0FDFD031B21
:1034D0005842584138BD2DE9F0410F460546144683
:1034E000114689B9204612F0D7F9014600F10808C3
:1034F000A4B90A4628463946FFF7FDFE014628468C
:10350000FFF705FF012007E001392846FFF7B9FE64
:10351000FFF786FF0028E4D1BDE8F0812846FFF7D9
:10352000A9FE0646FFF7A0FF013C48F82400002E44
:10353000DED0B307DCD1686A00F108039E42D7D31E
:10354000426813449E42D3D273681B0A0233A2EB33
:1035500083024260CCE70000F7B5866996F83C200C
:10356000A2F1080305460F46042B52D8DFE803F00A
:1035700003232B384C00D6E91110FDF7D7FC902F10
:1035800004460ED1C100002241F0020105F12800DD
:103590000AF030F928B14268D3071CD542F0010087
:1035A00002E0200140F002000146284603B0BDE8D9
:1035B000F040FFF7ACBE0022D6E911103346DFF72A
:1035C0000DFD0246E8E70096D6E91110002301221E
:1035D000DFF73CFE0246716B2846FFF78CFEE3E7FF
:1035E000D6E911100A2906D8FDF7A0FC30B1000178
:1035F00040F00600D8E7FDF74BFCF7E7D6E91121CC
:10360000064810F031FAE5E7D6E9111010F00CFB8E
:10361000E0E7120142F00A00C6E700BF04270608EF
:1036200010B5FFF7D5FE50B10B6813F0010007D1BC
:103630009A0704D11868034BC31A5842584110BD69
:103640000120FCE7141D06080021FFF735BF01210A
:10365000FFF732BF2DE9F04F2D2A85B0044688468A
:1036600016461D460BD10021FFF70BFEC0B18207A5
:1036700002D10379922B13D005B0BDE8F08F922AC6
:103680002ED10021FFF7FDFD014648B1830707D188
:103690004768FBB2952B18D12046FFF7EBFD013DA3
:1036A000A6F12303DFB2092F00F2EB80092B00F211
:1036B000CF80DFE813F0ED00ED00ED001E011E01EC
:1036C0001E014501ED00CD008F01962BE8D127F0BA
:1036D000FF07204647F09207FFF7CCFD4F60CBE78E
:1036E000962A13D1D0E9012303EBC203013513F865
:1036F000153C2D2B40F0AD802A46FFF7ECFE00284C
:1037000000F0A7806368023B6360B5E7A2F11E0387
:10371000012B5FD9202A00F08380052AC0D1002127
:10372000FFF7AFFD0746002800F0938010F0030A72
:1037300005D1436803F0FE03562B00F08A80012177
:103740002046FFF79EFD00F00F03022B40F0818022
:10375000BAF1000F7DD13B792C2B7AD1BB6803F0F5
:103760000F02022A75D11B09482B72D1FB68002B6E
:103770006FD09A076DD11A79302A6AD1D3F808B080
:103780004FEA10195846FFF74BFE002840F0FD8025
:10379000B749B8480CF0C0FBA1693A68096805460A
:1037A00053460CF09BFC2846FCF73AFD1E2E0AD12E
:1037B000FFF74DFF18BB3846FFF746FF00B9D34669
:1037C0000BF1FF3A0BE0FFF73FFFC0B93846FFF7B8
:1037D0003EFFF3E705F1FF3A8DB1AB46A94609F18B
:1037E000FF3949462046FFF74CFD23696269A3EB88
:1037F0000B03074642F82300B9F1000FD6D1002190
:10380000514508D16D1A012D3FF436AF362E00F028
:103810004281332E3DE12046FFF72CFD0131EFE7D9
:103820000021FFF72EFD0746FFF70EFF68B9384667
:10383000FFF70DFF68B1EA212046FFF71BFD204688
:1038400005B0BDE8F04FFFF762BD4FF48571F3E7B7
:103850002B26A91C89002046FFF71AFD46EA0523FE
:103860000746C0F80080436000F10801002D40F0D9
:103870001B81962E03D139462046FFF748FD394675
:10388000DDE7922E00F0FE80062E00F00481BDE7F9
:10389000691E2046FFF7F5FC01A9FFF799FD0028F6
:1038A000B7D0022F9ABFA6F10D095FFA89F94FF040
:1038B0002209AF1E002F09DA002D40F0CD80019AB9
:1038C000D30740F1CE8042F00101B8E739462046E7
:1038D000FFF7D7FC02A9FFF77BFD002899D0DDE9AF
:1038E000011201AB4846FFF753FD002891D0013F7C
:1038F000E0E7691E2046FFF7C4FC01A9FFF768FD59
:10390000002886D0AF1E002FD6DD791E2046FFF797
:10391000B8FC02A9FFF75CFD00283FF47AAF3946F6
:103920002046FFF7AEFC00092438DDE9011201ABA7
:10393000C0B2FFF72DFD00283FF46BAF023FE2E776
:1039400000212046FFF79DFC01A9FFF741FD00285B
:103950003FF45FAF01212046FFF793FCC0F307104F
:10396000332801990BD1CF0707D488077FF451AFD3
:103970000A68414B9A427FF44CAF022001E03F3885
:10398000C0B208F0F5FB019096E75846FFF76CFDD2
:103990004FEAC9030A46074643F0020104F1280032
:1039A00009F028FF47604846FDF785FB03785F2B49
:1039B000204608D1FFF75EFC00252046FFF75AFCA1
:1039C000A84608266CE6FFF755FC59462046FFF747
:1039D0009EFC3EE701212046FFF753FC00F00F0359
:1039E000022B07467FF415AF00212046FFF749FC64
:1039F00000283FF40EAF10F003027FF40AAF037902
:103A0000322B7FF406AF3909C900D0F808901B4863
:103A100041F0020109F0EEFE00283FF4FAAE4068E2
:103A200002AA4FEA191108F0E5FA029B002B3FF4B5
:103A3000F0AED9070AD49A077FF4EBAE1A680E49A4
:103A40008A4203D00E498A427FF4E3AE039A002AE9
:103A50007FF4DFAE01932FE72046FFF70BFC013D1B
:103A60002AE729462046FFF746FC0146E7E600BF65
:103A700004B6050868170608141D0608940706080A
:103A8000BC1A0608D4E9012303EBC20313F8053C72
:103A90002D2B7FF4DEAE2A4641462046FFF71BFD64
:103AA00000287FF4E9ADD4E62046FFF7E3FB013DB3
:103AB00041F82500DAE600BF0346006830B550B192
:103AC00084070AD14468E5B28D4206D100F10803AB
:103AD000200A136030BD0346FBE70120F9E7000030
:103AE0002DE9F04FA94B97B0CDE9073102900D4673
:103AF00005A8A74901920024FCF758FB40234FF486
:103B00000070CDE90934FCF7B3FB20230B90802033
:103B1000CDE90C34FCF7ACFB2146CDE90E0513A82A
:103B2000CDE9114409F030FE019B002B48D0022B57
:103B30000CBF3F2222460023696B964F09A8FFF76E
:103B4000FDFB00230A9C002C00F06481013C0B99D2
:103B500091480A9401EBC40251F83410D6785268A7
:103B6000C1F3170A8D4911F806B08D49895D632E9E
:103B700088BF41F4807100EB41080BF0300110293F
:103B80000BF00F091ED020294BD0002B00F01B8119
:103B9000B9F1020F40F00A81012A40D000211BF048
:103BA000010F02F1FF3306D0B8F802003840B0F53B
:103BB000805F08BF5308012B40F0E580E1B1E2E0EF
:103BC0003D22B8E702B1BBB108EB420825E0C3468D
:103BD00038F8023B03EA0701B1F5805F0ED195F892
:103BE0003C10C3F30B03994216D109A83146FFF7E5
:103BF000B3FC2846FEF728FF0023A3E7531C4B45E0
:103C000004D23246514609A8FFF798FBBBF80010D2
:103C100009A8FFF7B4FBEFE701329145D7D801239C
:103C200090E773B102F10043013B38F813303B4099
:103C3000B3F5405F21D1002109A80392FFF767FB8C
:103C4000039A08EB420491452BD8019B83B1052EC2
:103C50000ED1002109A8FFF714FB48B9012109A8DA
:103C6000FFF70FFB830744D000F00F00022845D177
:103C7000002408EB4903A1465AE0012ACFD995F860
:103C80003C30062B40F0F480464947480CF044F99C
:103C90006A6B2968044600230CF020FA2046FCF7E2
:103CA000BFFA039434F8021B01EA0700B0F5805F05
:103CB00016D195F83C00C9B288420ED1082805D12A
:103CC000314609A80392FFF747FC039A039228465E
:103CD000FEF7BAFE039A0132B5E7002A9FD0CEE77D
:103CE000531C5146324609A8FFF728FB039B19884D
:103CF0008EE70028BCD003793A2BB9D109A8FFF789
:103D0000B9FA09A8FFF7B6FA00230822514609A814
:103D1000FFF7A0FC70E733F8022D02EA0701B1F5C6
:103D2000805F10D1D2B2082A02D1013409F1010911
:103D30004345F0D1B9F1010F1CD11BF0400F19D050
:103D40000026314610E0214609A80393FFF799FAAF
:103D5000039B08B109F101090134E9E7FFF78AFA89
:103D60000136002818BF0146A64209A8F6D1FFF780
:103D7000CEFA41E71BF0800F04D0002109A8FFF71D
:103D8000C6FA013423463246C0E700BF3F3202087C
:103D9000F7BE020800F0FFFF80080608080C0608BE
:103DA000D007060810B6050844170608012A3FF494
:103DB00036AF12F001013FF4F2AEB9F1030F7FF418
:103DC0005EAF0121EBE609EA020303F0010338F8D4
:103DD000134004EA0701B1F5805F13D195F83C1058
:103DE000C4F30B04A14202F1010409D11BB931460D
:103DF00009A8FFF7B1FB2846FEF726FE2246E2E7B8
:103E00002246C5E6531C5146324609A8FFF796FAEA
:103E10002146FDE613A809F0CBFC129850B1416889
:103E200022460831FCF74AFA129B5A681A60119A26
:103E30005A60119395F83C30002B7FF420AF0D9B16
:103E4000002B3FF41CAF0E9B0B981B681093FCF7E4
:103E500037FA0E98FCF734FA0120FCF7AFF9DDE9E8
:103E60001001029B83E80300184617B0BDE8F08FED
:103E7000022B01D1034908E7042B0CBF0249034977
:103E8000034803E722B6050844B6050857B60508F7
:103E90006817060838B50446406808B9606038BD40
:103EA0004568FCF70DFA2846F7E70000F8B5054627
:103EB00030200E461746FCF7F4F9072D044605702E
:103EC000C66001D0012D0FD1B368C3F30F13A382D5
:103ED00007F093FC042320612783E3842020FCF770
:103EE000C7F9E0622046F8BD014B5B5DEFE700BF1C
:103EF000B80C060810B50446C06AFCF7E1F9204684
:103F0000BDE81040FCF7DCB930B5058D0446002251
:103F1000954201D8002030BDE36A03EBC20043683C
:103F20008B42F8D00132F3E770B504460D461646D1
:103F3000FFF7EAFFC0B9E38C228D9A4208D306331B
:103F4000D900E06AFCF7AFF9E38CE0620633E38462
:103F5000238DE26A591C02EBC300218502F833600D
:103F6000002343704380456070BD034618465B687C
:103F7000002BFBD1FFF7C8BFF8B544680E462CB93B
:103F8000F8BD042BFCD105230370F9E7254628462C
:103F90006D68002DF4D077683946FFF7B5FF00282B
:103FA000F5D00378043B022BEAD8062535700022B1
:103FB00039462046FFF7B8FF0378002BE1D10570A2
:103FC0006468F4E7036A1B8B012B1EBFC3685B1890
:103FD000C3607047836A10B504469B6F406A984778
:103FE000238B226A0133918C9BB29942238338BF81
:103FF000938410BD038B10B5013B0383836A044691
:10400000D3F88430406A984720460121BDE810402B
:10401000FFF7D8BF2DE9F04F85B004460D46039257
:1040200098461BB1CB8A43F00803CB82039BEB83FA
:10403000236ADA8A42F03002DA821B78002B46D1FA
:10404000A36A039AD3F8B460606A43462946B4462B
:1040500005B0BDE8F04F6047DB6A03EBC60B13F811
:104060003630053B012B1DD84FF0000917E0EB6AF5
:1040700003EBC90213F83930062B0ED1DBF804101C
:104080005368994209D1A36ABBF802201B69606A90
:104090001F460023B8470AF1010A09F101092B8DD7
:1040A0004B45E4DC0136236A1A8DB242D4DCBAF106
:1040B000000FC5D0A36ACDF80080D3F8B860606A5D
:1040C000039B52462946B04705B0BDE8F08F002655
:1040D000B246E8E7836A10B50446D3F88830406AF0
:1040E00000219847A36A606A1B6B0F219847A36A57
:1040F000606AD3F8CC300121984720460321BDE8FF
:104100001040FFF75FBF38B5836A04465B6C406AB6
:1041100000229847A36A606AD3F8C05000231A4669
:104120001946A8472046BDE83840FFF7D3BF836A49
:1041300089681B6D406A002209091847836A8968EB
:10414000DB6B406A184710B50446084611461A460C
:10415000FFF7ACFE236A436000238360E3690BB979
:10416000E06110BD1A469B68002BFBD19060F8E718
:104170002DE9F04F87B0054600AF0C4611B901217B
:10418000116013E011F0030619D10B79682B19D1D6
:10419000CB681B0913608C68002CF0D0012604F05A
:1041A0000F03022B0DD12109002EE9D0AB6A686AFA
:1041B000DB6A002298471C37BD46BDE8F08F002619
:1041C000EDE716B9A3681B091360A04658F8043F31
:1041D0004FEA132A08EB8A030AF1FF3BBB60C14692
:1041E00059F8040F0009FCF75BFFBB68994583444D
:1041F000F6D10BF1070323F00703ADEB030DC7F86E
:104200000CD0E946002358F8040F3B6007F1140175
:104210000009FCF75CFF7A697A600146484622F0A3
:1042200069FD3B687A6801339A454A4405D0914656
:104230004FF02E0209F8012BE5E75946F868FCF724
:1042400075FEAB6A0146DB6A686A00229847002E59
:10425000B1D00834BB689C42ADD054F8041FAB6A9F
:10426000686A1B6D002209099847F3E731B182683B
:1042700001F00303134304BF0B68836070472DE90B
:10428000F04107461E4659B111F0030510D14B68A5
:10429000D8B290420CD14FEA13280C1D454501DBE2
:1042A000BDE8F08154F8041F3846B0470135F5E702
:1042B00038463346BDE8F04118470000F8B50446DB
:1042C0000E4611461A4600238578076983700361FC
:1042D0000E4BFFF7D4FF6368BBB9618A51B1228AE4
:1042E00042B9A36A606AD3F8A0309847A36A606AAB
:1042F0001B6C9847238A628A31462046FFF78AFE64
:10430000003D18BF0125A5702761F8BD694B020863
:1043100070B54378012B05460C4606D1036A0A4660
:104320001B8B0221FFF70FFF2061A268216928463D
:104330004C23BDE87040FFF7C1BF70B5134642780B
:10434000012A05460C4604D10A460721FFF7FBFE69
:10435000A061A669E268284646233146FFF7AEFF12
:10436000B08A70BD024B89689D22FFF788BF00BFED
:1043700075500208024B89686B22FFF780BF00BFAF
:104380000D6C020838B543680D46044611464BB91A
:1043900005480BF0C1FD294660602046BDE8384065
:1043A000FFF764BF38BD00BF68170608014AFFF772
:1043B000E9BF00BF5BB605080B79092B70B50CBFD0
:1043C000858AC58A4FF6FF739D42044602D1064A8C
:1043D000FFF7D8FF218B628BA36A606A5B6F8A1A32
:1043E0002946BDE87040184768B6050838B5054647
:1043F00079B101F00F03022B0DD10C09204609F011
:104400003FF8002806DA0649064822460BF01AFE55
:104410006860002038BD044AFFF7B4FFF9E700BF29
:1044200081B60508FC16060886B6050870B5144660
:10443000054612780E4683B132B1032A04D0104AE1
:10444000BDE87040FFF79EBF032626706168286AAA
:10445000FFF78BFD00B1067070BD62B901232370B8
:10446000006A2146FFF788FD2378012BF4D1054A25
:1044700031462846E4E7062AEED0034AE0E700BFCB
:1044800096B60508A3B60508B0B605082DE9F341B0
:104490004378012B04460D461AD10B79102B0CBF23
:1044A0004FF001084FF0000808D0036A1B782BB9C1
:1044B000114A02B0BDE8F041FFF764BF01AA6D21C7
:1044C00005F10800FFF7F8FA00260746B74202D1C7
:1044D00002B0BDE8F081019B206A53F8261000224B
:1044E0000909FFF721FD4346024629462046FFF70A
:1044F0009DFF0136EAE700BFB7B605084278012AFA
:104500000B4602D1006A02F013BE816A026A406A59
:10451000203102F01CBE4278012A0B4602D1006A0B
:10452000FFF702BD816A026A406A103102F00FBED5
:1045300070B505460C4600292ED0CA0706D5836AF9
:104540005B6B4910686ABDE8704018478B0717D04D
:1045500004F00F04022C4FEA11110AD0062C0CD0E3
:10456000052919D0836A406A1B6BBDE87040C9B247
:104570001847BDE87040FFF7CEBF836A9B6BE1E749
:10458000836A0968DB68406A98472279034B2146B1
:1045900053F822302846D6E770BD00BFC00C06088D
:1045A0002DE9F74F05460C4616461F462046FFF7F5
:1045B0004BF840B16EB9AB6A9B6E3946686A03B07E
:1045C000BDE8F04F18472046FFF741F820B1002E14
:1045D000F1D103B0BDE8F08F002C48D0A30746D13D
:1045E00063684FEA132BDBB21E2B18D1DEB1043403
:1045F00004EB8B0B5C45ECD054F8041F3B46324671
:104600002846FFF7CDFFF5E75AF8041F019243460D
:104610002846FFF7C5FF09F10109019A11E01F2B98
:104620001FD1002EE3D0D5F80C8008F10103EB6018
:104630000BF1FF3304F1040A4FF00009009386F0F8
:104640000102009B4B45DFDC0BF101013B4654F8B6
:10465000211032462846FFF7A3FFAB6A41469B6A0A
:10466000ACE7202B03D1A46886F001069EE7214623
:104670002846FFF75DFFAB6A686ADB6E3A46314653
:1046800003B0BDE8F04F184738B5026A1278072A20
:1046900004460B4606D0022A04D0BDE83840144A2E
:1046A000FFF770BE9D6885B9A36A606A1B6B0F2116
:1046B0009847A36A606AD3F8CC3000219847204617
:1046C0000121BDE83840FFF77DBCAB070BD12B794A
:1046D000AF2B08D12046A968FFF72AFF2046BDE886
:1046E0003840FFF7F7BC29462046FFF721FFE0E7F7
:1046F000C9B6050870B54378CE68012B0446154647
:1047000006D1036A0A461B8B2946FFF71CFD706120
:10471000002371691A462046FFF77CFCF1682046A9
:10472000FFF706FF062D05D1A36A606AD3F888302B
:1047300000219847A36A606AD3F8BC500023AC46B6
:104740001A46BDE870400121604738B50C46054661
:10475000C968FFF7EDFEA1682846BDE83840FFF7BD
:10476000E7BE0B79342B70B504460D4610D189682D
:10477000FFF7DEFEED68AD6885B9A36A606A1B6B62
:104780000F219847A36A0422D3F8A03002211AE02F
:10479000836A406A1B6B0F219847ECE7AB071FD178
:1047A0002B799A2B13D1A36A606A1B6B0F21984750
:1047B000A9680029E6D02046FFF7BAFEA36AD3F81D
:1047C000A03004220321606ABDE8704018479B2B8B
:1047D00006D1A9682046FFF7ABFEEB689968E8E7C9
:1047E00029462046FFF7A4FECCE710B504468968A9
:1047F000FFF79EFEA36A606ADB6CBDE810400021F3
:10480000184700002DE9F7438D68044616465DB948
:10481000002A75D0836AD3F8A03002222946606A44
:1048200003B0BDE8F043184715F0030740F08A8055
:104830002B79372B13D132B1836A406AD3F8A03079
:1048400002220121984720462946FFF771FEA36AFC
:10485000606AD3F8A43003B0BDE8F04318479F2B3B
:1048600070D1EB681A79A12A5AD1A22101AA03F1C9
:104870000800FFF721F9A968804621B38B0722D1F0
:104880000B79372B1FD136B1A36A411CD3F8A03066
:10489000606A02229847A9682046FFF749FEA36A8A
:1048A000606AD3F8A43098474FF00109474510D10A
:1048B000B9F1000F24D1A36A606AD3F8A0300322B3
:1048C000791C98471CE02046FFF732FE4FF00009A4
:1048D000ECE7019B53F82710A9B18E0713D10E798D
:1048E000A6F13700464246412046FFF721FEB9F1C6
:1048F000000F11D04EB9184A29462046FFF742FD55
:1049000003B0BDE8F0830026EEE7A36A606AD3F83F
:10491000A43098470137C9E7002EFBD00F4AEBE7D8
:10492000AB685BB19A0709D11B79372B06D10422FA
:10493000294603B0BDE8F043FFF7DCBE0522294657
:104940002046F6E729462046FFF7F2FDA36A032238
:10495000D3F8A030012162E7D4B60508E5B6050812
:104960000122FFF74FBF70B50D46C9680446FFF737
:10497000DFFDA968A36A606AD3F89830C1F3071114
:10498000332918BF3F39BDE8704014BFC9B20221B6
:104990001847F8B54F680C4689680546FFF7C8FD0B
:1049A0003F0A0C3400260236B74204F1080400DC4A
:1049B000F8BD54F8041C2846FFF7BAFD54F8081C4B
:1049C000AB6A686AD3F89C3009092439C9B29847A0
:1049D000E9E72DE9F0410C464E6854F8081F0546FA
:1049E000FFF7A6FDA6F10D085FFA88F8360A012741
:1049F000B74201DBBDE8F08154F8041F2846FFF7F9
:104A000097FDAB6A686AD3F89C30414698470137F6
:104A1000EEE72DE9F0414E6804460D46360A8968F6
:104A2000FFF786FD032E83BFD4F80C8008F1010345
:104A3000E3604FF0000801277B1C9E4222DC032E1E
:104A400055D9E568606A6B1CE360A36A29469B6ED2
:104A50009847A36A606A9B6A41469847A36A606A5E
:104A60009B6801219847A36A606A1B6E9847A36AF6
:104A7000606ADB6D9847A36A606A9B6A2946BDE855
:104A8000F0411847296920460237FFF751FDB74228
:104A900007DAA36A606A5B6D9847A36A606A5B6E17
:104AA0009847EB68A26A606AD2F89C2003F00F0175
:104AB0000A2911D1C3F30713252B1ABF343BD9B2EE
:104AC00006219047B74205DAA36A606A1B6F424627
:104AD000002198470835AFE71979852901D132219E
:104AE000EFE79B680BB90721EBE73321E9E7BDE866
:104AF000F08110B504468968FFF71AFDA36A606A61
:104B0000D3F89830BDE81040032118472DE9F0474D
:104B10000D46D0F80C8055F8046F5FFA86F9A9F1BC
:104B20001E03D3F1000949EB030908F10103044610
:104B3000C360360A0027B74206DBA36A606A9B6A35
:104B40004146BDE8F047184755F8041F2046013795
:104B5000FFF7EEFCB742F0DAA36A606A1B6F4246C9
:104B600049469847E7E7000001F00F03022B70B5B4
:104B7000044612D00B79492B09D0483B082B18D892
:104B8000DFE803F0081707171717170507000123B9
:104B9000A37070BD8E680D6975B9A378002BF8D12C
:104BA000638A002BF5D020461D4ABDE87040FFF710
:104BB000E9BBD1E90265EFE7A3783BB3238A013370
:104BC0009BB2012B23820ED1618AD4E90903D1B1B2
:104BD000D3F8A03000229847A36A606AD3F8A030C7
:104BE00002220021984729462046FFF7A1FCA36A2C
:104BF000606A9B6B31099847A36A606AD3F8A43056
:104C0000BDE8704018471B6C9847E5E7638A01339D
:104C1000638229462046BDE87040FFF789BC00BF8B
:104C2000F0B605082DE9F041C568D1F80C800E46B4
:104C3000AB1C04460022D8F80810C3602B46FFF7CF
:104C4000AFFCB1682046FFF773FCA36A606A9B6EF5
:104C50006F1C39469847A36A606A9B6A2946984741
:104C6000A36A606A9B684FF0FF319847D8F80C1030
:104C70002046FFF75DFCA36A606A9B6A3946BDE87F
:104C8000F04118472DE9F047C668D0F814A0B0F8F5
:104C90001A908682B31CC36006F10108038BA0F84A
:104CA00016800446438388680D46FEF7CDFCF8B9AC
:104CB000E768A8687B1CE360FEF7C9FC20B9A36A1B
:104CC000606A9B6E41469847A36A606A9B6A394650
:104CD0009847E9682046FFF72BFCA36A606A9B6A45
:104CE00041469847A9683B4601222046FFF758FCF9
:104CF0002969C4F814A02046A4F81A90FFF718FCFC
:104D0000A36A606A9B6A3146BDE8F04718472DE9FF
:104D1000F347C668731CC360044688680D46FEF7F7
:104D200093FC0246E8B9E768A9687B1CE36020466B
:104D30003B46FFF735FC2046E968FFF7F9FBA8681A
:104D4000FEF785FCD8B92B690BB96B6923B1A36A4F
:104D5000606A9B6E31469847A36A606A9B6A3946CF
:104D6000984701AA712105F11000FEF7A5FE002762
:104D700081464F450BD169692046FFF7D9FBA36AED
:104D8000606A9B6A3146984702B0BDE8F087019B94
:104D900053F82780D8F80800FEF756FC024600BBFF
:104DA000D4F80CA0D8F808100AF10103E3602046FB
:104DB0005346FFF7F5FBD8F80C102046FFF7B8FB79
:104DC000D8F80800FEF743FCD4E909230028D6D11F
:104DD0009B6E314610469847A36A606A9B6A5146AB
:104DE00098470137C5E70000184B2DE9F041D3F88B
:104DF000187204460D463FBBC6688968731CC360C1
:104E000001223346FFF7CCFBA36A606A5B691F216E
:104E100001229847E96851B12046FFF789FBA36A50
:104E2000606AD3F8BC503A463B460121A847A36AC2
:104E3000606AD3F8C83001219847A36A606A9B6A08
:104E40003146BDE8F0411847BDE8F081340000204C
:104E500070B58D6804463DB9836AD3F8C8302946D9
:104E6000606ABDE870401847AB070ED12B795E2B06
:104E70000BD1A968FFF75CFBE9682046FFF758FBF8
:104E8000A36A0221D3F8C830EAE729462046FFF793
:104E90004FFBA36A0121D3F8C830E1E710B50446FF
:104EA0008968FFF745FBA36A606ADB6DBDE81040C7
:104EB000184700002DE9F041026A1278072A0446DB
:104EC00004D0BDE8F0411A4AFFF75CBA8D685DB9BD
:104ED000836A406A1B6B0F219847A36A606AD3F804
:104EE000C430BDE8F041184715F003021DD12B79FD
:104EF0001B2B1AD1C668EF68731CC360B9683346B0
:104F0000FFF74EFBA9682046FFF712FBA36A606A11
:104F1000D3F8C4309847A36A606A9B6A31469847C1
:104F2000F9682046FFF704FBD7E72946F9E700BFF9
:104F30000EB705082DE9F0410C46054654F8046FFC
:104F4000360A04EB8607BC4208D1AB6A686AD3F81C
:104F5000A03031460022BDE8F041184754F8041F44
:104F60002846FFF7E5FAEEE7896810B4034641B931
:104F7000826A406AD2F8A0400A4623465DF8044B94
:104F800018474A68120A022A0BD1CA684AB1940724
:104F900007D11279AC2A04D15DF8044B0622FFF741
:104FA000A9BB5DF8044B1846FFF7C4BF2DE9F041DB
:104FB0000E46054656F8043F0F464FEA13280024D4
:104FC000444501DBBDE8F08156F8041F2846FFF791
:104FD000AFFA6B683BB10234284657F82410BDE89D
:104FE000F041FFF743B90134EAE710B50446FFF793
:104FF000DDFFA36A606AD3F89C30BDE8104022212F
:10500000184770B58D68044645B9836AD3F8A03057
:1050100001222946606ABDE870401847A9071ED1E1
:105020006B68DAB2922A1AD11B0A022B0CD1EB68F8
:1050300053B19A0708D11B79AC2B05D1294603221D
:10504000BDE87040FFF756BB29462046FFF7AEFF8C
:105050006968A36A0122D3F8A030090ADAE7294671
:105060002046FFF765FAA36A0122D3F8A030114663
:10507000D0E7000001F00F03022B2DE9F0470546B1
:105080000C4604D1BDE8F0470909FFF737BA0029FB
:1050900055D011F0030652D10B792C2B38D18968E9
:1050A000FFF746FAE668002E49D016F0030846D10D
:1050B0007768FAB28E2A334609D13F0A06F104090D
:1050C00007F1FF3AC24510DC013756F827301A794C
:1050D000312A12D199682846FFF72AFAAB6A686A22
:1050E000DB6CBDE8F0470221184759F8041F284639
:1050F000FFF71EFA08F10108E4E7322A1FD1996888
:10510000AB6A686A1B6DBDE8F047022209091847BF
:105110002D2B14D18C6894B163681B0A022B06D026
:10512000271D6368B6EB132F10D3BDE8F087E36843
:10513000002BF5D09A07F3D11B79AC2BF0D1214687
:105140002846064ABDE8F047FFF71CB957F8041F88
:105150002846FFF78FFF0136E3E700BF1AB70508BF
:105160002DE9F8430446006AC68A1746B2070D4681
:1051700006D5374A29462046BDE8F843FFF702B96D
:1051800001F00F02022A18D1A37809098BB1838B91
:10519000013383834FF000094FF00108002955D0F7
:1051A0000022FEF7C1FE03780646002B38D0294ABC
:1051B000E0E7438B01334383ECE70A79BA4289463F
:1051C0000BD18968A37809091BB1838B01338383D1
:1051D000E2E7438B01334383DEE79A4218D1A37899
:1051E000002BC6D10122A270896879B301F00F02A9
:1051F000022A18BF894646F0040618BFD9F80810DD
:10520000C68206BF0909994609094FF00308C5E798
:10521000896846F002060909C6824FF00508BDE715
:105220000423037080F80180236A1B8B032B0DD1AC
:10523000482F0BD1B9F1000F08D0D9F80C10204637
:10524000FFF7D4F8737843EA00137370BDE8F8836E
:1052500057B605082EB7050849234822FFF780BF37
:105260004F234E22FFF77CBF2DE9F04F0E468DB045
:10527000016200214270C1603378072B0446154655
:1052800005D08B4A0DB0BDE8F04FFFF77BB8012A7F
:1052900005D0036B021D1B68C06A294698476378D6
:1052A000D6F80C80032B10D10BAA462108F10C0074
:1052B000FEF702FC236B0B9A9B680146E06A984755
:1052C00063687083002B40F0BC80D8F81010C1B127
:1052D00001F00F03022B10D10B09752B3FD006D81C
:1052E0003E2B3ED05E2B0CD0724A2046CAE740F2DD
:1052F0008E529342F8D1032304E06F4A2046FFF711
:1053000041F80223049309AAD8F81430089319210C
:1053100008A8FEF7D1FB4FF000090690069B9945BF
:1053200021D16378012B16D9236B04995B68E06A5D
:1053300098476378042B0ED1206A049BE26A03939A
:10534000438B02930023CDE900330521D2E90232D9
:10535000006906F062FA6368002B72D114E0002342
:10536000D0E70123CEE7099B53F829100B79082BCE
:105370004FEA890B02D109F10109CFE7052B06D0CD
:105380004E4A2046FEF7FEFF0DB0BDE8F08F8B6859
:10539000002BF5D09A07F3D1CA68002AF0D11A7908
:1053A0002C2AEDD19E6806F00F02022AE8D1D3F82C
:1053B0000CA0BAF1000FE3D01AF0030FE0D19AF875
:1053C0000430302BDCD10AAAA4210AF10800FEF730
:1053D00073FB360940F28C439E4207461BD10128DD
:1053E00005D10A9A136803F00F03022B04D0344A44
:1053F000099B53F80B10C4E7E168012D01F101038B
:10540000E3601AD01268236BE06ADB6812099847E0
:1054100098B92C4AECE740F2B5339E4215D10128E9
:1054200003D10A9B1968CB0701D4274AE0E7012D75
:1054300003D0E06A491002F0BFFB6368002B9AD0EA
:10544000D046D8F80030A3609EE740F202439E4267
:1054500023D1012804D90A9B1A6812F0010601D150
:105460001A4AC5E7012DE8D0531007930A9A0BA9F1
:1054700052F82600FEF7D4F808B9154AB8E7E36AEF
:105480000B9805930CF011F8013602460799059820
:1054900002F099FBB742E9D1CFE7012DCDD0236BC4
:1054A0000246D3F810B0E06A0A9B3146D847C4E7F9
:1054B00038B705084EB7050852B7050863B70508A1
:1054C00071B705087DB7050881B705088DB70508D0
:1054D0009FB705084278012A0B4602D1006A01F005
:1054E00027BE816A026A406A183101F030BE0000AE
:1054F0002DE9F14F8F0704460D46164613D001F0F3
:105500000F03022B18D102F0FD06012E4FEA1111F4
:1055100004D001B0BDE8F04FFFF7DCBF01B0BDE83B
:10552000F04FFEF7F8BF4968CBB22D2B7FD00BD8D8
:10553000062B0ED02C2B13D0514A2946204601B001
:10554000BDE8F04FFEF71EBF2E2B00F084809D2B90
:10555000F2D1002EF0D105F10802090A20467FE0C1
:10556000022A02D0A968FEF7E3FFEF68002FE3D01C
:1055700017F00309E0D17B68DAB28E2AB8460DD164
:10558000022E4FEA132805D007F1040A08F1FF3B69
:10559000D94515DB08F1010857F8288098F8043040
:1055A000312B27D1022E13D1A36A606A5B6E984714
:1055B000A36ADB6C0121606A01B0BDE8F04F1847B7
:1055C0005AF8041F2046FEF7B3FF09F10109DFE78F
:1055D0002046D8F80810FEF7ABFF012ED4E90903E6
:1055E00005D19B6D9847A36A0021DB6CE3E7DB6C78
:1055F0000121E1E7322B9FD1012ED4E909030CD11F
:105600005B6D9847A36AD8F808101B6D0022606A8A
:10561000090901B0BDE8F04F1847022E01D11B6EF9
:105620009847A36AD8F808101B6D0122EFE7AA6813
:10563000002A81D0002E7FF47FAF5168090A022929
:1056400007D1D3682BB1980703D11B79AC2B3FF45A
:1056500073AF083282E7002A7FF46EAFA96821B9E0
:1056600001B0BDE8F04F00F073B88E0703D10B799D
:10567000922B0A46E1D005F1080201216EE700BF36
:10568000AAB705082DE9F047C7681E46BB1CC360D2
:10569000836A04460D469B6A406A3946904698479D
:1056A000A36A606AD3F88C3007F10109494698472C
:1056B000A96800222046FFF71BFF2D6965BB414604
:1056C0002046FEF735FF236A19780629D4E9090335
:1056D0001CD1D3F8CC302946984720460121FEF74B
:1056E00071FCA36A606ADB6D9847A36A606A9B6E6F
:1056F00039469847A36A606A9B6A49469847A36AF5
:10570000606AD3F89030BDE8F0471847B200D3F88C
:10571000A83005329847E8E72B79AD2B07D1A96867
:105720003B4600222046FEF73BFFED68C6E7E968EE
:105730002046FEF7FDFEA36A606AD3F88830012197
:105740009847731C424629462046FFF79BFFCCE74B
:105750002DE9F84304460D46904601F1FF39002635
:105760004FF0FF37B9F1FF3F0CD17B1C05D1A36A85
:10577000606AD3F8AC30294698470026AE421DD166
:10578000BDE8F88358F8261071B18A070CD10B795F
:10579000222B09D101370BD1A36A606AD3F8B0304C
:1057A0004A46314698473746013609F1FF39D9E76D
:1057B0002046084ABDE8F843FEF7E4BD58F8261035
:1057C000B74208BF896800222046FFF791FE0136E4
:1057D000D4E700BFBEB705082DE9F0470446904660
:1057E00099460F4621B9BDE8F0471946FEF7A0BE1D
:1057F000C668731CC360156835B315F0030A23D15E
:105800002B797B2B20D1A968FEF792FE52463146B8
:105810002046FEF7DFFBE96852462046FFF768FEA8
:105820004B4608F10402791E2046FFF7D5FFA36A14
:10583000606ADB6F3146984720460321FEF7C2FBC2
:10584000BDE8F047FEF7D6BB29462046FEF770FEBE
:10585000204600223146FEF7BDFBA36A606ADB6D7D
:105860009847DDE737B50C46054601AA7A2104F1D1
:105870000800FEF721F9E368019A01462846FFF780
:10588000ABFF03B030BD2DE9F04F8B6803F00F0381
:10589000022B89B004460D4640F00081CB68002BF6
:1058A00000F0FC80980740F0F9801A792C2A40F02B
:1058B000F5809A6802F00F01022940F0EF8012098A
:1058C0007C2A40F0EB80DB681A79302A40F0E680D1
:1058D0009B68069307AAA42106A8FEF7EDF8431ECD
:1058E000022B00F2DB80079B01281A6800F0C980B8
:1058F000022800F0C4809E68F10740F1CF80710853
:1059000000F0CC80D3F8049032B1930704D1117920
:10591000A639022940F2C280B9F1000F08D019F06F
:10592000030F05D199F80410A639022940F2B68078
:10593000AB6801932B696F690293E5686369218BFA
:105940000493638B039305F1010BAB1C618319F086
:10595000010805F104010593A582A4F816B005F12C
:10596000030AE16005D1494620460592FEF7E0FDB5
:10597000059A11462046FEF7DBFDA26A606A926E28
:1059800051469047A26A606A926AA91C9047A26A2F
:10599000606A526D9047002201992046FFF7A8FDEA
:1059A00002992046FEF7C4FDA26A606A926A5946CF
:1059B000904731462046FEF7BBFDA26A606AD2F8E6
:1059C0009C200E219047A26A606A926A51469047D5
:1059D000D4E90902B8F1000F57D1936D9847A36A33
:1059E000606A1B6E9847A36A606AD3F89C30002EE9
:1059F000ACBF002101219847A36A606ADB6EAA1C34
:105A000001219847049B6361039B6383002F43D06C
:105A1000A36A606ADB6D9847B8F1000F03D1A36AEF
:105A2000606ADB6D984739462046FEF781FDE668DF
:105A3000606A731CE360A36A31469B6E9847A36A51
:105A4000606A9B6888F0010101319847A36A606A27
:105A50009B6A29469847A36A606ADB6D9847B8F14C
:105A6000000F03D1A36A606ADB6D984727B1A36A70
:105A7000606A9B6A3146984709B0BDE8F08F0326FB
:105A800040E791460326024646E7526D9047494655
:105A90002046FEF74DFDA6E73E46D7E7E668238B96
:105AA000B4F81A9063836FEA46436FEA5343D4F81D
:105AB00014A0A382771CF31CE968E3602046E78208
:105AC000FEF736FDA36A606AD3F888300121984753
:105AD000A36A606A9B6A39469847A36A606AD3F8EA
:105AE0008C3006F10208414698470022A9682046FA
:105AF000FFF7FEFC29692046FEF71AFDA36A606ADB
:105B00009B6E39469847A36A606A9B6A41469847EC
:105B1000A36A606AD3F8903098476969C4F814A002
:105B20002046A4F81A90FEF703FDA36A606A9B6AF8
:105B3000314609B0BDE8F04F18472DE9F74F04464C
:105B4000174698460E4629B9194603B0BDE8F04FEE
:105B5000FEF7EEBCC5682B1DC360136805F1010A92
:105B600005F1020B05F10309002B00F0D28013F0C0
:105B7000030240F0CE8019797B2940F0CA809968F1
:105B800001920093FEF7D4FCA16A606A496D8847D0
:105B90004FF464712046FEF7B6FADDE90032204684
:105BA000D968FFF7A5FC022229462046FEF712FA23
:105BB000A36A606A9B68032198473A1D4346711E99
:105BC0002046FFF7BAFFA36A606A9B686FF0020184
:105BD0009847A36A606AD3F880602A4651465B46BC
:105BE000B047A36A606A5B6D9847A36A606A5B6EA0
:105BF0009847A36A606A1B6E9847A36A606A5B6CE9
:105C0000002240F291319847A36A606A5B6E984720
:105C1000A36A606A5B6E9847A36A606A5B6D984787
:105C2000A36A606A1B6D00220A219847A36A606A12
:105C30001B6E9847A36A606A1B6B0F219847A36A83
:105C4000606AD3F8C05000231A460321A8472046B3
:105C5000FEF740FAA36A606ADB6E4A460021984765
:105C6000A36A606ADB6D9847A36A606A1B6B0F21A9
:105C70009847A36A606A9B6E49469847A36A606A20
:105C80009B6802219847A36A606A9B6A59469847B5
:105C9000A36A606A5B6E9847A36A606A5B6E984706
:105CA000A36A606A9B6A51469847A36A606A5B6C04
:105CB000002240F291319847A36A606A1B6B0F2162
:105CC0009847A36A606A5B6D9847A36A606A5B6DD8
:105CD0009847A36A606AD3F8C05000231A4603218C
:105CE000A8472046FEF7F6F9A36A606ADB6D98477D
:105CF000A36A606A9B684FF0FF319847A36A606AA5
:105D00009B6A49469847204603B0BDE8F04FFEF72E
:105D100071B919462046FEF70BFCA36A606A5B6DF9
:105D2000984720464FF46471FEF7EDF9A36A606A64
:105D3000DB6D984737E72DE9F041CD6804460E4604
:105D400065BB0378C3B1036A1D78ADB940F29E31DB
:105D5000FEF7E1FBB1682046FEF7EAFBA36A606A42
:105D6000D3F8BC602A462B460121B047A36A606A7B
:105D7000DB6DBDE8F0411847B1688B0707D001F033
:105D80000F03022B08D12046FEF7D2FBEEE70029D5
:105D9000F9D00B793A2BF6D1BDE8F081AF0740F08E
:105DA000AF806B68DAB25B2A11D1ED68002D4AD161
:105DB000006A0378072BEFD1896801F00F03022BEB
:105DC000EAD10422BDE8F041D140FEF7ADB8562A31
:105DD00013D101228968FFF78BFBE9682046FEF7A3
:105DE000A7FBA968A36A606AD3F89C3009093E3909
:105DF000C9B298470222B1687DE0572A25D11B0A13
:105E00005F1E013355F82310FEF792FB002F03DDD0
:105E1000A36A606A5B6D9847B16800222046FFF76D
:105E200067FB04350026BE42B6DA0136BE4203DA0D
:105E3000A36A606A5B6D984755F8041F00222046EC
:105E4000FFF756FBEFE7A9075AD16B68DAB2062ACB
:105E500056D1B768002F53D0BA0751D17A68D1B262
:105E600006294DD11B0AB3EB122F4FEA122847D156
:105E7000A8F10203012B43D8BB6823B1980702D1D4
:105E80001B79222B3CD0FB6823B1990702D11B79E7
:105E9000222B35D0B8F1020F06D03B6923B19A0707
:105EA00002D11B79222B2BD0A9682046FEF740FB9C
:105EB000E9682046FEF73CFBB8F1030F07D1204606
:105EC0002969FEF735FBA36A606A5B6E9847A36A8F
:105ED000606A1B6E9847B96800222046FFF708FBEE
:105EE000F96800222046FFF703FBB8F1030F7FF4A7
:105EF00053AF396900222046BDE8F041FFF7F8BAF8
:105F000029462046FEF714FB002274E70023032AEB
:105F10002DE9F04104460D46164642700162C36009
:105F200080F8342002D1C08E50BBA063A36A606A9F
:105F30001B684FF000083146A4F836802A4698477F
:105F400006212046FEF73EF86778EE68012F04BF71
:105F5000A5F82280A5F82480B6B1B20714D1337910
:105F60003F2B11D1B168FEF7E3FAA36A606AD3F858
:105F7000C4309847A36A606A5B68BDE8F04118477F
:105F80008000FAF78EF9D0E72B78072B00F2938088
:105F9000DFE803F0049125414141410E314620469E
:105FA000FEF7C6FAA36A606A1B6B0F219847DCE70D
:105FB000012F12D10023A370F168574B46222046CF
:105FC000FEF75DF92B8B032B07D131692046FEF7D5
:105FD0000DFAEB8A43EA8013EB827169DFE7A36A6B
:105FE0003168DB68606A98476378012B07D100232A
:105FF000A370B168494B4C222046FEF740F9F16886
:106000002046FEF795FAEB8ADB07AED5A36A606AF5
:10601000DB6D9847C6E7012FD6F80C8005D1206AC2
:1060200004223946FDF780FF6F83A36A3168DB687D
:10603000606A98472B78032B24D1A36AD3F8A03049
:106040000122606A002198472B78062B28D1A36A89
:10605000606A1B6C984701212046FEF75CFAA36A30
:10606000606A1B6C9847A36A606A1B6C98470023A0
:10607000B26841462046FFF705FB2B78062B7FF4DC
:1060800074AF8FE7042B04D1A36A0222D3F8A030A7
:10609000D7E7052BD8D1A36A0322D3F8A030D0E7E5
:1060A00020460121FEF737FAA36A606AD3F88830E8
:1060B00001219847DBE7012F04D104220A21284659
:1060C000FDF732FF17212046FEF725FA162120465C
:1060D000FFF700FAB168A36A606A9B6B09099847E9
:1060E0001A212046FFF7F6F931692046FEF720FA1B
:1060F0000A212846FDF708FF0246D4E90903117872
:10610000042902D11B6B0F2150E71D69528800231F
:106110000A21A84729E700BF595202086152020824
:10612000036A10B51A8B0446FEF707F901462046AC
:10613000BDE81040FFF7CEB92DE9F04F8D682B79FF
:10614000032B85B004460AD12946FFF7E9FFAA6967
:10615000D38A43F00103D38205B0BDE8F08F026A11
:10616000D28AD20706D4624A294605B0BDE8F04F6C
:10617000FEF708B9162B40F0AD80C668E968331DFC
:10618000C360FEF7D5F9A36A606A5B6C002240F237
:1061900092319847A36A606AD3F8C07000231A4608
:1061A0001946B847E76863690093638B0193BB1C8A
:1061B000E360238B6383A36A606A9B6AA78207F10B
:1061C000010806F1010B4146A4F816809847012208
:1061D00059462046FDF7FEFEA36A606A5B6D98474C
:1061E00020464FF46571FDF78EFFA9682046002216
:1061F000FFF77EF9A36A606AD3F8943006F10209CA
:10620000002249469847A36A606A9B6A59469847A4
:10621000A36A606AD3F8D0309847A36A606A5B6D5E
:106220009847A36A606A5B69012240F23631984759
:10623000A36A606AD3F89C3008219847A36A606A11
:10624000DB6E06F1030A524600219847A36A606A92
:10625000DB6D9847A36A606AD3F894300122314617
:106260009847A36A606A9B6A51469847A36A606A26
:106270009B68012198472046FDF7BCFEA36A606A2F
:10628000D3F8D4309847A36A606A9B6A4946984716
:1062900029692046FEF74CF9A36A606A9B6E414665
:1062A0009847009B6361019B6383A36A606A9B6A52
:1062B0003146984769692046FEF73AF9A36A606A51
:1062C0009B6A39469847A36A606ADB6D05B0BDE8F2
:1062D000F04F184703AA7A2105F10800FDF7ECFBFF
:1062E000EB68039A01462046FFF727FC34E700BF1E
:1062F000C5B705082DE9F04F85B0C5681E460E9B51
:1063000003936B1C0293AB1C0446C3600F46934679
:1063100029460122FDF75EFE39462046FEF708F9C0
:10632000A36A606AD3F894300022691C9847A36A74
:10633000606A9B6A29469847A36A606AD3F8D0309E
:106340009847D4F80C9009F10103E36000275F45FA
:1063500018DB2046FDF74EFEA36A606AD3F8D430FE
:106360009847A36A02999B6A606A984703992046F6
:10637000FEF7DEF8A36A606A9B6A494605B0BDE88D
:10638000F04F18473346D4F80CA01A6801920AF16E
:106390000102E260019AD2F8088004360137B8F1B0
:1063A000000F4FD1BB4542D1A36A606ADB6D9847AD
:1063B0000025A846019B2046D968FEF7B9F825B309
:1063C000A36A606A1B6B0F219847A36A606A9B6A85
:1063D00041469847A36A606A9B6801219847A36A6F
:1063E000606A1B6B0F21984729462046FFF772F819
:1063F00029462046FEF782F8A36A606A9B684FF040
:10640000FF3198472046FDF7F5FDA36A606AD3F88F
:106410009430012249469847A36A606A9B6A5146B4
:106420009847A36A606A9B68012198478FE72046D6
:106430001E4A1968FDF7A6FF204605B0BDE8F04FDB
:10644000FDF7D8BD18F003052DD198F80420762A61
:10645000434603D1DD68D8F808802D09A36A606A35
:106460005B6D984741462046FEF762F8A36A606A72
:10647000D3F89C3008219847A36A606ADB6E5246C5
:1064800000219847002D8FD029462046FFF722F89B
:10649000D4F80C8008F10103E36002224146204653
:1064A000FDF798FD86E70025D8E700BFDCB70508B3
:1064B0002DE9F347C76898467B1C16460D46C36016
:1064C00002223946DDE90AA90446FDF783FD002EC4
:1064D0002DD1A36A606A9B6803219847294620460C
:1064E000FEF726F8A36A606A9B686FF0020198477E
:1064F000A36A606A1B6B0F219847A36A606A9B6A54
:1065000039469847A36A606A9B68012198474946C3
:106510002046FEF70DF8A36A606A9B684FF0FF31D2
:106520009847204602B0BDE8F047FDF763BDCDF8BF
:1065300000A04346324629462046FFF7DBFED7E758
:10654000F0B5CE683379782B85B005460C4609D175
:10655000B36801930023009389681A46FFF7A8FFE8
:1065600005B0F0BD742B03AA4FF0770113D106F1EB
:106570000800FDF7A1FA3769A168039B0246F0689D
:1065800027B900902846FFF7B5FEE9E7BC68CDE9DA
:1065900000042846E2E704F10C00FDF78DFA002321
:1065A0000093A168039B0246ECE7000001F00F0393
:1065B000022B70B504460D46164602D01E4AFDF762
:1065C000E1FE31462046FDF7B3FFA36A606A5B6DCA
:1065D00098476378012B4FEA151610D1226A137879
:1065E000033B032B0BD85068314600F0A1FD034656
:1065F000206A1A78032A08D13146FDF795FC314606
:106600002046BDE87040FEF765BF00223146FDF729
:106610008BFC236A5B685B68002B02460CBF01237E
:10662000002304D00178012904BF0021017029460C
:106630002046FDF7FBFEE2E7AAB705082DE9F04F7B
:1066400087B0CDE90221044605AAA42103A81D466E
:10665000FDF732FA00260190B1463746B0464FF0BA
:10666000010B019B9E4211D127B1A36A606A5B6B4B
:1066700049469847029AD4E90903002A76D0D3F80C
:10668000C0403B4642462946A04713E0059B53F8CD
:1066900026A0BAF1000F5BD01AF0030F58D19AF878
:1066A0000420A62A1AD1B80707D5324A51462046F7
:1066B000FDF768FE07B0BDE8F08F1D2E01D92E4A08
:1066C000F4E70BFA06F2DAF80810204649EA020964
:1066D000FDF72EFF013501270136C2E7A72A0DD1AC
:1066E000A26A606A126C9047DAF8081047F0020755
:1066F0002046FDF71DFF08F10108EDE7A82A27D184
:10670000DAF80C2072B191070CD11179AA2907D1BE
:106710009268DAF808102046FFF748FF0135DBE7FA
:10672000AC290FD0DAF8081001F00F02022A01D0CC
:10673000124ABBE7A26A606A926B09099047DAF8CD
:106740000C10D5E7062251462046FDF7D3FFE5E7BA
:10675000BB0701D50A4AA9E7B8F1000F01D0094AE1
:10676000A4E751462046FDF7E3FED7E7D3F8BC4047
:1067700087E700BFF4B70508FBB7050803B80508AD
:1067800010B8050817B8050870B50D4641780129FD
:106790000446134603D12A46FDF7D5FC6861A36A77
:1067A000606A9B6C98476E6900231A463146204602
:1067B000FDF730FCA36AB18A9B6B606A9847E96871
:1067C00029B18B0703D10B79A32B08BF00212046E9
:1067D00002230022FFF732FFB08A70BD00238968D0
:1067E0001A46FFF72BBF00002DE9F8430C468968D5
:1067F0000546FDF79DFEE668002E56D07768296AAB
:10680000FBB209788E2BA36819BF04F10C0601278F
:106810003F0A0836072903F00F024AD1022A46D15F
:106820001A099A2A47D133681A79302A3FD19B68CE
:10683000002B3CD10A212846FDF76DFE2A6AD36A57
:10684000128D32B93168404A2846BDE8F843FDF759
:1068500099BD5978C9070FD559682846FDF75BFEE1
:10686000022FD5E909030AD8D3F8BC4000231A4601
:106870000221A047012416E0013A0833E1E77268DB
:1068800011793229F0D1B46821793029ECD191689D
:106890005B6C012209099847A16800230122284660
:1068A000FFF7CCFE0324A74226D8BDE8F8830024D6
:1068B000F9E7022AFBD140F25922B2EB131FF6D1BD
:1068C00033681A79302AF2D19B68002BEFD013F08D
:1068D0000304ECD11B792F2BE5D1AB6A686AD3F89E
:1068E000BC80224623462146C04733682246996829
:1068F0002846FDF787FFBDE704F10108B84556F8C3
:1069000024104FEA84031AD20A79322A17D1334469
:10691000D3F8049099F80430302B10D18968AB6A11
:10692000686A5B6C002209099847D9F808100023AF
:1069300001222846FFF782FE08F10104B3E728464A
:10694000FDF7F6FDA046F7E71EB8050810B5026A88
:106950001278072A04460B4606D0022A04D0BDE866
:106960001040064AFDF70EBD20461946FFF73CFFD2
:106970002046BDE81040FDF7ADBB00BF31B80508AB
:10698000D1E90212FFF712BE036A10B51A8B044652
:10699000FFF7FAFE01462046BDE81040FEF79ABD1B
:1069A0002DE9F04F044685B0884602AA422108F13D
:1069B0000800FDF781F8236A00271E8B8346BA463C
:1069C0005F450AD1D8F80C100B79032B50D1324611
:1069D0002046FDF7B2FC054658E0029B53F82730ED
:1069E000019303AA6C2103F10800FDF765F8039BEE
:1069F00019680A09732A05460DD02046FDF798FD4F
:106A00004FF00109A94527D3019BD96869B12046F8
:106A1000FDF78EFD09E0022809D02A4A2046FDF73D
:106A2000B1FC35460AF1010A2E460137C8E759681C
:106A30000B09412B0CD040F2CD429342F2D040F2F0
:106A4000A352934206D0B3F5707FE6D10425E9E75F
:106A50000125E7E70325E5E7039B606A53F8291062
:106A6000A36A00221B6D0909984709F10109C9E7CA
:106A7000442B17D18F68324639462046FDF75DFC1E
:106A8000BA69D38A43F001030546D3820027ABEBF2
:106A90000A0ABA450BD829462046FEF71BFD05B069
:106AA000BDE8F08F32462046FFF76EFE93E7A36AFB
:106AB000606AD3F8BC6000231A460121B047013751
:106AC000E7E700BF3CB805082DE9F3418D6805F004
:106AD0000F030A2B04460E4607D0002D31D015F0C7
:106AE00003012ED12B79652B1ED10095002501AA1B
:106AF00065216846FCF7E0FF019B002103EB800065
:106B000040F2CA52834215D1F26840F21A439A42C7
:106B100037D1236A1F78B7B13B4A3146204602B0CD
:106B2000BDE8F041FDF72EBC622BEDD1AB680093C0
:106B3000ED68DCE753F8047B97420CBF0131033169
:106B4000E0E70021E0E7A36A606A5B6B9847A36A0D
:106B5000606A9B6B05219847A36A606AD3F8A030EE
:106B60003A460121984701AA29462046FDF700FB35
:106B7000A36A606ADB6A0222394602B0BDE8F041CE
:106B80001847A36A606A5B6B984706F10C006A4677
:106B90006A21FCF791FF00270646B742D4E90903B2
:106BA00013D1D3F8A030002231469847294601AAD4
:106BB0002046FDF7DDFA0025B542D4E909030DD1E1
:106BC000DB6D984702B0BDE8F081009A9B6B52F8EC
:106BD00027209168090998470137DEE7009ADB6AA8
:106BE00052F82580D8F808703F09394601229847A5
:106BF000D8F80C1029B939462046FEF76BFC013550
:106C0000DAE70909F8E700BF54B80508836A37B521
:106C100004460D465B6B406A00219847A36A606A90
:106C20001B6B0F2198472946204601AAFDF7A0FAC1
:106C30000199204603B0BDE83040FEF74BBC000090
:106C40002DE9F04F9BB0CDE9020110209D4D144677
:106C5000F9F70EFB2B69436058220021064604A871
:106C600020F08CF84FF0FF33012113A809938DF821
:106C7000104006F089FD039BD900012241F002017A
:106C800013A806F0B7FD01234360002116A80AF0FF
:106C900069FF029A95F81C321268002104A8FDF7DA
:106CA00052FA054611A800F029FF874B0B9F01906F
:106CB0000D900E934FF0000B0FB1059C1CB30B9C75
:106CC00014B1059B002B3ED00198DFF8FC91DFF852
:106CD000FCA1594600F019FF0B9C0027DDF8148039
:106CE000002C00F03981B8F1000F00F0F1800C9C0D
:106CF00004A8E168FDF7BAFAA38A069A0399404608
:106D000009F0ECF92CE13B8B042B4FF001023946E2
:106D100004A807D1FEF7A8FA079BBF689B4538BFB8
:106D20009B46C9E7FFF7F2F83B8D9C42F4D2FB6A21
:106D300003EBC40113F83430012B02D13846FDF7C0
:106D40001BF90134F0E7E28A520716D5218D01398B
:106D500013D3E76A07EBC1024FEAC10E507810F077
:106D6000020F25D04BB1D3E9008C92E8030083E8F1
:106D7000030047F80E80C2F804C04FF000032384DC
:106D80000027B4F828C0674518DB00239C454ED186
:106D9000D4F804E0BEF1000F08D00020BEF828A00F
:106DA0000346504553DB002B40F08A80A46887E7F8
:106DB000002BCCD1012808BF1346C8E72378D4F8AC
:106DC0002C80012B4FEAC70A08EBC70905D1D9F877
:106DD00004300A2B12D10137D3E718F837300DD918
:106DE000012B0BD14FF0030308F83730238B032B13
:106DF00016D0E38A43F01003E38203E018F80A3068
:106E0000032BF3D018F80A30042B03D099F8013083
:106E1000DB07E0D5238C5A1C2284A9F80230DAE77C
:106E2000D9F8040006F02CFB0128EBDCE1E7E26A6C
:106E300002EBC30112F83320052A06D14A78D7079E
:106E40005FBF228C4A800132228401339EE7DEF844
:106E50002C2002EBC00912F83020053A012A14D880
:106E6000002710E0E26A02EBC70812F83720062A72
:106E700008D1D9F80410D8F80420914204BFA8F82A
:106E8000023001330137BC45ECD1013089E7E06ABB
:106E900000EBC20110F83200062802D14878C00782
:106EA00002D548881844488001329445EFD1628B5E
:106EB00012FA83F26283228C12FA83F3238475E739
:106EC0000022F2E734000020AC0D0608B00E0608E0
:106ED000238B042B17D10F9B1BB9584604F03EFCA3
:106EE0000F9000230D9303224A4B1093214604A8D0
:106EF000FEF7BAF9059B23B90422214604A8FEF740
:106F0000B3F9A468EAE6023B012B21D837B95B4606
:106F100007AA05A911A803F07DFD0746CDE90D7A62
:106F20000222214604A8FEF7F1FF059B002BE8D1C1
:106F30000322214604A8FEF7E9FF059B002BE0D1C0
:106F40000422214604A8FEF7E1FF0028F8D0D8E784
:106F5000019BCDE90D39E3E7B8F1000F7FF4C7AE2F
:106F6000DDF81490D5F81080B9F1000F16D0019813
:106F700000F0D3FD002F41D10F9808B104F003FCBD
:106F80000298FCF787FF2846AD68FCF7B3FF002D99
:106F9000F9D10598002835D0F9F742F9139C1898D3
:106FA000C4F3DC046400033400EB94008000F9F7C0
:106FB0005FF924F003040444F460DDE91441B06097
:106FC00001F1040CA1450BD1189A00239342CED0B5
:106FD000199951F82300F16841F823000133F5E7CE
:106FE00051F839303BB1042B1FBF5CF839205210E7
:106FF000DB0820F8123009F10109E3E7384603F015
:107000002BFDB9E72A46314640461BB0BDE8F04F9C
:1070100004F014BC8C0F0608F0B52DED028B8842ED
:1070200083B007460C4604D1012003B0BDEC028BAF
:10703000F0BD244B984201D10020F6E79942FBD0E5
:1070400006F008FE0546204606F004FE8542F3D110
:107050001D4B9D4213D17A6863689A42ECD13E1D64
:10706000043400257B68AB42DED954F8041F56F87F
:10707000040FFFF7D1FF0028DED00135F2E72146EB
:10708000384607F0C1F80028D6D0104B9D42CBD12E
:10709000384609F07FF9B5EE400AF1EE10FAB0EE8D
:1070A000408AC1D1204609F075F98DED010A18EE2C
:1070B000100A019B00F0004003F00043C31A58423D
:1070C0005841B2E7C81006084C280608BC1A060842
:1070D000C90010B50122044641F00201083006F053
:1070E00089FB43683BB9A368C3F3DC03013B5B0046
:1070F00043F001034360C3F34F0010BD70B5054674
:107100000E460024EB69A34208D8314605F114006D
:107110000AF0E5FBEC69013C204670BD2B6A314664
:1071200053F82400FFF778FF0028F5D10134E9E790
:1071300010B501220446FCF7F7FE0378012B05D1B8
:107140002378012B8CBF04230223037010BD70B57C
:1071500005460E46104619461C46FCF7D5FE037838
:107160005A1E012A06D87368002221462846BDE827
:1071700070401847032B02D173680122F5E7366887
:107180004288042B21462846B44608BF0023BDE8A8
:10719000704018BF012360474379012B07D08368F3
:1071A0001944036981605A8C9142C8BF5984704761
:1071B000002383714379012B1EBF036AC26A43F81F
:1071C000212070476FF00301FFF7E6BF0421FFF7AE
:1071D000E3BF6FF00201FFF7DFBF426A0346407969
:1071E000032888BF586B114494BF18468018596211
:1071F0007047827903460AB118467047C26A4079DF
:107200000328114401D8D962F6E7986AD96202448A
:10721000586B1044704710B50C460121FFF7E9FF89
:10722000047010BD10B51446FFF7B6FF0121FFF73B
:10723000E0FF047010BD53220121FFF7F3BF542279
:107240000121FFF7EFBF57220121FFF7EBBF5822C3
:107250000221FFF7E7BF59224FF0FF31FFF7E2BFEE
:107260005A220021FFF7DEBF5B220021FFF7DABFC1
:107270005D224FF0FF31FFF7D5BF19B103215F2227
:10728000FFF7D0BF5E22FBE7A1F13002D2B20021AE
:10729000FFF7C8BF62226FF00101FFF7C3BF10B54F
:1072A000632204464FF0FF31FFF7BCFF0123A371B7
:1072B00010BD10B501F164020446D2B24942FFF795
:1072C000B1FF0123A37110BD10B501F1670204469F
:1072D000D2B24942FFF7A6FF2269D38A43F00103E5
:1072E000D38210BD38B504461D46FFF79BFF2A46E2
:1072F00020460249BDE8384013F00CB9F37102088A
:1073000070B504460D46C06819461646FFF7E0FE04
:107310003246034629462046BDE87040FFF7E2BFEB
:107320000B4610220121FFF7EBBF11320B46D2B200
:107330000121FFF7E5BF20B40B4602F1140551000F
:10734000C1F10101EAB25DF8045BFFF7D9BF163263
:107350000B46D2B24FF0FF31FFF7D2BF19320B46C6
:10736000D2B20021FFF7CCBF70B4C4682678042ED7
:107370001D4608BF6668638808BF46F823505D1C39
:10738000658070BCFFF7AEBF03F128011346CAB297
:107390000021FFF7A7BF022A02F12A020B46D2B250
:1073A00014BFC1F101010121FFF79CBF03290AD0DD
:1073B00004290AD101210B460A4443EA8203C94346
:1073C0002F22FFF78FBF0021F5E700210223F3E70B
:1073D0000B4630220139FFF785BF10B4144641EA4D
:1073E0000223214431225DF8044BFFF77BBFF8B53F
:1073F00016461F46FFF7D0FE8479054604BB437945
:10740000022B25D9C46A036AC4F1FF2453F827303C
:1074100004F57F04FE34442E1C4412D814F1400FAE
:1074200014DB3F2CD4BF00270127E41BB91C2846DE
:10743000FFF7DFFE06706FB9442E98BF40344470EA
:10744000F8BD7F2C94BF00270127EEE70127ECE76A
:107450000127EBE76B79442E98BF04F58044042B99
:1074600005D1B4F5004F24BF012385F8383064F00E
:107470007F03E41143708470E2E710B50B460446C5
:1074800042220021FFF7B3FF0123A37110BDF8B51D
:1074900005460C4621F400471646CAB90B040ED522
:1074A0005921FFF7B8FE59212846FFF7B4FE5921AC
:1074B0002846FFF7B0FE59212846FFF7ACFE3B46B1
:1074C000422200212846FFF792FF0123AB71F8BD4D
:1074D0003B4640220021FFF78AFF210A21F07F016D
:1074E0003143C9B22846FFF796FEEEE70B46B2FAE3
:1074F00082F120B4490902F14705EAB249005DF87A
:10750000045BFFF774BF0B464B220121FFF76FBFEF
:1075100010B50B4604464A220021FFF768FF0123FD
:10752000A37110BD264BD3F81832022B2DE9F0477A
:10753000044689460ED88669B1420BD9C56A4369AB
:107540008E1BED1A40F2FF7756EA050304D1E36A79
:10755000C4E90539BDE8F087062E01D90F2D1AD9E7
:107560001F2DAA4628BF4FF01F0A1F2D10D8032E2B
:10757000B04628BF4FF0030801212046FFF72DFE3B
:107580004AEA48130370A5EB0A05A6EB0806DBE7F9
:107590004FF00008F0E7BE42B0464FF0020128BFAE
:1075A000B8462046FFF719FE4FEA181303F07003A0
:1075B0002B4363F07F03037080F80180AA46E2E763
:1075C0003400002010B5044631B955224FF0FF3188
:1075D000BDE81040FFF726BE022904D1FFF72BFEBD
:1075E0002046FFF741FE56226FF002012046EFE7EA
:1075F000134621B143224FF0FF31FFF7F8BE44227A
:10760000F9E7134621B145224FF0FF31FFF7EFBEF6
:107610004622F9E7322938B5044611D0332912D071
:1076200000252939CAB220464FF0FF31FFF7FAFD95
:1076300065B12046D322BDE838400021FFF7F2BDF6
:1076400001250621EDE701250721EAE738BD012ADA
:1076500010B40B46044608D0022A0ED15DF8044B44
:1076600069224FF0FF31FFF7DDBD11461B32204686
:10767000D2B25DF8044BFFF743BE4FF0FF31F5E7A0
:1076800070B50D46044611462AB92B461322BDE8B3
:107690007040FFF735BE022A04D1FFF7CCFD20462B
:1076A000FFF7DEFD2B4618226FF001012046EEE7C2
:1076B00010B4044643B90F2A06D8503A5DF8044B7B
:1076C000D2B20121FFF7AEBD03F1240120461346DB
:1076D0005DF8044BCAB20121FFF704BE10B40446A2
:1076E0004BB90F2A07D8403A5DF8044BD2B24FF09D
:1076F000FF31FFF797BD03F12601204613465DF8E1
:10770000044BCAB24FF0FF31FFF7ECBD70B4DDE9B6
:107710000365D2B203EB460443EA062315B10132F6
:107720000134D2B2091B70BCFFF7DCBD07B5CDE94F
:1077300000230B4634220021FFF7E8FF03B05DF879
:1077400004FB07B5CDE900230B4636224FF0FF318D
:10775000FFF7DCFF03B05DF804FB10B50446C0681A
:10776000FFF7CCFC2322034601212046BDE8104050
:10777000FFF7B8BD01F110033F2B73B506460C4669
:1077800008D8A1F18002D2B2012102B0BDE8704058
:10779000FFF748BD012122220DF10505FFF742FD4B
:1077A000294604F07F00E3B2E4112A4605F8010DF2
:1077B000601C0128F5D8013403F0400314D11BB933
:1077C0007F2305F8013C951E491B3046FFF711FD4C
:1077D00001AC6A1E014612F8013FA24208D11044D2
:1077E000401B037002B070BD002BEDD00023E8E712
:1077F00063F07F0301F8013BEDE770B51446D6B2A4
:10780000049A134305460B6907BF2022C4F1010106
:10781000E1432122FFF7A8FD31462846BDE870402C
:10782000FFF7F9BC1A4308BF32220B6916BF332297
:1078300001214FF0FF31FFF797BD00000D2910B572
:1078400004460BD10949C068FFF758FC23220346C0
:1078500001212046BDE81040FFF744BD4231CAB2C5
:10786000BDE810400121FFF7DDBC00BFDC230608A6
:1078700038B504460D460F21FFF7E0FF20462946A4
:10788000FFF796FC02215C22FFF7CCFC20466FF04C
:107890000301BDE83840FFF77FBCF8B504460F464A
:1078A0000F211D461646FFF7C9FF2046FFF7D8FCFB
:1078B00039462046FFF7E1FD31462046FFF778FCC8
:1078C000FFF7C1FC012220462121FFF72EFD2046B3
:1078D0000821FFF79FFE2A4620460021BDE8F84018
:1078E000FFF786BE4379012B70B5044614D0C26BF6
:1078F000436A00259B1AC36305642069038DAB426C
:107900000CD86379032B1BD1606AE36AA0622363FE
:107910001844F8F7C6FC6063012070BDC36A03EB2E
:10792000C50213F83530052B08D101212046967881
:10793000FFF753FC0670236C013323640135DCE749
:10794000042BE9D1D4E90A13626A8A4202D1216B7D
:10795000994203D0A26223630020DEE794F8383016
:107960001BB10649064804F0A9FBE268C38A5268C5
:10797000616B006903F048FFCEE700BF66B80508F9
:10798000B01706082DE9F74F16460023C0E9042377
:10799000378C83608371C362436280F83830738CA4
:1079A000B6F82490B6F81A80B6F816A0B6F81EB04D
:1079B000417101221F449742B8BF17464FEA89051B
:1079C000013F826105F0040508F003021543FA0047
:1079D00002F07802B38B04460AF00F0A15433F0900
:1079E0004FEA59094FEA980847EA090242EA0A02AF
:1079F00042EA08021A4352EA0B0234D1012120461E
:107A0000FFF7EBFB05706379022B18D9D4E90F78E7
:107A10007D0008F0010305F07E054FEA5808BF0914
:107A20001D4358EA07094FF00101204618BF45F0F1
:107A30008005FFF7D2FB0570B9F1000FE8D1636A4A
:107A4000B18AE363E068FFF743FB2B490246204617
:107A500012F060FD0025738BB28B1344AB4248DDFE
:107A6000318D002241E0012120460193FFF7B5FB53
:107A700065F07F053A0105704FEA8A15019B02F017
:107A8000300205F0400515430BF001021543DA0002
:107A900002F0080215434FEA880202F0040215437F
:107AA0004FEA490202F002021543BF084FEA5909A2
:107AB0004FEA5A0A4FEA58085B084FEA5B0B93E714
:107AC000F36A03EBC2035878C0070DD55888A84263
:107AD0000AD15968E068FFF7FBFA074902462046D9
:107AE00012F018FD0135B6E701329142E8DC0521BC
:107AF000F0E703B0BDE8F08FDB71020810B5044673
:107B00004420F8F7CEFBC46010BD10B50446C16137
:107B10008800F8F7ADFB206210BD10B50446006A7E
:107B2000F8F7CEFB2046BDE81040F8F7C9BB10B50A
:107B3000044601618800F8F79BFB606110BD10B539
:107B4000044611B1C068F8F7BBFB6069BDE810409E
:107B5000F8F7B6BB012938B504460D460BDC0269BF
:107B6000406992004FF0FF311FF008F900232570A3
:107B70006370636038BD4068F8F77AFB6368E06063
:107B8000A360F3E70246407810B548B9137854680B
:107B9000022B08BFD368214408BF1819516010BDDB
:107BA0000020FCE7002343700378012B9EBF43694C
:107BB000426843F82120704742684B1E13444942F3
:107BC0000B404360704738B50C461546FFF7DAFFA7
:107BD00010B10444A04200D138BD00F8015B2D0A69
:107BE000F8E710B50C460221FFF7CCFF10B1047086
:107BF000240A447010BD38B50D4604211446FFF721
:107C0000C1FF28B1057084702D0A240A4570C47024
:107C100038BD012970B5054606DC002909DA0239AC
:107C200021F00104FE2606E08B1E012BF7D800246C
:107C3000F8E70024F22646F435412846FFF7D1FF45
:107C400044B17F2C09D844F4304141F080012846EA
:107C5000FFF7C7FFC5E9066470BDA300A201DBB250
:107C600002F4E0421A4342F450624FF2AD2128463A
:107C7000FFF7C1FFEEE7C16910B5044629B17F29BE
:107C80000BD841F43041FFF7ACFFA169204641F425
:107C90003D41BDE81040FFF7A4BF8B008A01DBB275
:107CA00002F4E0421A4342F450624FF20D21FFF712
:107CB000A2FFEAE7114341EAC301FFF792BF072A97
:107CC00085BF083AD200D20042F04002072985BFA2
:107CD00008391143114341F0800141F48C41FFF711
:107CE00080BF30B4DCB244EA02225C101D0104F40F
:107CF0008064C3F3033305F4E04523432A43194367
:107D000030BCFFF778BF38B5436953F8214043686A
:107D1000E41A043C0546C4F34A0141F46041FFF70C
:107D200060FF2B78022B0AD1B4F5006F07D36FF3F5
:107D30000A0414F5006F14BF0020012038BD012093
:107D4000FCE7F8B5446954F822404268A41A043CA0
:107D5000074665101E46BBB9EDB245EA012141F464
:107D60005041FFF73EFF3B78022B0BD1FF2C09D986
:107D700024F0FF0414F5807F14BF0024012426465C
:107D80003046F8BD0124FAE76211C5F30A0502F492
:107D900000522A43A512231205F48065C4F305346A
:107DA00003F4006325431A4345EA811142F400427B
:107DB00041F47041FFF71FFFE2E738B5436953F81C
:107DC00021404368E41A043C0546C4F34F02C4F35F
:107DD0000A3142F4784241F47041FFF70CFF2B78EE
:107DE000022B0AD1B4F5800F07D36FF3150414F5F5
:107DF000800F14BF0020012038BD0120FCE7F8B53A
:107E0000476804460D46164613460A464FF240217F
:107E1000FFF767FF2046330C2A464FF2C021FFF7D9
:107E200060FF3846F8BD072910B4044609D8FF2A78
:107E300007D842EA01215DF8044B41F40051FFF7F5
:107E4000D0BEB2F5803F08D2134620460A465DF800
:107E5000044B4FF24021FFF744BF20465DF8044B2E
:107E6000FFF7CDBF2DE9F84341EA0207072FDDF800
:107E7000209006460C4615464AD803FA09F7FF2F0C
:107E80000CD8914201D0FFF71AFF47EA042141F4D0
:107E900040513046BDE8F843FFF7A3BEFF2B4FEA41
:107EA000C10814D8914218D043EA012343F4005189
:107EB000FFF797FE44EA891141EA08013046FFF7CF
:107EC00090FE48EA8511214341F4C051E1E7914217
:107ED00003D03A46FFF7A7FFF3E784F0070901252F
:107EE00005FA09F545F434413046FFF77AFE3A4683
:107EF00049463046FFF797FF44EA891141EA0801F5
:107F000041F4C0513046FFF76CFE45F43C41C0E7F8
:107F1000BDE8F88308B50378012B04D9FF2902D9FD
:107F2000054805F0B9F8C9B241EA0221BDE80840A8
:107F300041F41041FFF755BE71B8050808B5037844
:107F4000012B04D9FF2A02D9054805F0A5F8D2B2C1
:107F500042EA0121BDE8084041F41841FFF741BE63
:107F600071B80508D2B242EA012141F42841FFF775
:107F700038BE38B5436953F8223042689B1A43F043
:107F800001030C4605460A460A3B4FF24021FFF723
:107F9000A8FE2346284622464FF43241FFF78AFEC8
:107FA000210101F0800104F00704214341F48841DC
:107FB000284641F07801BDE83840FFF712BE0000C6
:107FC00073B51F2B069E05460C4611D81143072991
:107FD0000ED81A49895D44EAC20241F0010142EA21
:107FE000C12141EA831102B0BDE87040FFF7F9BD3D
:107FF00003FA06F1B1F5805F0DD242EA461641EA76
:10800000043246F4784141F09001284602B0BDE8C0
:108010007040FFF7F0BD1F3B214628460096FFF752
:1080200021FF064B9B5DE10043F0010341EAC321C0
:10803000214341F4F8612846D5E700BF840E0608C5
:108040002DE9F7431F2B0A9F06460C461546984616
:1080500010D841EA0203072B0CD8204BD95D44EA23
:10806000C12141EAC20141EA881103B0BDE8F043F1
:10807000FFF7B7BD08FA07F2B2F5805F0DD245EA07
:10808000471141F4784142EA043241F08001304620
:1080900003B0BDE8F043FFF7AEBD4FF0010909FAA8
:1080A00005F949F434413046FFF79BFDA8F11F0361
:1080B0002A46294630460097FFF7D4FE074BDB5D82
:1080C00044EAC50141EAC32141F4F8613046FFF7B3
:1080D00088FD49F43C413046C7E700BF840E0608DE
:1080E000436953F821104368CB1A043B013110B4A3
:1080F000C3F34A0204460ED0D91C0CDA23F4FF6104
:1081000021F0070111F5006F05D15DF8044B42F431
:108110006041FFF766BDC3F30A33204642F438429C
:108120005DF8044B43F47041FFF765BD436953F8B4
:1081300022204368D31A043B013230B405464FEA8B
:1081400063040ED0DA1C0CDA23F0FF0212F5807FF4
:1081500007D1E4B244EA012141F4504130BCFFF7B9
:1081600040BD5A11C4F30A0402F4005222439C1287
:10817000181204F48064C3F3053300F40060234351
:10818000024343EA8111284642F4004230BC41F4E4
:108190007041FFF730BD37B5144602220B460092FE
:1081A000214607220546FFF70BFFE10041F48F410E
:1081B000284603B0BDE83040FFF713BD07289ABF3B
:1081C000024B33F810004FF413707047880E060806
:1081D000C36C19440369C164012B04DD436D5A8CDF
:1081E0009142C8BF5984704770474FF0FF31FFF785
:1081F000EFBFFFF7FABF6FF00301FFF7E9BF70476A
:1082000038B5C36C1944036A9942054608D9083148
:1082100021F00304406AE100F8F745F8C5E9084099
:1082200038BD70B504460E4601211546FFF7E8FF3C
:10823000E16C626A02EBC10302F8316001215970FE
:108240005D602046BDE87040FFF7C2BF70B50446D0
:108250000E4601211546FFF7D3FFE16C626A02EB7F
:10826000C10302F8316002225A705D60204601218C
:10827000BDE87040FFF7ACBF00221146FFF7E6BF34
:108280000A460221FFF7E2BF70B50D1E044605DD68
:10829000FFF7B6FF00231E46AB4205DB294620460A
:1082A000BDE87040FFF794BFE26C616A1A4401EBCD
:1082B000C200012D46700CBF94F82800002001F880
:1082C00032000133E8E7F8B5D0E90B530133AB4294
:1082D00004460E46174606D90435406BA900F7F749
:1082E000E2FFE5626063D4E90C30C6F30E015A1C6C
:1082F000226300EB830541EAC73220F823204FF6C2
:10830000FF73A06D6B8032460021FFF732FEA06D37
:108310000022BDE8F8400321FFF7FCBD0246007DC6
:1083200028B1D36C526A5B1A013B12F833007047D4
:1083300037B5456DED8AED070B46144608D5022288
:108340000092806D06222146FFF77AFE03B030BD11
:10835000806D03B0BDE83040FFF7DCBD70B5002490
:1083600005462646EB6CA34200DC70BD6B6A03EB4E
:10837000C4035A78012A07D15E70B5F84A105A68CA
:1083800021442846FFF7D4FF0134EBE7F8B5044653
:108390001E4617460D46FFF7E1FFA06D3A463146EF
:1083A000FFF741FDA06D29460322BDE8F840FFF725
:1083B000F2BE38B504460D46FFF7D0FFA06D294642
:1083C0000322BDE83840FFF7E6BE10B50821044699
:1083D000FFF7EFFF002220461146BDE81040FFF7EF
:1083E00020BFF8B5044617461E460D46FFF7B6FFF8
:1083F000A06D3A460021FFF716FDA06D324601211F
:10840000FFF711FDA06D29460322BDE8F840FFF7F4
:10841000C2BEF8B5C76C04460E46BF1A0025E36C11
:10842000AB4200DCF8BDBD4211D0636A03EBC5036B
:108430005A78012A0BD15A68B24208D100225A70E8
:10844000B4F84A10324629442046FFF771FF01353F
:10845000E5E738B5002205460C461146FFF7D9FF7F
:10846000E200A86D42F002020021FFF7DCFC0022CE
:1084700028461146BDE83840FFF7D3BE13B5446D1A
:10848000E48AE407134607D502220092806D062293
:10849000FFF796FD02B010BD806D02B0BDE8104040
:1084A000FFF74CBDF8B5C3699E5C602E04461546C7
:1084B00006D1476813480A46134907F0C3FD3860E0
:1084C000022D0DD8636D9A8C52B9DB8ADB0707D475
:1084D0000E4B5A5D31462046BDE8F840FFF7A1BE7D
:1084E000002211462046FFF794FFB4F84A20636C3F
:1084F0001A44521B013A00212046FFF7BFFF002219
:10850000E8E700BFFC16060883B80508880F0608D0
:1085100073B503681A785D88042A04BF5A6842F864
:1085200025106A1C044602265A800021B0F8482013
:10853000FFF7A4FF00960022A06D33461146FFF717
:108540003FFD00960022A06D2B461146FFF738FD37
:1085500002B070BD73B5002204460D461146FFF708
:1085600058FF626D2068D38A43F02003D3822946E6
:10857000FEF7C4FD0226B4F8482005460021204637
:10858000FFF77CFF00960022A06D11460123FFF744
:1085900017FD00960022A06D11460323FFF710FD82
:1085A00000960022A06D11462B46FFF709FD002220
:1085B0001146204602B0BDE87040FFF732BE000011
:1085C0000D2902D10749FFF7C5BF0F2903D10022AA
:1085D0005421FFF73BBEB1F10E0218BF0122012169
:1085E000F7E700BFDC230608F8B5C76C446A07F15B
:1085F0000053023B04EBC3040546D4E9020184E8BE
:108600000300667856B9B5F84A203A44013A314633
:108610002846FFF733FF01236370666028464FF05A
:10862000FF31BDE8F840FFF7D3BDF8B504461E465C
:1086300017460D46FFF792FEA06D3A463146FFF70A
:10864000F2FBA06D29460322BDE8F840FFF7A3BD69
:1086500010B402F1290400230A46E1B25DF8044B8C
:10866000FFF7E3BF70B504460E46154662B1037DC1
:1086700053B1084604F004FF021E05DD20467021B8
:10868000BDE87040FFF7E2BD06353246E9B220464C
:108690000023FFF7CAFF002220461146BDE87040C4
:1086A000FFF7BFBD07B51346022200920722FFF76E
:1086B00087FC03B05DF804FB38B50D4614463BB9A2
:1086C000037D2BB1806D5268FFF7ADFB207838BD7C
:1086D000237833B96268806D2946FFF7A4FB002038
:1086E000F5E7012B06D162680132806D2946FFF75C
:1086F000D9FFF4E79A1E012A04D86268520042F0BA
:108700000102E8E7542B01D10022EEE7014804F012
:10871000C3FC00BF98B80508F8B50546FFF71EFE74
:1087200000242746EB6CA34200DCF8BD6E6A06EB22
:10873000C4025378022B0ED1577001210023284622
:10874000FFF7BAFF06F83400B5F84A1001222144B9
:108750002846FFF7EDFD0134E4E738B504460D4641
:10876000FFF7DAFFA06D2946FFF7BAFCA36D0122DF
:108770005A7038BDF8B504460E4617460A461946E3
:108780001D46FFF746FEE36C616A9B1B01EBC302CB
:1087900011F833303B705378012B0DD0022B14D0DD
:1087A000CBB9B4F84A20E36C1A44921B2946204600
:1087B000BDE8F840FFF762BE5268AA420BD0A06D38
:1087C0002946BDE8F840FFF77ABA0023294620463B
:1087D000FFF772FF3870F8BD10B5134604460A461D
:1087E0000121FFF7C7FF20464FF0FF31BDE81040E1
:1087F000FFF7EEBC70B5049E04461D46FFF7ECFF84
:10880000324629462046BDE87040FFF7E5BFF0B587
:1088100085B001250DF10F030DF10E010095002229
:108820000446FFF7E7FF9DF80F709DF80E602A469B
:1088300039462046FFF7F5FC314620460022FFF777
:10884000F0FC2A4639462046FFF7EBFC0022314671
:10885000204605B0BDE8F040FFF7E3BC2DE9F0414C
:10886000DDE9068604461D46089FFFF7B5FF424630
:1088700029462046FFF7B0FF3A4631462046BDE87C
:10888000F041FFF7A9BF2DE9F04186B002260DF1B6
:108890001703012501930DF115010DF11603029641
:1088A000009500220446FFF7D9FF9DF817809DF838
:1088B00015109DF8167020460022FFF7B2FC3246D4
:1088C00041462046FFF7ADFC2A463946204606B011
:1088D000BDE8F041FFF7A5BC30B587B00DF1170337
:1088E0000025019302230446009301220DF1160393
:1088F0000DF115010295FFF7B1FF20461921FFF791
:1089000058FD2A462946204607B0BDE83040FFF70B
:1089100088BC73B504460E46154672B901220DF1A6
:108920000701FFF759FF0C3500233246E9B2204614
:1089300002B0BDE87040FFF778BE0021FFF7EEFC03
:1089400020B901220DF107012046EAE70A46204638
:108950000DF10701FFF740FF9DF807202046012396
:108960000421FFF713FDA06D00220121FFF7A7F9F5
:10897000D9E7000037B500220DF107010446FFF7E3
:108980002BFF9DF807302BB107490848656807F0B1
:1089900059FB286022212046FFF70BFDA36D012221
:1089A0005A7003B030BD00BFA6B80508FC16060813
:1089B000022A7FB504460E46154614D8436D9A8C9C
:1089C0008AB9DB8ADB070ED4184B0DF10F015A5D13
:1089D000FFF702FFE3699DF80F10585D602813D17F
:1089E000595504B070BD0DF10F0120460022FFF76C
:1089F000F3FE626CB4F84A3013445B1B0022591E2C
:108A00002046FFF795FCE5E78842EAD0FFF7D6FB62
:108A100002460846FFF7D2FB0549646800901346FA
:108A20000448324607F00EFB2060DAE7880F06089C
:108A3000B0B80508FC16060870B504460D46164683
:108A40004BB90F21FFF7BCFD324629462046BDE851
:108A50007040FFF7ADBF70BD03297FB504461646D1
:108A600013D101220DF10F01FFF7B6FE1825314693
:108A7000204600230DF10F02FFF77CFE2946204619
:108A800004B0BDE87040FFF794BC052906D101226F
:108A90000DF10F01FFF7A0FE1725E8E70223009371
:108AA00001220DF10F030DF10E01FFF7A3FE1925B1
:108AB000DDE7F0B5044685B00E461546CAB9022377
:108AC000077D02750DF10E01009301220DF10F03D8
:108AD000FFF790FE27752B46324623212046FFF7ED
:108AE000A4FD00221146204605B0BDE8F040FFF786
:108AF00098BB012A09D100230DF10F022946FFF787
:108B000039FE2B4632462421E8E70DF10F01002201
:108B1000FFF762FE2521204605B0BDE8F040FFF7D3
:108B200048BC10B50446D0E90C3003F18043013B4A
:108B300000EB8303DA7822F08002DA70043B98427B
:108B40000BD893F90320002AF8DA1A88A06DC2F333
:108B50000E020021FFF70DFA05E059B9A06D4FF4A0
:108B60000051FFF73EF8A06D0022BDE81040032140
:108B7000FFF7D0B910BD10B504460121FFF7D1FFB2
:108B8000A06D01220021FFF7D9F9002220461146ED
:108B9000BDE81040FFF745BB73B5046B05460E46B4
:108BA000DCB1436B04F18044013C03EB840292F995
:108BB0000120002A20DA33F82430C3F30E038B425D
:108BC0001AD100230DF107020121FFF7D3FDA86D93
:108BD00000220121FFF79EF901242846FFF79CFDA2
:108BE000A86D3146FEF7DEFF44B10021284602B0F1
:108BF000BDE87040FFF795BF0024EEE702B070BDFE
:108C000038B50D46044611467AB1806D4FF40051D7
:108C1000FEF7E7FFA06D00220121FFF77BF929464F
:108C20002046BDE83840FFF798BDFFF77AFFF6E72A
:108C30002DE9F04104460D4672B3D0E90C3C03F136
:108C40008043013B0CEB83030021184616460F4678
:108C500090F901E0BEF1000F09DA90F903E0BEF1EE
:108C6000000F04DA002F08BF0746E1B90146013EB4
:108C7000A0F10400ECD1A06D21BB6FF0030672439C
:108C80009E18B44518D94FF40051FEF7AAFFA06D05
:108C900000220321FFF73EF925F400412046BDE8FC
:108CA000F041FFF75ABDB0F80080B1F802E068F378
:108CB0000E0EA1F802E0D9E79A5AC2F30E02FFF7AE
:108CC00058F9E4E74B8847F6FE7262F30E034B80D7
:108CD00025F400423146FFF74CF9A06D32461321CE
:108CE000FFF718F9A06D32463146FFF79CF8A06DEA
:108CF00032460121FFF70EF93D88C5F30E05CBE79B
:108D00007FB504460E4615468AB90DF10F01FFF7EF
:108D100063FD3246204601230921FFF786FC2A46DF
:108D20002946204604B0BDE87040FFF77ABA012A10
:108D300035D11146FFF7F2FA024688B902230093B3
:108D40000DF10E010DF10F032046FFF753FD012336
:108D500032460E21204604B0BDE87040FFF765BCE6
:108D60000DF10F02204600230221FFF703FD2B46E1
:108D70009DF80F2020460421FFF708FBA06D00227C
:108D80000221FEF79CFF0DF10E0120460022FFF7A5
:108D900023FD4FF0FF312046FFF71AFAD7E70DF118
:108DA0000F010022FFF718FDA06D4FF40851FEF7E8
:108DB00018FFCCE738B5FFF718FA04460122806D9A
:108DC0000021FFF7BBF822212046FFF7F2FAD4E991
:108DD0000C35013B05EB830523636B8847F6FF7277
:108DE000C3F30E03934228D01322A06D0021FFF796
:108DF000A5F8A06D4FF42051FEF7F3FEA368A06D17
:108E00001A680021FFF792F9698847F6FE73C1F3EB
:108E10000E029A420BD1A06D4FF48E41FEF7E1FE97
:108E2000A36820461968BDE83840FFF7B5BEC1F316
:108E30000E012046FFF791FCF2E738BD2DE9F34122
:108E40000E460021174604461D46FFF767FA024604
:108E500048BB0DF107012046FFF7BEFC1DB90121FB
:108E60002046FFF7B5F910212046FFF7A2FA1DB9F9
:108E70009DF8073084F828302046FFF74DFCA06DA0
:108E80004FF420515EB3FEF7ACFE3A460121A06DCF
:108E9000FFF74CF945BB4FF0FF31204602B0BDE86B
:108EA000F041FFF795B90A4620460DF10701FFF79B
:108EB00093FC1DB901212046FFF78AF99DF80700B0
:108EC000431E022BD3D9FFF779F90949D4F804805E
:108ED0000246084807F0B6F8C8F80000C7E7FEF7F2
:108EE00080FE3A463146D2E702B0BDE8F08100BFCD
:108EF000C0B80508FC1606080023FFF79FBF012332
:108F0000FFF79CBF426D83682DE9F341D58A928CAF
:108F10001E68C66005F011031343044600F0F98093
:108F200015F0010506F1020721D1B0F848202946C5
:108F30004FF00208FFF7A2FACDF80080A06D0123E0
:108F40002A462946FFF73CF8CDF800802A46A06D56
:108F500001232946FFF734F805212046FFF729FAB7
:108F6000B4F848102A4601312046FFF7E1F9D4E968
:108F700015309A8C002A67D1D98A11F0010508D1E1
:108F80004FF42051FEF72DFEA06D3A462946FFF71B
:108F9000CDF800221146A06DFEF7E4FF2021204607
:108FA000FFF707FA4FF42051A06DFEF71AFE3A467C
:108FB0000021A06DFFF7BAF8636DD98A11F00101A5
:108FC00000F08E80A06D012200210225FEF7B6FF81
:108FD0000095A06D052306220021FFF731F8A06D52
:108FE0002A460021FEF71FFFA06DFEF744FE39461A
:108FF0002046FFF7D1FD636DDB8ADB0740F18980F6
:10900000B4F84820204601320021FFF737FAA06D5E
:109010004FF48E41FEF7E5FDA06D436823641422F2
:109020000021FEF78BFFA06D4FF40451FEF7D9FD30
:10903000A06D01221421FEF76DFF2221204602B00F
:10904000BDE8F041FFF7B5B94FF40051FEF7C9FD97
:10905000A06D00221321FEF75DFFA06D002201210B
:10906000FEF758FF751C3A46A06D0421FEF781FFFC
:1090700029462046FFF790FD00221146A06DFEF71D
:1090800071FF20212046FFF794F90336A06D4FF4BD
:109090002051FEF7A6FD3246A06D0121FFF746F8EC
:1090A000A06D4FF40051FEF79CFD0022A06D03213E
:1090B000FEF730FFA06D44F22071FEF792FD3146BD
:1090C0002046FFF769FD0322A06D0421FEF736FF5D
:1090D0004FF43051A06DFEF784FD2A46012168E768
:1090E000B4F8482020460132FFF7C8F90521204690
:1090F000FFF75FF9D4E91530D98A11F001017FF447
:1091000061AF0122FEF71AFF22212046FFF751F935
:109110006DE702B0BDE8F08170B50546D0E9156095
:10912000F68AF6070C460BD544EAC4049200FEF713
:109130007AFEA86D44F4CC51BDE87040FEF751BDF5
:10914000BDE87040FEF70EBF2DE9F84F04460F460C
:109150009146FFF703F90025A8464D4510D100269A
:10916000B3464E452BD171422046FFF731F8B4F893
:109170004A20E36C39461A44BDE8F84FFFF7CCBFEC
:10918000E66CD4F824A0013E761B0AEBC6025378A5
:10919000022B12D182F80180012339462046FFF7C5
:1091A0008BFA0AF83600B4F84A10E36C1944013916
:1091B0003A46491B2046FFF7BBF80135CDE7E36C83
:1091C000D4F824A003F1FF38A8EB06081AF83820D9
:1091D000BAB1B4F84A501D44013DAD1B2A460021E6
:1091E0002046FFF74BF91AF83820012304212046C6
:1091F000FFF7CCF8002229462046FFF799F80AF835
:1092000038B00136ADE70000037D37B504460D46A2
:1092100013B15F4803F040FF426DD38A43F001036E
:10922000D382FFF779FA012D0BD1A3681968204684
:109230000231FFF792FAA368196820460131FFF75F
:10924000ABFC012200212046FFF77EFF0022022115
:109250002046FFF76DF8A06D01220021FEF7E3FD27
:10926000A06D00221221FEF755FEA368A06D1A68BA
:109270000021FEF77EFEB4F848100022013120469E
:10928000FFF756F8E168A06DFEF72AFFA368A06D0E
:109290001968FEF787FC236BBBB1626B03F1804357
:1092A000013B02EB83039A420FD893F90310002984
:1092B00026DA1A88A06DC2F30E020021FEF759FECD
:1092C000A06D00220321FEF725FE01212046FEF7B6
:1092D000DBFFBDB9A06D14222946FEF72FFEA06D5D
:1092E0004FF40451FEF77DFCA06D01221421FEF71E
:1092F00011FE2221204603B0BDE83040FFF759B8E7
:10930000043BD0E7A368196820460231FFF744FC0C
:10931000A06D14220221FEF711FEA06D0022012192
:10932000FEF781FDA06D01221421FEF7F3FD0DF182
:10933000070120460122FFF74FFA00230DF1070233
:1093400020460121FFF716FA204602220021FEF7EF
:1093500068FF012220460221FFF7F6FE2046302159
:10936000FFF727F8A06D4FF42051FEF73AFCA368F1
:10937000A06D1A6801210132FEF7D8FE20460121B6
:10938000FEF782FF204603B0BDE83040FFF72CB95E
:10939000D6B80508F8B5164604460D46520093B1F6
:1093A000CB1C1A440221FFF7CFFE45EA0623012217
:1093B0001D212046FFF715F8002220461146BDE882
:1093C000F840FEF72EBF8B1C1A440221FFF7BCFEAB
:1093D00033462A461C21ECE72DE9F74304460F46A5
:1093E00016460121B0F84820DDF828904FF0020819
:1093F0001D46FFF743F80123CDF80080A06D1A4603
:109400001946FEF7DDFD55EA09052DD12046FEF788
:10941000A5FFA06D2A464146FEF705FD39692046A5
:10942000FFF776F8A06D03221A21FEF7B4FEA06DB7
:1094300032460121FEF7F7FC324602212046FFF7B3
:1094400083FE25B16FF001012046FEF7C1FEA06D3D
:1094500003222B21FEF79FFE00221146204603B077
:10946000BDE8F043FEF7DDBE06F102094A4641467B
:109470002046FFF769FE49462046FEF7A9FEFEF7A3
:109480006DFFCBE72DE9F341044615460F46B0F8D2
:10949000482001214FF002081E46FEF7EFFF01238E
:1094A000CDF80080A06D1A461946FEF789FD3543B8
:1094B00018D12046FEF752FFA06D2A464146FEF71E
:1094C000B2FC39692046FFF723F8A06D03221A2168
:1094D000FEF761FE00221146204602B0BDE8F041D1
:1094E000FEF79FBE204642464146FFF72DFE20462E
:1094F000FEF734FFE5E770B5042A86B004460E4651
:1095000015462AD102294FF0000518D101220DF18C
:10951000170100950DF11603FFF76CF9A06D2A46AF
:109520003146FFF7BFF826212046FEF742FF002212
:109530001146204606B0BDE87040FEF772BE0DF140
:10954000150301930123009302950DF116030222E6
:109550000DF11701FFF782F9E5E7012A01D9032A86
:1095600004D1324601212046FFF7EEFD13350023DA
:109570003246E9B22046FEF709FFD8E738B50422A3
:1095800004460D460021FFF7DFFD20460421FEF7CB
:109590001FFE1F21FEF70DFFA06D4FF42051FEF7B7
:1095A00020FBA06D2A460021FEF7C0FD00222046C8
:1095B0001146BDE83840FEF734BE37B504460D46C7
:1095C0000021FFF7AEFA20464FF0FF31FEF700FE14
:1095D000A36819680231FFF7DFFA20460022542100
:1095E000FEF734FE204600225421FEF72FFE2046CF
:1095F00000225421FEF72AFE204605220221FFF711
:10960000A3FD0322204600231C21FEF7EAFEA368E7
:1096100020461968FFF7A1F8A06D2946FEF7C2FAA7
:1096200020460121FFF77DFA20460221FEF72CFE9D
:10963000A06D01220021FEF781FCA06D4FF42051A6
:10964000FEF7CFFAA368A06D1A6802250232002146
:10965000FEF76CFD002300951A46A06D0121FEF770
:10966000AFFC204601220021FEF7DBFD002211465F
:109670002046FEF7D6FD204600225421FEF7E6FDE7
:10968000294620460522FFF75FFD002303222046DE
:109690001C21FEF7A6FE20461021FEF78AFEA06DD3
:1096A0004FF42051FEF79DFAA368A06D1A680021BF
:1096B0000132FEF73BFDA36820461968FFF76CFAFC
:1096C000A06D4FF40051FEF78CFAA06D002201212D
:1096D000FEF720FCA368196820460131FFF75CFA09
:1096E0000121204603B0BDE83040FEF771BD000007
:1096F000436D73B5DD8A15F00106044613D00122CF
:109700000021FFF721FD002202212046FEF710FE76
:109710000022A06D1146FEF786FBA06D00221221EB
:10972000FEF7F8FB1BE0027D002A47D03146FEF72A
:10973000F5FD5428C5F3871525D12046FEF755FDC4
:10974000ADB9A06D2A462946FEF7ACFF636D9A8C31
:10975000002AE2D1DB8A03F01103002BDDD1226B5A
:10976000E168204602B0BDE87040FFF761BAA06D25
:1097700032463146FEF757FB01232A460421204694
:10978000FEF704FEE2E70DF1070132462046FFF73F
:1097900023F89DF80710A9420DD02846FEF70EFDCC
:1097A00002460846FEF70AFD074966680346074871
:1097B00006F048FC3060002DC8D0DDE70DF1070150
:1097C000FFF70AF8C2E700BFDEB80508FC16060876
:1097D000F8B5164604460F46FEF7C0FD3146204652
:1097E000FEF70EFD0025E36C2A46B5420CD1B4F815
:1097F0004A20394620461A44FFF78EFC2946204667
:10980000BDE8F840FEF7E4BC5819616A013521F85B
:109810003020EAE773B50D4616460DF10701002228
:109820000446FEF7D9FF721C2A4420460221FFF7A6
:10983000CFFF012345EA06222821204602B0BDE8D9
:109840007040FEF7A3BD37B504460D4600220DF16A
:109850000701FEF7C1FF2A4620460221FFF7B8FFA5
:1098600001232A462721204603B0BDE83040FEF7F9
:109870008DBD37B50D4600220DF107010446FEF7F8
:10988000ABFF5DB1204604220121FFF7A1FF1E219D
:10989000204603B0BDE83040FEF78BBD2A46A06DE0
:1098A0000121FEF7C0FA20461E21FEF782FD2A465E
:1098B0002946204603B0BDE83040FEF7B2BC37B5BC
:1098C00004460D468AB103220121FFF73DFC022226
:1098D00001212046FFF77CFF00232A460B2120466A
:1098E00003B0BDE83040FEF7A0BE0DF10701FEF762
:1098F00073FF022211462046FFF76AFF01232A4622
:109900000A21ECE77FB5012504460DF10F030DF1A7
:109910000E0100950022FEF76DFF9DF80E109DF8D8
:109920000F6020460022FEF77CFC2A463146204686
:1099300004B0BDE87040FEF774BCF8B504460F46AD
:1099400001211D461646FEF79FFC2046FFF7DAFF71
:109950000F212046FEF734FE2046FFF7D3FF39469D
:109960002046FEF7FAFE20464FF0FF31FEF78CFC52
:1099700031462046FFF710F92046FEF736FCA06D71
:1099800001220021FEF7DAFA002211462046FEF7F6
:1099900048FCA06D4FF42051FEF723F9A06D2A4634
:1099A0000021BDE8F840FEF7C1BB0000138B2DE994
:1099B000F34104460161D81E43424341237500230D
:1099C0000E46E364118CA36962658B42154605D28D
:1099D000E069F6F768FC2B8CE061A361626D538B44
:1099E000928B1344EA8A510748BF013392074FF024
:1099F000000248BF01331146934240F0DB80227DD4
:109A0000002A40F0EB80A2699A4200F2E980226AC3
:109A1000002360219A4240F0EC80042E14BF012103
:109A20000221A06DFEF796F8626D0023A4F848307D
:109A3000938CD28A02F01101194305D0D20740F16C
:109A4000DD801523A4F848308B492068FDF756FBCC
:109A50002F8C6B8C94F814803B4406466364A06D95
:109A6000B8F1000F00F00C81626D918C002940F07C
:109A7000CA80D28A12F0010F0CD13946032F6F8BA6
:109A8000A8BF0321032F88BF01F1FF3112F0110F8E
:109A900000F0BB80B4F84820023292B2A4F84A2009
:109AA0001A44511A0227FEF7B4F80097A06D01235B
:109AB00000220721FEF784FA072200971146A06DC5
:109AC0000323FEF77DFA0722009733461146A06D67
:109AD000FEF776FA636D9A8C1AB9DB8A03F03003CD
:109AE0002BB1B4F84810A06D0022FEF713FAA06D58
:109AF00001220021FEF7E3F8A06D02220121FEF70A
:109B0000DEF80322A06D0621FEF7D9F8A06D4FF410
:109B10002451FEF766F8A368A06D1A68012104328B
:109B2000FEF704FB6A8BA06D0221FEF77CF9A06DA5
:109B3000022300224FF48541FEF7BCF8A368A06D14
:109B40001A6800210532FEF7F1FAA368A06D1968C2
:109B50000431FEF727F86B8BA06D4FF002125A43C9
:109B60000221FEF760F9A06D03222C21FEF713FB02
:109B7000A368A06D19680531FEF714F800250226C8
:109B8000636D5A8BAA4248DC032A0DD99A8C5AB9C4
:109B9000DB8ADB0708D4B4F84A20636CA06D1A4452
:109BA000033A0621FEF7CAF9204602B0BDE8F041AB
:109BB000FFF7A8B9E069815401321DE7C86A00EBDC
:109BC000C20001324178CF0741BF4788E0690909E7
:109BD000C155616D088D9042F0DC14E70022F8E772
:109BE000227D002AE2690CBF00216021D15401339B
:109BF00009E7606A20F8331001330BE70BB9132330
:109C000020E714231EE7002144E7EF8AB4F8482038
:109C1000BF067FF543AF01323FE700962B46062291
:109C2000A06D0021FEF7CCF9E3695A5D22B1012352
:109C300003212046FEF7AAFB022D12DC636D9A8CED
:109C40007AB9DA8AD2070CD4022D02D15B8B032BAE
:109C500007D10A4BA06D595D0022FEF730F801359F
:109C60008EE7B4F84A10636C194401390022491B8D
:109C70002046FEF75DFBF2E7C8100608880F0608CD
:109C8000E26B0421FDF79FFFD4E91530DF8A17F05E
:109C9000010742D0226C0421FDF795FFB4F848106B
:109CA000A06DFDF7B6FF4FF4A023A364A06D42465C
:109CB0000621FEF704F80227A06D01221421FEF709
:109CC00029F90097B4F84830A06D06224146FEF706
:109CD00077F90097A06D012342464146FEF770F9DF
:109CE0000097A06D032342464146FEF769F90097AD
:109CF000A06D334642460721FEF762F92046FFF782
:109D000001F9636D9A8C002A49D0002319462A8DE7
:109D10009A425BD802B0BDE8F081B4F84830616C7B
:109D200005339BB24FF00208A4F84A301944FDF7FE
:109D300070FFCDF80080A06D3A4601230721FEF7A1
:109D40003FF9CDF800800722A06D11460323FEF7EE
:109D500037F9CDF8008007223346A06D1146FEF793
:109D60002FF9B4F84810A06D3A46FEF7D3F8626CAC
:109D7000A06D3946FEF757F8B4F848103A46204629
:109D80000331FEF7D5FAB4F84820A06D3946FEF746
:109D9000E9F8A06D04222D21FEF7FDF9AEE7DE8A79
:109DA00016F00106B1D1104F2B8CB342ADDDB4F8E3
:109DB0004A20636C17F8011BA06D1A44013A921BEC
:109DC0000136FEF7BBF8032EEED19EE7EA6A02EBFE
:109DD000C30012F83320052A04BF4288E06903F16A
:109DE000010308BF815492E7880F06082DE9F3416B
:109DF0000E4601EB4201044615461F46FEF78EFA59
:109E000070288DF8060035D1E26C636A03EBC2035B
:109E10000021204613F80C6CFEF780FA072805464F
:109E20000DD888B12046FEF7DFFBE36C626A03F1D0
:109E30000053013B02F8336002B0BDE8F0815428C2
:109E4000F0D01F4803F028F902460DF10701204623
:109E5000FEF7C2FC2046FEF7C8F932460321012373
:109E6000FEF794FA2A463146204602B0BDE8F0419A
:109E7000FEF7D7B946EA05286FB18A1C20460221B1
:109E8000FFF762F9434600221D212046FEF7A9FA9A
:109E900000221146E8E7354304D00A462046022155
:109EA000FFF752F90DF1060120460022FEF794FC5F
:109EB000012342461B212046FEF768FAE8E700BF6F
:109EC000E6B805082DE9F041C66CD0F824C0DDF8ED
:109ED0001880013E0CEBC60715467A78012A044625
:109EE00013D1D7F804E09E450FD0C6450DD01CF81D
:109EF00036300B7079682960FEF78BFA20464FF0F8
:109F0000FF31BDE8F041FEF763B90A462B68012135
:109F10002046FEF72FFCF1E77FB5002303934FF0B7
:109F2000FF33009303AA0DF10B010446FFF7CAFFAC
:109F30009DF80B50039E294632462046FEF771F9E4
:109F400032462946204604B0BDE87040FEF769B9A4
:109F5000F7B504460E461546002A57D1134601218F
:109F60000DF10702FEF706FC022211462046FFF71C
:109F70002FFC012320460D220A21FEF756FB0DF18E
:109F8000070120460222FEF727FC0DF107012046BB
:109F90000122FEF721FC2A460DF107012046FEF7BB
:109FA0001BFC9DF80770204639460122FEF739F95F
:109FB000394620460222FEF734F902221146204695
:109FC000FFF706FC012320460C220A21FEF72DFB99
:109FD000022211462046FFF7B7F82B462A462046B4
:109FE0001C21FEF7FEF92A4629462046FEF719F9FC
:109FF0002046FEF791FB204601223146FEF763F929
:10A00000204603B0BDE8F040FFF786BFFEF784FBB3
:10A01000AB1E5A425A413146204603B0BDE8F040DB
:10A02000FEF751B970B5044686B00D46164623B901
:10A0300006B0BDE87040FEF7BBBC00221146FEF73B
:10A04000E8F9204600220121FEF7E3F932462946CD
:10A050002046FEF727FA002304934FF0FF330093C6
:10A0600004AA0DF10F012046FFF72CFF049D009577
:10A0700001262B4605AA0DF10F0120460596FFF794
:10A0800021FF022300930599A06D33462A46FDF770
:10A09000D7FF06B070BD7FB504460D46164623B9FE
:10A0A00004B0BDE87040FEF7FDB900221146FEF78E
:10A0B000B0F9324629462046FEF7F4F94FF0FF3357
:10A0C0000025009303AA0DF10B0120460395FFF72D
:10A0D000F9FE02230093039AA06D29460123FDF7A0
:10A0E0006FFF2A462946204604B0BDE87040FEF7BF
:10A0F00098B800007FB50E4600210446FEF70EF921
:10A10000831E012B05468DF80B0038D8002E34D065
:10A11000012E19D10B460391009103AA0DF10B01F9
:10A120002046FFF7CFFE039D44F240212B462A46EE
:10A13000A06DFDF7BFFD9DF80B102A46204604B028
:10A14000BDE87040FEF76DB8022E0ED10B460391AC
:10A15000009103AA0DF10B012046FFF7B3FE039D0A
:10A1600044F2C0312B462A46E2E7104B64689A5D00
:10A170000F49104805F066FF206004B070BD70B94B
:10A1800001220DF10B012046FEF726FB324611217C
:10A190002B462046FEF7FAF82A462946CEE7FEF778
:10A1A0000DF8054964680246E3E700BF0429060884
:10A1B000EEB80508FC160608F7B805082DE9FF41BA
:10A1C0000D4601210446FEF7A9F8002107468DF847
:10A1D0000A002046FEF7A2F8BB1E012B06468DF8AA
:10A1E0000B0000F2D380831E012B00F2FA80A5F150
:10A1F00009030C2B9CBF0D35EDB21F2D01D0212D75
:10A2000024D10023009301220DF10A030DF10B016B
:10A210002046FEF7EFFA9DF80A30022B07D07A4B62
:10A220007A495A5D7A48666805F00CFF30601F2D48
:10A230000CBF2E212F212046FEF7BBF80022022161
:10A24000204604B0BDE8F041FDF7EBBF0126022334
:10A25000039303AA0DF10B01204600960023FFF79C
:10A2600031FE32460DF10A012046FEF7B5FA1D2DEA
:10A270007DD8DFE805F04C4C4C4C4C4C7C7C7C7C15
:10A280007C7C7C7C7C7C7C7C7C7C7C7C252D320F6B
:10A290000F374347192DA06D9DF80A60039B4FF0BF
:10A2A000010206D14FF48141FDF704FD0122314640
:10A2B000C6E7032E0CBF44F2C0014FF48241F3E71E
:10A2C000039B01224FF48641A06DFDF7F3FC11E0E2
:10A2D000039B012244F24001F6E7039B01224FF465
:10A2E0008041F1E7039941F60903A06D43EA81112A
:10A2F000FDF777FC9DF80A100122A1E7039941F6CA
:10A300000923F2E7039B012244F24031DCE79DF888
:10A310000A609DF80B30B34205D03E493C4867685F
:10A3200005F090FE38600022032E1146204614BF2F
:10A3300006260026FEF76DF80122039BA06D4FF460
:10A340008541FDF7B7FC2E44334BA06D33F8161052
:10A35000FDF747FCA06D42F20101FDF742FC4FF40E
:10A360000051A06DFDF73DFC0022012168E7204669
:10A370000121FDF72DFF244B28495A5D24486468CC
:10A3800005F060FE206004B0BDE8F08157EA0008E7
:10A3900027D1012600960DF10A0302220DF10B01CF
:10A3A0002046FEF727FA322D17D0332D17D0464618
:10A3B00000232A4612212046FDF7E8FF56B1A06D82
:10A3C00000220121FDF77BFC0023032211212046FE
:10A3D000FDF7DCFF0022114632E70625E8E70725F6
:10A3E000E6E720464FF0FF31FDF7F2FE3846FDF775
:10A3F000E5FE02463046FDF7E1FE09496468034682
:10A40000034805F01FFEBDE70429060807B9050843
:10A41000FC16060817B90508980E06082AB905089B
:10A4200038B905082DE9F0430446C16885B0FEF748
:10A43000B3FB626DD18A928C01F0110313432ED0CD
:10A4400011F0010117D1B4F8482020460132FEF77F
:10A4500015F8636D9D8C55B9A06D4FF42051FDF733
:10A46000C0FBE268A06D01322946FDF75FFE0521C1
:10A470002046FDF79EFF21212046FDF79AFF636DE0
:10A48000DA8AD20706D49B8C23B9E16820460131D1
:10A49000FEF782FBA06D12220021FDF74FFDA06D9B
:10A4A000FDF7E9FB237D002B5ED1A36D656C5B6836
:10A4B000A36323685B88E363636D013D5E8BDF8A82
:10A4C000B3F81C90B3F81E80EA0006F0030302F014
:10A4D000780207F00F071A432D09B60845EA07036B
:10A4E000334343EA090353EA0803A06D65D1012110
:10A4F000FDF769FBB4F85060B4F85270A06D7200BB
:10A5000007F0010302F07E027F08B60957EA06054C
:10A5100042EA030218BF42F080020121FDF753FB1B
:10A52000002DEBD1636DA76D998A20687E68FCF7DA
:10A53000CFFD4749024638460FF0ECFF626D538B62
:10A54000918B108D0B44AB4271DCA36D9F88BE1BB9
:10A55000A4F850600025D4E915301A8DAA4268DCB1
:10A560004368DB1BA4F852302369042B21D1A36D6F
:10A57000D3E9027623685868237D5BB9A56BE16B4C
:10A580003544002962D001318900F5F78CFEE36B78
:10A5900040F823500023656D217DCDE90233EB8A1D
:10A5A000CDE90003033128693B463246C9B201F0C8
:10A5B00034F9012005B0BDE8F08342F080020121AA
:10A5C000FDF701FBBA012B0103F0300302F040025A
:10A5D0001A4308F001031A434FEAC90303F00803C2
:10A5E0001A43B30003F004031A43AD087F0876084A
:10A5F0004FEA59094FEA580870E7D36A03EBC103E1
:10A600005F78FF070ED55F88AF420BD1596820688D
:10A61000A76DFCF75DFD0E49024638460FF07AFF44
:10A6200001358BE701318142E7DB0521EFE70021AE
:10A63000F9E7DB6A03EBC50213F83530052B03D1CC
:10A6400052880121FDF7BFFA013584E72846A1E7CA
:10A65000857B02082DE9F04188B004460D4607AE1F
:10A66000002940F0BD800121FDF758FE07468DF816
:10A67000170078BB01462046FDF750FEC0B9012205
:10A6800031462046FEF7A8F800220DF117012046BA
:10A69000FEF7A2F804220F2102232046FDF776FEE2
:10A6A00000221146204608B0BDE8F041FDF7B9BDD3
:10A6B0003A4631462046FEF78FF89DF81C2020468A
:10A6C00001230421FDF762FEA06D3A460121FDF74A
:10A6D000F6FAD9E7E36C626A013B02EBC30032F899
:10A6E000332040F202239A422BD147684FF00108F1
:10A6F0002046FDF77AFD434632460DF11701CDF8AD
:10A7000000800795FFF7DEFB20462A462946FDF725
:10A7100080FE9DF8170006280DD007280ED00528CA
:10A7200054D10095079AA06D3B462946FDF748FC99
:10A7300000220221B6E7CDF80080F3E70223009360
:10A74000F0E72B460791324606A920460095FFF711
:10A75000B9FB2A460DF117012046FEF73DF82046C9
:10A760002A462946FDF755FE9DF81800831E012B49
:10A7700008D9FDF723FDA14965680246A04805F008
:10A7800061FC28609DF8170006280BD0072813D01D
:10A7900005281BD10799890141F4B841A06DFDF747
:10A7A00020FAC5E70799A06DC90041F04201FDF705
:10A7B00018FA4FF4B541F1E70799A06DC90041F0CF
:10A7C0008201FDF70EFA4FF4B141E7E7FDF7F6FC21
:10A7D0008C49656802468A4805F034FC2860A7E782
:10A7E000012940F0FB80FDF799FD07468DF8150023
:10A7F00050BB01462046FDF791FD022105468DF82C
:10A8000018002046FDF78AFD05438DF81C0008D08E
:10A81000394620460322FEF797FC03212046FDF728
:10A82000D7FC0223CDE901630023009306A920464B
:10A830000DF115030122FEF711F80F21204608B093
:10A84000BDE8F041FDF7B5BDE36C626A013B02EB88
:10A85000C30132F8332040F202239A423ED120460F
:10A86000D1F80480FDF7C1FC02230022CDE90623C4
:10A87000009306AA2B460DF11501FFF723FB069F57
:10A8800000953B46204632460DF11701FFF71AFBB3
:10A890009DF81700431E022B08D9FDF78FFC5A497B
:10A8A00065680246564805F0CDFB28609DF8150006
:10A8B00006280FD007280FD0052840F085800023F8
:10A8C00000930799A06D43463A46FDF7B9FB08B0DF
:10A8D000BDE8F0810123F3E70223F1E702230793A8
:10A8E000009306AA00230DF1160120460695FFF7F6
:10A8F000E9FA204600220DF11501FDF76DFF9DF8E4
:10A900001600831E012B08D9FDF758FC3F496568E6
:10A9100002463B4805F096FB2860069D0095002303
:10A92000204632460DF11701FFF7CCFA9DF81700CB
:10A93000431E022B08D9FDF741FC334966680246E5
:10A940002F4805F07FFB30609DF8150006280ED0DB
:10A95000072825D0052837D1079941EA851141F408
:10A96000A841A06D08B0BDE8F041FDF73AB9012655
:10A97000AE40A06D46F43441FDF733F945EAC50118
:10A9800041F04001A06DFDF72CF9079941EA8511CE
:10A9900041F4A441A06DFDF724F946F43C41E0E701
:10A9A0000126AE40A06D46F43441FDF71AF945EAA0
:10A9B000C50141F08001A06DFDF713F9079941EA47
:10A9C000851141F4A041E5E7FDF7F8FB1049646803
:10A9D00002460B4805F036FB206078E70025334639
:10A9E00006A900950122FDF705FF02232A460F2143
:10A9F000204608B0BDE8F041FDF7C8BC5BB90508CA
:10AA0000FC16060852B9050865B9050878B90508A5
:10AA10006EB905082DE9F04180465C2016460F46C8
:10AA20001D46F5F73EFC866008260446C0E900870F
:10AA300006624020F5F71CFCE66260622020F5F714
:10AA400017FC60632020F5F72CFC2946A065FDF774
:10AA50006EF82046BDE8F08110B504460021806DF7
:10AA6000FDF76DF8A06DF5F72BFC606BF5F728FC92
:10AA7000E069F5F725FC606AF5F722FC2046BDE8A1
:10AA80001040F5F71DBC000002F00F03022B10B5BB
:10AA9000044608D00A460C490C4805F0D3FA636A0C
:10AAA0001860002010BD836A12090020834204D17F
:10AAB000238C042BF5D10649EEE7E16A51F820100A
:10AAC0009142EFD00130F1E783B905086817060815
:10AAD00089B9050870B50646B2B1900714D110794E
:10AAE0002E2811D194687CB1A2070DD16568EAB215
:10AAF000922A09D12D0A022D06D1A2681A60049B60
:10AB0000E2681A60012070BD0A460448044905F055
:10AB100099FA736A18600020F5E700BF6817060805
:10AB200095B905087FB504460D46104603A91E4693
:10AB3000F8F776FD48B90C490C482A4605F082FA28
:10AB4000636A1860002004B070BD039803F084F9B4
:10AB500030EA06020346F6D0054900962A46034825
:10AB600005F070FAECE700BFB1B9050868170608F0
:10AB7000B7B90508038C032B70B5C46A03D1856A85
:10AB800000239D4205D144F82120FDF70BF8012058
:10AB900070BD54F82360964201D00133F1E70020E4
:10ABA000F6E7FDF768B8032910B504460184426250
:10ABB0000FD1826AC06A002192001CF0DFF80121E7
:10ABC0002046FCF7C7FF20460021BDE81040FDF7F6
:10ABD00020B8042914BF01210221F1E700F00F037E
:10ABE000022B02D10009F6F766BA0148704700BF90
:10ABF000AFD2050870B5054610460E46FFF7EEFFCA
:10AC00000378732B19D14378BBB103460A22002085
:10AC100013F8014F5CB91F2808D90B490B481F23B3
:10AC2000324605F00FFA6B6A1860002070BD303CA8
:10AC3000092C02D802FB0040EAE7054903483246E6
:10AC400005F000FAEFE700BFCDB905086817060860
:10AC5000DAB90508F8B5054610460E461F46FFF757
:10AC6000BDFF174C01780022A44663788B421BD1AC
:10AC700090F801E0A3789E4516D190F802E0E378C1
:10AC8000734511D16BB91CF82200B84208D90D499F
:10AC90000D483B46324605F0D5F96B6A1860002036
:10ACA000F8BDC378002BEED00132152A04F104045C
:10ACB000DBD106490448324605F0C4F9EDE700BF90
:10ACC00040100608CDB9050868170608E3B905085D
:10ACD0002DE9F34706460F46002A3CD093073AD1A8
:10ACE00013792F2B37D1926802F00F03022B08D172
:10ACF0000F23FFF7AFFF01248440204602B0BDE8D8
:10AD0000F08742B312F0030A25D113799F2B22D189
:10AD1000D5682B79A12B1ED192680F23FFF79AFFDC
:10AD20004FF0010909FA00F401AAA22105F1080077
:10AD3000F8F7C2FE8046C245DFDA019A0F2352F8C7
:10AD40002A2039463046FFF785FF09FA00F0044310
:10AD50000AF1010AEFE7044904483A4605F072F99E
:10AD6000736A00241860C8E7E9B90508681706087F
:10AD700010B50446024805F0CFF8206010BD00BFB2
:10AD80006817060804292DE9F84380460C460DD8BB
:10AD9000151F01F1300930264E450DD055F8040F2E
:10ADA00000F00F03022B0AD00D4900E00D49D8F83E
:10ADB0002400FFF7DDFF00242046BDE8F8830009EA
:10ADC000F6F779F907461CF017F80228ECD13B7822
:10ADD000722BE9D17B78B342E6D10136DCE700BFC4
:10ADE00023BA0508FAB905082DE9F0470F4686B0E1
:10ADF000044603A938461E469146F6F768F90378DB
:10AE0000762B054640F01981B9F1020F40F0C6805B
:10AE1000A7F29C570E2F00F20781DFE817F00F0012
:10AE200037003A00050105010501050105018D0006
:10AE300005015F003D0032002F00BC004EF6B468F3
:10AE40004FF42C69326829462046FFF7D3FE72681A
:10AE5000074629462046FFF7CDFEFA0249EA500987
:10AE600002F47042400142EA090200F02000B901F8
:10AE700001F04001024348EA010129E04EF6B168C1
:10AE8000DEE74EF6B1684FF42469DBE74EF6B868AA
:10AE9000D6E74EF6BD68D3E73068FFF79FFEAA49B4
:10AEA0001BF0B8FFC0B132680F2329462046FFF7D8
:10AEB000D1FE07467068FFF791FEA4491BF0AAFF78
:10AEC000002840F0B1803A0342F421624EF6F1616D
:10AED0002046FCF790FEE6E10F27EBE73068FFF72E
:10AEE0007DFE03783268722B17D10F232946204646
:10AEF000FFF7B0FE2946726807462046FFF77AFE44
:10AF00004EF6106180464FEAC812D2B242EA0732CA
:10AF100042F4216241EA5801DAE729462046FFF768
:10AF200069FE2946726880460F232046FFF792FE8D
:10AF30004FF46E410746E6E74EF6905832682946D0
:10AF40002046FFF757FE05AB00930746726804AB37
:10AF500029462046FFF7BEFD002800F0A481049A90
:10AF6000072329462046FFF775FE059A064629461F
:10AF70004FF47F732046FFF7D5FDFA02B90102F4C2
:10AF8000704201F0400142EA900241EA080142F4B5
:10AF9000206231439CE74EF68058CFE7B9F1030FAA
:10AFA00042D1DFF8C081002700F1010A03224146A7
:10AFB00050461BF047FF90BB2B7983BB644B326834
:10AFC00013F8278029462046FFF714FE72680746CB
:10AFD00029462046FFF70EFEB268814629462046E4
:10AFE000FFF708FE4FEA0813DBB243F4206343EA9D
:10AFF0005003400100F02000FA0202F470420343C3
:10B00000134308F0F0084FEAC912D2B248F46E4870
:10B01000B90148EA590801F040011A432BE701370A
:10B02000042F08F10408C1D14B464A494A482A4630
:10B0300005F008F8636A186035E1B9F1030FF3D839
:10B04000DFE819F0040015001501C90240F2D243EF
:10B050009F4205D14FF43F412046FCF7C2FD22E15B
:10B0600040F2AC539F42DFD14BF63071F4E740F22F
:10B07000C632974210D1014632682046FFF704FDE0
:10B0800001462046FCF73FFE002840F00C81334982
:10B09000606AFFF76DFE06E1B7F5747F09D10146DE
:10B0A00032682046FFF7F0FC01462046FCF785FE9B
:10B0B000EAE740F2DA32974209D1014632680F23BB
:10B0C0002046FFF7C7FDC10041F48E41C4E7622B63
:10B0D0004AD1039B032B0CD0052B40F08C80C37806
:10B0E0005F2B40F0888003796E2B02D0772B40F0E5
:10B0F000828069781A4B00224FF0FF3758788842D7
:10B1000005D195F802C09878844508BF1F780132B0
:10B110000E2A03F10303F1D17B1C85D03268294646
:10B120002046FFF7B1FC039B052B024609D12B7982
:10B13000A3F177067342734139462046FCF701FEBE
:10B14000A2E70023F8E700BF41BA05084BBA05089B
:10B15000A00F06085EBA0508681706086BBA05084E
:10B1600004100608A10F0608692B44D14378742BFC
:10B1700041D13068FFF732FDB84B017800221F46FD
:10B180005E788E4222D190F801C09E78B4451DD1E0
:10B190008678DEB9AE1C31460B460131187800289E
:10B1A000FAD1691D8B423FF63FAF02EB4202082104
:10B1B000BF5CFA43D200F800013B0A4008409E42BF
:10B1C0000AD941EA071141F43F4145E701320E2A0D
:10B1D00003F10303D4D127E713F801C9BCF1740FBD
:10B1E0004FEA510101D10143E9E7BCF1650F7FF45A
:10B1F0001BAF1143E3E740F2FB339F4202D14BF216
:10B20000726129E7B7F57F7F02D14BF2626123E7D4
:10B2100040F2FE439F4213D1326829462046FFF791
:10B2200057FD10F43F4F024607D145044ABFC1B253
:10B2300040F4344141F435410EE74EF62D1147E616
:10B24000782F7FF4F1AE326829462046FFF740FDA3
:10B2500010F4FE4F024607D110044ABFD1B242F4A7
:10B260003C4141F43D41F7E64EF6BD0130E67368DE
:10B2700003F00F03022B40F09E8040F2C3439F4235
:10B2800014D1014632680F232046FFF7E3FC7268B1
:10B29000074629460F232046FFF7DCFC39460246C5
:10B2A0002046FCF70CFD06B0BDE8F08740F2EB331A
:10B2B0009F421CD14FF6B0294FF2800732680F230E
:10B2C00029462046FFF7C6FC7268804629460F23B0
:10B2D0002046FFF7BFFC47EA000242EA082249EA9B
:10B2E0000001F5E54FF690294FF2A007E6E740F29E
:10B2F00009539F42F6D040F2C7439F422AD1326899
:10B300000C2301462046FFF7A5FC07467068FFF7AF
:10B3100065FC0146064652481BF07CFD0346A0B181
:10B32000504831461BF076FD70B12A464E494F48D1
:10B3300004F088FE636A0022186042EA072242F4A1
:10B3400000424FF2EF31C3E50123494A03EBC30347
:10B35000D25CF2E7B7F56E7F15D14FF480473268C3
:10B36000294607232046FFF775FC72688046294668
:10B3700007232046FFF76EFC424603463946204627
:10B38000FCF798FC8FE7DFF8F080002703224146A6
:10B3900028461BF057FD40B9EB7833B9354B13F80D
:10B3A00027703F0147F48047D9E701370F2F08F195
:10B3B0000408EBD138E640F2C6439F422BD840F256
:10B3C000C2439F421FD840F2ED339F423CD0B7F5B5
:10B3D000926F00F0888040F2AE339F4237D040F247
:10B3E0008E439F4200F0DF8040F28F439F4200F087
:10B3F000DC8040F291439F4200F0D980972F40F0CB
:10B400009F800323A2E0A7F2C447022F22D8DFE8DF
:10B4100007F04C354F0040F26B539F4240F08C8058
:10B420004FF460573268072329462046FFF712FC85
:10B43000294680467268FF232046FFF773FB47EAE0
:10B44000000141EA082107E64FF42057EAE74FF4EC
:10B450004057E7E74FF40057E4E700BF0410060841
:10B460002F1006083810060851BA05086817060894
:10B470002E100608C80F0608C90F06084FF240280C
:10B4800032680F2329462046FFF7E4FB726807461F
:10B490004FF6FF7329462046FFF744FB3A46034622
:10B4A00041462046FCF71DFCFDE64FF2C028E7E7C9
:10B4B000014632680F232046FFF7CCFB294607469A
:10B4C00072684FF0FF332046FFF72CFB3A4683B2F9
:10B4D00005464FF240212046FCF703FC2B0C3A4670
:10B4E0004FF2C021DDE7014632680F232046FFF707
:10B4F000B1FB05AB00930746726804AB29462046B2
:10B50000FFF7E8FA00283FF4CEAE049A0F2329464D
:10B510002046FFF79FFB059A06462946FF23204653
:10B52000FFF700FB820842EA073246F4684142F422
:10B53000706241F05001CBE440F267539F4238D033
:10B5400040F269539F427FF46FAD0523824A29463A
:10B5500032F82370326807232046FFF77BFB05ABE8
:10B5600000938046726804AB29462046FFF7B2FA82
:10B5700000283FF459AD049A294607232046FFF7D7
:10B5800069FBF904059A064615D51F23294620466E
:10B59000FFF7C8FA47EA0807800147EAC60700F440
:10B5A000F861394358E50023D0E70123CEE74B4645
:10B5B000CCE70423CAE73B0406D53E2329462046B0
:10B5C000FFF7B0FA4008E5E77C2329462046FFF75D
:10B5D000A9FA8008DEE740F29F439F4221D100276D
:10B5E0003268072329462046FFF734FB72688146FC
:10B5F000072329462046FFF72DFB29468046B268DF
:10B600001F232046FFF78EFA47EA090747EA80170B
:10B6100047EAC80120E54FF40067E1E74FF480579F
:10B62000DEE7B7F5946FF6D040F2C1339F42F5D014
:10B6300040F2AE339F422BD14FF4C05832680723FB
:10B6400029462046FFF706FB72680723074629466E
:10B650002046FFF7FFFAB26802F00F03022B814683
:10B660000ED1072329462046FFF7F4FA47EAC9011D
:10B6700041EA080141EA8011EEE44FF4D058DDE7D9
:10B6800007232946204648F48068FFF74BFAEDE788
:10B6900040F23C539F4222D14FF6903832680F233C
:10B6A00029462046FFF7D6FA726881460F232946BD
:10B6B0002046FFF7CFFAB268074629460F232046F7
:10B6C000FFF7C8FA40EA092040F4704242F0F00265
:10B6D00048EA0701FFF7FCBB4FF6B038DEE740F25F
:10B6E0008D539F42F8D040F26B539F42C5D0B7F5BF
:10B6F000AD6F7FF499AC014632680F232046FFF707
:10B70000A9FA72680F23294607462046FFF7A2FAD6
:10B7100005AB00938046B26804AB29462046FFF78C
:10B72000D9F900283FF4BFAD049A0F2329462046DB
:10B73000FFF790FA059A06462946FF232046FFF7B1
:10B74000F1F93F0247EA083746F4684147EA9002B8
:10B7500041F04001FFF7BCBBB00F060838B5054605
:10B760003020F4F785FD2022044600211BF006FB63
:10B7700029462046FCF7DBF9A562A800F4F778FD1E
:10B78000E062204638BD10B50446C06AF4F798FD63
:10B7900020460021FCF7D3F92046BDE81040F4F71D
:10B7A0008FBD012910B5136823D90178302920D124
:10B7B000417841F02001782900F1020406D133F0EC
:10B7C000100314D110231360201A10BD6F2904D167
:10B7D00033F008030BD10823F5E7622904D133F0D5
:10B7E000020304D10223EEE70BB9012313600446E0
:10B7F000EAE7002BFBD10A23F8E708B51020F4F79D
:10B8000050FD0123837008BD10B503F0010302242D
:10B81000C0E901128470C37010BD9DF8043042600D
:10B8200003F00103C370009B8360029B0373C36832
:10B83000039A817062F31F23C360704770B504469A
:10B840000D4623881046CBB10A460023214605F059
:10B85000EBF82346002213F8011B1D1B090605F116
:10B86000FF3503D4D30725D51C4B19E013F8011B72
:10B87000C1F3801606FA05F52A43EEE7A378666859
:10B88000042B0FD0052B16D0032B0A46A368314694
:10B890001DD105F0C9F8124B0360E37853B1114B89
:10B8A000036007E01049A468102002F0C7F9C0E95E
:10B8B0000154C66070BD0D49257BE468102002F07C
:10B8C000BDF9C4F31724C0E90156C460F2E705F0DE
:10B8D000ABF8E378002BEDD0C6E700BF801C06086C
:10B8E000381B0608641C0608201B0608081B0608EF
:10B8F00038B5144612F4807218BF1A461D46FFF779
:10B900009DFF620902F008022A44E1B2BDE8384016
:10B9100003F070BAD0E90003184770B505460C462D
:10B920008E18B44200D170BDD5E90003984704F8E1
:10B93000010BF6E738B504460025D4E90003984723
:10B9400000F07F0343EAC5150306F6D4284638BD48
:10B950002DE9F04186B00546FFF7DCFFC4B2042CA8
:10B9600006D8284B53F82440204606B0BDE8F081A5
:10B970002846FFF7DFFF064630B9062C04D12846DB
:10B98000FFF7C8FF204CEFE70A2C10D1002130460A
:10B9900009F082FF0027044600F10408B742E3D013
:10B9A0002846FFF7D5FF013748F8040FF6E7314680
:10B9B00002A8F5F769FC049932462846FFF7ADFF67
:10B9C000631F012B0CD82846FFF7A4FF052C02A803
:10B9D00003D108F083F80446C6E708F085F8FAE7D3
:10B9E000072CDDE903104FF0000303D10A22D7F73B
:10B9F000F5FAF0E7093C624200936241D7F726FC72
:10BA0000E9E700BF94100608342406082DE9F8433E
:10BA10002B4E04460F46904600252068FFF77AFF1C
:10BA20005FFA80F9B9F1FF0F01D1BDE8F883C107D2
:10BA30000CD52068FFF77EFFC20748BFA3684FEA16
:10BA400050054FEA850554BFED19ED184FEA59032B
:10BA5000082B21D8DFE803F0050505050505171BB0
:10BA60001E00DB070DD52068FFF764FF5FEA990928
:10BA700023D0B9F1010F0CBFA368E3680246294641
:10BA800016E00120F2E763689B680120F6E763682F
:10BA9000DB68FAE73346F8E703F18043084A093BDD
:10BAA00052F82330F1E751F804CB9C4441F804CC20
:10BAB000013AF8D205EB8005AFE74346DEE700BF69
:10BAC000C81006082DE9F04F8FB080460991FFF7A6
:10BAD00031FF00F003039A1C0492C20800F004092D
:10BAE0000792002B3FD11046F4F7C2FB4FF0000A3B
:10BAF0000146079A06464046FFF70FFF5746CDF826
:10BB000020A05446CDF814A05546B9F1000F00F01E
:10BB100098804046FFF70EFF049B8146032B08BF29
:10BB200001308000F4F7A4FB4FF0000B0690CB45EA
:10BB30007DD1FFF762FE049B022B834640F08C8090
:10BB40003246002312F8011B901B090600F1FF305A
:10BB50007AD4069A9BB231465846FFF755FE5846AE
:10BB60000FB0BDE8F08F0798F4F782FB079A014603
:10BB700006464046FFF7D1FE049B032B404618D1F2
:10BB8000FFF7D8FE04463018335D411C00270A1A1F
:10BB90001D0602F1FF3204D44FF0000ACDF820A0B8
:10BBA000B0E711F8013BC3F3801505FA02F2174321
:10BBB000EDE7FFF7BFFE049B052B07460BD1404680
:10BBC000FFF7B8FE08904046FFF7B4FE0024824617
:10BBD0000594254699E710F0200B23D04046FFF747
:10BBE000A9FE824617F0400002D04046FFF7A2FEB1
:10BBF0001AEB000418D0C51C25F003050AEB05005C
:10BC0000F4F74FFB05900544BBF1000F04D05246FA
:10BC100029464046FFF781FE4FF0000ACDF820A0EC
:10BC2000544672E7DA46DDE7A2460894D0E7099960
:10BC30004046FFF747FF069B43F82B000BF1010B33
:10BC400075E7CDF8189074E712F8011BC1F3801462
:10BC500004FA00F0034377E7099BCDF82880CDE98B
:10BC60000B35059B0D93FB0610D5154DD5F8CC0073
:10BC700020B9014606F0BEF8C5F8CC00314605F003
:10BC80002EFE324631460AA8FFF7C0FE049B032B66
:10BC900006D13444B9F1000F03D0069B43F8294084
:10BCA000069C089B0293BFB2CDE90047079B04990D
:10BCB000CDF80CA032465846FFF7AFFD4FE700BF66
:10BCC000340000202DE9F04786B0836804930446D1
:10BCD0000368059302A80F463E49F4F767FA042269
:10BCE0000DEB02012046FFF718FE9DF806509DF867
:10BCF0000420AB084D2A03F02F030CD19DF805203A
:10BD0000062A08D11BB105F00302032A03D19DF8CE
:10BD100007201F2A02D9304800F0F0FF23B1043B6E
:10BD2000032B01D92D48F7E715F04005F3D1204644
:10BD3000FFF700FE81462046FFF7FCFD4FEA49066B
:10BD40000336804600EB96008000D7F800A0F4F799
:10BD50008FFA26F00306CAF808003044CAF80C002F
:10BD60004D450DD10025454539682AD12046FFF7BC
:10BD7000A9FE78600120F4F721FA06B0BDE8F0874B
:10BD80002046FFF7D7FDC3074FEA500613D43046CD
:10BD9000F4F76EFA3246014682462046FFF7BDFDB3
:10BDA0002046FFF7B7FD31465046F5F7BFF8064687
:10BDB0005046F4F785FA3B689B6823F81560013517
:10BDC000CEE72046CE68FFF7C3FD46F825000135D3
:10BDD000C9E700BFF7BE02089DBA0508A9BA050861
:10BDE0001FB50C46014601A817F0CAFE214601A85E
:10BDF000FFF768FF04B010BD024B82681A61C26889
:10BE0000DA60704734000020838803F4C071B1F514
:10BE1000C07F02460FD0190604D5C37B00EB830216
:10BE20001069704713F4807006D0D37B02EB830255
:10BE30001369586870470148704700BFA97103082B
:10BE400070B5274CF5F718F800250123E561A4F833
:10BE50002432D4F828320BB1A4F82452A4F830527A
:10BE600003F0E2FF1F4B204E20486564C4E90F3504
:10BE700003211F4BA364C4F8185284F81C5203F02A
:10BE800057FD0121304603F053FDAA22BA21304666
:10BE900003F058FE00210846C4E90366C4E92C55A6
:10BEA000C4E96D55E566C4F8CC50C4F8B85005F047
:10BEB000A1FF0A21C4F8440105F011FD40F2E2613E
:10BEC000D4F8440105F00BFD002106F1440005F013
:10BED00049FE40F21A7240F2DA63C4E9522370BD9F
:10BEE00034000020381A060890000020800000204E
:10BEF000102806087047D0E90230184708B5074BEC
:10BF0000D86E08B9064808BD002241F6B241043097
:10BF100001F070FC0028F5D04068F4E73400002000
:10BF2000FC2E0608034BC0000A4640F00201D86808
:10BF300003F008BE34000020034BC10041F00201B1
:10BF4000D86803F00DBE00BF34000020034BC000D2
:10BF50000A4640F00201186903F0F4BD34000020E5
:10BF6000034BC10041F00201186903F0F9BD00BFA5
:10BF700034000020F8B51C46930707460E461546C8
:10BF800008D113689A88910615D5520610D5B38842
:10BF90009B0501D52560F8BD50B9114B9E4207D0D5
:10BFA00010490C2001F04AFEC0E901652060F2E76B
:10BFB000C4E90057EFE70C4A934202D16B68236053
:10BFC000E9E70A4A9342E5D130B101F043FE084B5C
:10BFD000834214BF06463E466B68C4E90036DAE782
:10BFE000B41F0608A8100608982806088028060826
:10BFF000E028060800232DE9F041C2E900330E468F
:10C000000746144601F026FE0A2E054602D120609E
:10C01000BDE8F081192E07D1838803F4C0731BB1EA
:10C02000144BC4E90037F3E76B7B5BB105EB83038B
:10C0300022461B693146384698476368042BE7D18E
:10C0400000236360EB7C002BE2D005EB8303F1005F
:10C050001869002241F00201043001F0CBFB0028F6
:10C06000D6D04268234629463846BDE8F041FFF75E
:10C0700081BF00BF702E0608F0B593B00546684634
:10C080000E4617461C46F4F7B3F840B93A46314617
:10C090002846FFF7AFFFF4F781F813B0F0BD002C8E
:10C0A000FBD1019B044918680AF0D8FB0028F4D1A1
:10C0B0000198F4F7B5F800BFF418060808B519B9E7
:10C0C00003F025FFF4F7ACF803F026FFFAE70EB40F
:10C0D00003B503AA52F8041B019203F04BFFF4F7D7
:10C0E0009FF8000070B5124EC4000546306944F058
:10C0F000020400222146043001F07CFB0246A0B974
:10C10000F06E30B12146043001F074FB08B1406894
:10C1100070BD00220748214601F06CFB024620B9A1
:10C12000054906482A46FFF7D2FF5068F0E700BFEE
:10C1300034000020AC2A0608B5BA0508F81706082E
:10C140000A4B10B50446D3E90303984207D0E10037
:10C15000002241F00201043001F04CFB20B92046DE
:10C16000BDE81040FFF7BEBF406810BD340000209E
:10C17000032837B505460C4607D1084601F0A4FF51
:10C1800000B30E24204603B030BDCA072FD54B1094
:10C1900008282AD801A252F820F000BF85C1020861
:10C1A000CDC10208EBC10208EBC10208C1C10208FF
:10C1B000EBC1020885C10208C9C1020885C1020895
:10C1C000002BDED01E24DDE7002BDBDAB3F1404F7D
:10C1D00006D14FF0804003B0BDE8304005F028B9EB
:10C1E0005B425B0043F00104CCE7DB43F9E7062840
:10C1F00025D101F00703022B10D08B071FD10B684C
:10C200001A7BE2B103EB82031A69204B9A4216D1E2
:10C21000486840B98B68C86801930CE0CC08204698
:10C22000F4F732FF18B1400040F00104AAE701A979
:10C230002046F4F74CFF0199F4F70EFEF3E7204691
:10C2400001F008FDC37ABBB100EB8300214603690E
:10C2500028469847B0B9042DB4D0A5F10803022BA5
:10C2600012D90B4B20465D5D01F000FD09490346E4
:10C270002A460948FFF72BFF062DECD1640044F055
:10C2800001047FE704467DE700247BE7E9420308D9
:10C2900036290608C1BA0508201706082DE9F0411D
:10C2A00005460E461746984601F0D4FC847A54B1F0
:10C2B00000EB8404434624693A4631462846A446A6
:10C2C000BDE8F0416047284601F0D0FC0249024633
:10C2D0000248FFF7FCFE00BFCABA0508201706088F
:10C2E00000231A461946FFF7D9BF0000F0B51546DE
:10C2F000124A87B00C46116904910646D16805912F
:10C3000002A80F49C2E90335F3F750FF2246376808
:10C3100031466846F7F7E4FBB4FA84F2520939462D
:10C320006846FAF78DFC044615B1FFF7D9FF0446BD
:10C330000120F3F743FF204607B0F0BD3400002092
:10C34000F9BD020807B50022019101AB0121FFF7F9
:10C35000A5FF03B05DF804FB07B5CDE900126B46FD
:10C3600000220221FFF79AFF03B05DF804FB30B40E
:10C370005568003D144618BF0125C5F1020302EBC4
:10C3800083030A462918206830BCFFF787BF0000E6
:10C3900010B5044603F064FE30B1002320461A466F
:10C3A0001946FFF77BFF0446204603F073FE28B9C9
:10C3B000BDE810400249034803F0AEBD204610BD61
:10C3C000D0BA0508201706087FB5114B0592C000AA
:10C3D00040F002000190186902900620CDE90301A7
:10C3E000D86E78B1002241F6E241043001F002FA41
:10C3F00040B1406801AB00220521FFF74FFF07B0B5
:10C400005DF804FB01A905200BF004FBF7E700BF72
:10C410003400002070B5164604460D46FFF7EAFDCD
:10C42000336893B9A30709D12268084B9A4205D112
:10C43000E28807492B460748FFF749FE204601F0EE
:10C4400015FC054902462B46F5E770BDE0280608B5
:10C45000F1BA0508F4180608FABA050807B56A46DD
:10C46000FFF7D8FFDDE9000109B102F063FC03B07A
:10C470005DF804FB2DE9FF41174606460C461D46B4
:10C4800001F0E8FB374A904208D12B463A46214654
:10C49000304604B0BDE8F04104F088BB818811F457
:10C4A000C07812D0062C2DD12F4F00233B62FFF70E
:10C4B000ABFC0346304698472860D8B93B6A002B4E
:10C4C00018BF1C462C60002015E0062C1AD101AACA
:10C4D00019213046FFF78EFD019B7BB901AA8A2105
:10C4E0003046FFF797FF039401AA00210120FFF7D0
:10C4F0003EFF2860012004B0BDE8F08101AA41465A
:10C500004046F4E7002CE9D1384601F0A3FB174977
:10C510000AF0A4F901AA60B147213046FFF76AFD8D
:10C52000019B73B101AA21462046FFF720FF286036
:10C53000C9E79B213046FFF75DFD019B0BB10397D7
:10C54000D2E70B49384603F0B9FD30B109490A4832
:10C5500003F0E2FC28600220CDE73846FFF718FF21
:10C56000F8E700BFF01B060834000020141A060884
:10C57000A819060802BB0508B01706087FB540F2E7
:10C58000933102AA0546FFF735FD029CDCB1204637
:10C5900001AA694601F0FCFC0024009BA34201D8DB
:10C5A00004B070BD019B53F8240007F0F5FD02AA0A
:10C5B000014606462846FFF72DFF02993046FFF751
:10C5C000B1FC0134E9E7284602AA40F29931FFF7AD
:10C5D00021FF029DAB68A342E2D9EB6853F8340017
:10C5E000E60080B104280ED007F0EEFD03785F2B43
:10C5F00009D0EB6853F8340007F0CEFDEB68334404
:10C600005968FFF78FFC0134E4E7000073B5054675
:10C610000C46164601F01EFB437B5BB10422CDE9BC
:10C62000002600EB83022146136928466A46984794
:10C63000009B43B1284601F019FB044902462346FA
:10C640000348FFF744FD02B070BD00BFFABA050809
:10C65000F418060873B50C46064601F0FBFA838809
:10C660001906054632D4C37BB3B14CB900EB830342
:10C670001A69174B9A4203D01020F3F7F9FD0446CC
:10C68000EB7BAA8805EB8303D2051B69214648BFD3
:10C690001B683046984778B96A460F213046FFF745
:10C6A000A9FC009B53B11CB91020F3F7E1FD04462F
:10C6B0002146684604F06AFB02B070BD304601F0C6
:10C6C000D5FA044902460448FFF701FD3046F3E776
:10C6D000ED5C030819BB05082017060837B50446AA
:10C6E00001F0B8FA818811F4C0750AD0104B00220D
:10C6F0001A62FFF789FB0346204603B0BDE83040CD
:10C7000018476A4619212046FFF774FC009B3BB985
:10C71000204601F0ABFA074902460748FFF7D7FC6D
:10C720006A4629462846FFF722FE03B030BD00BF07
:10C730003400002026BB05082017060830B5054642
:10C7400095B000F059FF284601F084FA848814F46B
:10C75000C0740AD01B4B00221A62FFF755FB034638
:10C76000284615B0BDE8304018476A4619212846CA
:10C77000FFF740FC009BE3B102A8F3F739FD014647
:10C7800040B96A46FFF7F3FD0446F3F707FD20467C
:10C7900015B030BD039B0C4918680AF05FF80346DA
:10C7A000039823B103F084FB064B1862EFE7F3F71D
:10C7B00037FD284601F05AFA044902460448FFF7BB
:10C7C00086FC00BF34000020A819060826BB050817
:10C7D000201706082DE9F04F8DB013680293044628
:10C7E000002857D102F10408C1F307294FEA490391
:10C7F000CFB253FA81F14FEA810B58F821607610DD
:10C800005ED13546BB00039308EB8703009308EB2A
:10C810000B03019308EB870A4FF0000B019B9A452D
:10C8200052D1D9444FEA490B07F1010A002E5FD1DA
:10C830000BEB0A05A800F3F71BFD814614B1046059
:10C8400057460126039A414609EB86001AF052FA30
:10C850003C46A344AB4506D948464FEA8B01F3F763
:10C8600022FD5D468146DFF804A22646DDE900325E
:10C87000934240F08A80321B21464B465208029870
:10C88000FFF70CFD04464846F3F71AFD20460DB0AD
:10C89000BDE8F08F546802F10808A5E726FA0AF30C
:10C8A000D80708D558F82A0001F0F0FB18B101F0BC
:10C8B000C7FA013805440AF1010A5745EED1A1E74C
:10C8C0004FF0000A5546F8E7DAF800206AB9DAF8BE
:10C8D000040050B1810708D1026864498A4204D13A
:10C8E00003F02DF90BF1FF3B83440AF1080A95E7A9
:10C8F00055445D44A800F3F7BBFC81460CB10460CD
:10C9000001244FF0000A5745A3D026FA0AF3DA07AC
:10C9100058F82A0035D5830716D10368544A934244
:10C9200002D0544A93420FD108AA07A901F030FB64
:10C93000079A089909EB840092001AF0DBF9079B2B
:10C940001C440AF1010ADEE708A9FFF783FEA7EB02
:10C950000A03039004930398FFF7F0FE03460028B0
:10C96000EFD0049A2244954207D8E900484605933F
:10C97000F3F799FC059B81466D0049F8243001349A
:10C98000E9E749F824000134DBE7009BD3E9002BF9
:10C99000002A62D11BF0030726D1DBF80030534593
:10C9A00022D1DBF808309F4203D3009B0833009369
:10C9B0005CE7DBF80C3053F837004FEAC70888B162
:10C9C00004280FD000F00703022B01D008F0F6FB7B
:10C9D00049F82600DBF80C30B20043444A445B6857
:10C9E000536002360137DCE708AA6A215846FFF790
:10C9F00011FD002108AA0846FFF7B9FC0021FFF746
:10CA000029FE03900398FFF799FE07460028CCD033
:10CA1000731CAB4207D3E9004846F3F744FC4FEAE6
:10CA200045088146454607F00703022B03D03846E8
:10CA300008F0C4FB074608AA0F215846FFF7EAFC96
:10CA400008AA002101200A97FFF791FCB3004B448C
:10CA500049F8267002365860D4E7B3004B4449F8D1
:10CA600026200236C3F804B09FE700BF141606085C
:10CA70004C2806082C1E060870B5830786B00C46A5
:10CA800015461BD103681D4A934202D01C4A9342AB
:10CA900014D102AA01A901F07BFA019BA34227D37A
:10CAA00019D8029B043D03EB84049C4201D106B0DB
:10CAB00070BD54F8042D45F8042FF6E702A9FFF7DE
:10CAC000C9FD002306469C420193304606D8FFF775
:10CAD00035FE0028EBD00B4922460BE0FFF72EFE77
:10CAE000019B28B1E21A013A013345F82200EAE736
:10CAF000019A05490548FFF7EAFA00BF4C280608E5
:10CB00002C1E060849BB050834BB0508D8160608C4
:10CB10002DE9FF4183071546CFB2C1F3072436D173
:10CB20000368384A934202D0374A93422FD1029089
:10CB3000029803AA01A901F02BFA01983B1983423C
:10CB40005AD80399002601EB8003A64214D1C01BDA
:10CB500001EB8701801B05F04DF9039945F826008C
:10CB6000BC0005EB86080B1942468B420AD1002314
:10CB7000029304B0BDE8F08153F8042D45F8262057
:10CB80000136E2E753F8040D42F8040FEDE7002107
:10CB9000FFF760FD002380469F42019317D80021D4
:10CBA000084605F027F906464046FFF7C7FD01464F
:10CBB000C0B9B368A3421FD345F8246005EB8402D3
:10CBC00005EB8301AA4211D11B1BB360D1E740469C
:10CBD000FFF7B4FD019B78B1FA1A2244013345F8FE
:10CBE0002200D9E7304604F07AFEDDE7F768881ABC
:10CBF000385842F8040DE5E7019A04490448FFF764
:10CC000066FA00BF4C2806082C1E060834BB05082F
:10CC1000D81606082DE9F04F85B000AF07F10802DD
:10CC200005460C46FFF7E6F9D7E9020129B102F003
:10CC300081F81437BD46BDE8F08F0028F9D107F11F
:10CC4000080240F29D312846FFF7D4F9BB6823B9AA
:10CC50001E491F482246FFF73AFA07F10802284604
:10CC60001721FFF7C7F9391DB86807F01BFB82468B
:10CC70002046F4F715FAD7F8049009F10106851952
:10CC8000EB1D23F00703ADEB030D6B464A465146FF
:10CC90004FEAD30B68461AF02DF82E2309F83B30E3
:10CCA0002046F4F708FA81462046F4F7F9F96E4475
:10CCB0000246494630461AF01DF829466846F4F700
:10CCC00035F901221E21FFF77FFBB2E763BB0508A0
:10CCD000AC18060808B50446F3F7CCFB18B10449B4
:10CCE0000448FFF7EBF9044902482246FFF7EFF941
:10CCF00069BB05081C18060890BB0508014608B565
:10CD00000148FFF7DBF900BFD81606082DE9F0430C
:10CD1000831E87B0054688461746062B3BD8DFE8BA
:10CD200003F0093A3A093A040F00B94212D04FF021
:10CD30000E09ECE03A4607B0BDE8F04301F0ECB96B
:10CD4000384603F08DF940B13946404603F0B6F954
:10CD50000028ECD04FF01E09D9E017F0030440F092
:10CD600000813A68A14B9A4240F0FB8007F1040928
:10CD70007B68A342DBD959F8046F304603F070F9A1
:10CD8000002800F05D813146404603F097F9002805
:10CD9000E0D10134ECE711F0010F00F0FF804E10FC
:10CDA000F90740F1CE807C10232800F2DA80DFE81A
:10CDB00000F0B2B6D8BABED8D8D8D8121D20233DBC
:10CDC00046484AD850586A72121D20233D46484AA8
:10CDD000D850586A729446EA040090EA40034FEA39
:10CDE000400900F1A88049F0010990E086EA0400BA
:10CDF000F3E706EA0400F0E7002C02DA7C48FFF7CC
:10CE00007DFF1F2C09DC6FF040432341B34204DB5C
:10CE10004FF040432341B34205DD3046F11704F0A3
:10CE2000F7FA8046C0E006FA04F0D6E7002CE5DB0E
:10CE30001F2C2046A8BF1F2046FA00F0CDE730196E
:10CE4000CBE7301BC9E786FB0404B4EBE07FC4D01A
:10CE5000E3E7002C00F0F680214630460DF0A2FFFB
:10CE6000BBE7002C00F0EE8007EE906AB8EEE70A10
:10CE700007EE904AF8EEE77A80EE270A07B0BDE8A1
:10CE8000F04303F01FBA002C00F0DC80214630464E
:10CE90000DF07AFFA1E7002C1CDA07EE906AB8EEDD
:10CEA000E70A394607B0BDE8F04303F077BA3346E6
:10CEB0000120E20706D580FB0302B2EBE07FACD194
:10CEC000012C8AD083FB0332B2EBE37F4FEA640488
:10CED000EFD0A2E7EBD101207FE7002C00F0B28079
:10CEE0000021022008F0D8FC2146814630460DF092
:10CEF00059FF400040F00100C9F8080021463046C3
:10CF00000DF042FF400040F00100C9F80C00484617
:10CF100007B0BDE8F083A642FFF61CAF07E7A642C4
:10CF20003FF718AF03E7A6427FF714AFFFE6A6422C
:10CF3000BFF610AFFBE6C11707B0BDE8F04304F041
:10CF400067BABB072AD13B682A4A934219D107EE38
:10CF5000906A3946B8EEE70A03F020FA81460028C5
:10CF6000D5D1254B40465D5D00F080FE0446384635
:10CF700000F07CFE21490090234621482A46FFF715
:10CF8000A6F8204A934209D107EE906ADFED1E0A07
:10CF9000B8EEE70A394602F06BF8DFE7062D03D159
:10CFA00043462425B8461F46404600F053FE037B07
:10CFB00033B9A5F109030C2B0DD80D35EDB2F3E70C
:10CFC00000EB83003A46036941462846984781466C
:10CFD0000028EED09BE7A5F116030C2B16D843468C
:10CFE0000F35B846EDB21F46DEE700BF4C280608F5
:10CFF000BEBB0508BC1A060804290608D3BB0508F1
:10D00000201706082814060800000000242D04D963
:10D0100043460F3DB846EDB21F46242DA1D102A9CB
:10D020004046FFF717FB04462046FFF787FB002822
:10D030003FF47DAE394601F0E7F80028F4D089E6E8
:10D0400037468EE701490248FFF738F8E6BB050886
:10D050003C190608014608B50148FFF72FF800BF44
:10D06000201706082DE9F041044617461E460D46D6
:10D0700041B1186800F0EEFD6368834202D00548B4
:10D08000FFF7E8FFA06833463A462946BDE8F0417D
:10D09000FFF704B9F2BB0508014608B50148FFF7E0
:10D0A0000DF800BF8C17060807B50022019101ABEF
:10D0B000012102F04DFEF3F7B3F80000014608B578
:10D0C000024809B9FEF7FAFFFFF7EEFFA8190608B4
:10D0D00008B500F0CBFD024902460248FEF7F7FF13
:10D0E000FCBB050820170608410008B5024841F0BE
:10D0F0000101FFF7D9FF00BFD417060808B50248A1
:10D1000042F23A51FFF7D0FFB017060830B593B09E
:10D11000044668460D46F3F76BF848B920462946A1
:10D12000FFF710F90446F3F739F8204613B030BD85
:10D130000199024800F0C8FD0024F6E71C06060825
:10D14000054BD861B3F8242212B2012A04BF002291
:10D15000A3F82422704700BF3400002002480023B7
:10D1600043643C30FFF7ECBF34000020EFF3108144
:10D1700072B6084AB2F824321B0443BFB2F8243214
:10D1800003F1FF331BB24FF6FF73A2F8243281F391
:10D190001088704734000020EFF3108172B60C4BFA
:10D1A000B3F82422013212B2A3F8242252B9DA6968
:10D1B0002AB9D3F8282212B993F830222AB10022D2
:10D1C000A3F8242281F3108870470122F8E700BFFA
:10D1D0003400002070B5EFF3108572B60F4B93F852
:10D1E0003022082A18D0B3F8244224B2012C04BFFC
:10D1F0000024A3F8244293F83142561C224402F042
:10D200000702293283F8306203EBC203C3E902014B
:10D21000012085F3108870BD0020FAE7340000205B
:10D220000228F8B52C4C034610D0E26972B1EFF336
:10D23000108272B6E06938B10021012BE16103D19F
:10D2400082F31088F2F7ECFF82F31088B4F82432EE
:10D250001BB243B9EFF3108272B6B4F8246236B24F
:10D2600016B182F31088F8BDD4F82C724FF6FF7314
:10D27000A4F8243297B1D4F828526B68C4F8283245
:10D280000BB9C4F82C322B682E6082F31088284624
:10D290009847EFF3108272B6AF42ECD194F8305257
:10D2A000BDB194F8313203F12901013304EBC1011E
:10D2B00003F00703013DD1E9020184F8313284F81B
:10D2C000305282F31088FFF721FFBDE8F840FFF7E6
:10D2D00063BF82F31088F8E7340000200120FFF7D5
:10D2E0009FBF08B5FFF7FAFF30BF08BD08B5FFF7CD
:10D2F000F5FF30BF08BD000038B1044A13699842F9
:10D3000002D010611846704700207047340000209A
:10D3100001F00F0108290DD8DFE801F011050A0C12
:10D320000C0C0C0C0E0000280CBF0E201E207047A9
:10D3300004F07EB804F097B8C00040F002007047D7
:10D3400008B500F0D3FD10EE100A2BF05DF941ECAA
:10D35000100B08BD00F0CABD08B551EC100B2BF046
:10D36000ABF9BDE8084000EE100A02F0ABBF02F0D6
:10D37000A9BF0000F0B593B00546684616680F4691
:10D380001446F2F735FF78B9002E0CBF394600215C
:10D39000234632462846FFF76DF80546F2F7FEFEB3
:10D3A000012D0CD1284612E0019B23601049206812
:10D3B00002F084FE034620685BB9F2F731FF236870
:10D3C000002DF3D10BB90623236036B9002013B02A
:10D3D000F0BD02F06DFD2060F7E70649304602F02F
:10D3E0006DFE0028F2D03046FEF7D2FFE5E700BF21
:10D3F000A8190608141A0608036803B94068FFF75D
:10D400009DB91346C1F30722C9B2FEF747BF1FB546
:10D4100001F00F03012B04460CD011F00E0F0BD0BE
:10D42000023B012B0AD9012201A900F035FF50B1BE
:10D43000019801E000F048FE04B010BD04B0BDE862
:10D44000104000F009BD204600F006FDF4E708B5E5
:10D4500028B1062803D0FEF79BFFF2F7E1FE08BDD6
:10D4600010B50C4619B9BDE81040FFF7F3B8FFF747
:10D47000F1F884421CBF0023C4E90030002010BD35
:10D4800040F2FA43984217D840F2F643984209D83E
:10D490005E281DD075281DD03E2814BF4FF0FF30E8
:10D4A00001207047A0F59F60022815D8DFE800F042
:10D4B0000C0E02000520704740F28E53984214BFB4
:10D4C0004FF0FF3003207047062070470720704759
:10D4D00002207047002070470420704738B503468B
:10D4E00014460D4661B152B111462846984760B1C5
:10D4F0006B683BB96C6045F00103AC60E3602C469F
:10D50000204638BDAB68DC60F5E76368EB606560BA
:10D51000002BF5D144F00103A560EB60F0E7F8B50E
:10D52000064631B1002511F0010304D00023EB6061
:10D5300029460846F8BDCC68CB6014F0010307D13A
:10D54000E768E36022463046FFF7C8FF3C460146E5
:10D550000A4630462946FFF7C1FF21460546E2E765
:10D560008A422DE9F04184460F4606D100235168D6
:10D570005360BDE8F041FFF7D2BFD66896B11446BC
:10D58000E468E307FCD524F0010451686368934222
:10D5900006F0010816D1002339B9984518BF1E4678
:10D5A0006660D1603846BDE8F0815360D360604664
:10D5B000FFF7B5FF05466060EE60B8F1000FF1D0EF
:10D5C000A560EFE71D46DB689342FBD100225A605D
:10D5D000DA606046FFF7A3FF0028EDD0E86005465B
:10D5E000EAE70000034B82B0186801ABC01A02B032
:10D5F000704700BF3400002007B5064A1368526820
:10D6000001A95B1A9A4201D8FFF778FD03B05DF8D3
:10D6100004FB00BF3400002010B503461446500C34
:10D62000C2F34F0221B1E10702D40C48FFF712FD0B
:10D63000904206D198420FD0094902460948FEF7A8
:10D6400046FD984204D9C21A07490648FEF73FFD35
:10D650009A4201D20549F1E710BD00BF03BC05089D
:10D660000DBC0508201706081FBC050827BC0508C7
:10D670002DE9F74FDDE90CA7002406468B46154639
:10D680000193A046A146019B9C4204D1B1453CD2E6
:10D690002248FFF7DFFCB44210D2BAF8022092050C
:10D6A000F6D45BF8240009F101099AF80220012A56
:10D6B00024D100F009FD07F8240017E0BAF80010A3
:10D6C000C900002241F00201284600F093F888B911
:10D6D000BAF80220D30505D5BAF800201049114840
:10D6E000FEF7F5FCDAF8042047F8242001340AF1AB
:10D6F000080AC8E7406808F10108D6E7022A01D104
:10D7000000F09EFB47F82400F0E72B68B8EBD30F3E
:10D7100001D20548BDE703B0BDE8F08F42BC050863
:10D720003DBC0508201706084CBC050870B586B03E
:10D730000446154602EB800203A81E4600F031F8AD
:10D740000B9B01930A9B009303AA3346294620466C
:10D75000FFF78EFF06B070BD08B50148FFF79CFCCF
:10D7600056BC050807490346002231F8020B9842CF
:10D7700006D20132222AF8D103EB530343F0010011
:10D78000704700BF2412060810B50446416019B95D
:10D790000123A160236010BDC800F2F782FD01469D
:10D7A000F6E74160C90041F00701016082607047FF
:10D7B00003789B0710B5044602D48068F2F780FD19
:10D7C0002368002262F3DF036260236010BD0378E8
:10D7D0009B0710B5044602D48068F2F771FD2368F8
:10D7E00003F0040343F0010323600023C4E9013381
:10D7F00010BD00002DE9F04F022A85B004460E4608
:10D80000904612D0426882B1904BC1F386010B441E
:10D8100093F83232B3FBF2F102FB1133826802EB70
:10D82000C30552F83330B34213D0237813F001020A
:10D83000019213D006F00702022A0FD016F003025D
:10D8400003D130688249884207D0B8F1010F05D072
:10D850000025284605B0BDE8F08F01925B076AD528
:10D860002768A56827F007072F44BD4232D3B8F1D7
:10D87000010FEDD1D4E90032B2EBD30FC3F3DC01D9
:10D8800011D104316160A068C900F2F70CFDD4E940
:10D890000032A2EBD30223F00703A060D2000021E4
:10D8A000184419F06BFA2368A168C3F3DC02501C1A
:10D8B00001EBC20560F3DF03236041F83260002210
:10D8C00006F007066A60022EC3D0237862F30003D5
:10D8D0002370BEE72868B04224D1B8F1020F17D1F7
:10D8E0002368D5F80480083B7A1B05F10801236002
:10D8F000083A284619F02EFA2568A368C5F3DC0219
:10D9000025F007051D44002143F83210C5F80480B6
:10D910004E4BC6F386061E44A368EB1ADB1086F84E
:10D92000323296E7019B23B9314600F06DFC0028A6
:10D93000D3D1083599E763682BB9B8F1010F87D1C6
:10D94000204600F087F806F0070BBBF1020F2BD141
:10D95000F008F3F799FB81466368B9FBF3F203FB28
:10D96000129A57460025A26852F83700FB0002932E
:10D9700002EBC703F8B9B8F1010F7FF469AF226871
:10D98000C2F3DC010131002D18BF2B4661F3DF0229
:10D99000BBF1020F2260C3E9006003D0227860F37C
:10D9A000000222701D4654E731460620FEF7E0FBD8
:10D9B0004FEA6009D0E7042819D1002D08BF1D46A1
:10D9C00063680137B7FBF3F203FB1277BA45CAD19C
:10D9D000B8F1010F7FF43CAF002D32D02368002254
:10D9E00008332360BBF1020F2E606A606CE7B0421F
:10D9F00018D1B8F1020F0ED1216860680839216092
:10DA0000791CB1FBF0F500FB1511A06850F831103E
:10DA1000A9B9F80011500D4AC6F38606164486F8D7
:10DA20003272BFE701990029CAD13146CDE90232ED
:10DA300000F0EAFBDDE902320028C1D0D9E7042179
:10DA4000E7E7204600F006F886E700BF3400002034
:10DA5000042706082DE9F04146680446701CFFF7CC
:10DA600081FE0546C000A768F2F71BFC23686560CD
:10DA700003F0060343F001032360A0603D1D4FF057
:10DA80000008B04504D13846BDE8F041F2F718BCB3
:10DA900055F8041C39B1042905D001222046FFF7AE
:10DAA000A9FE2B68436008F101080835E9E710B5C5
:10DAB00000230446016043608800F2F7F2FBA06097
:10DAC00010BD03682DE9F74F04460F46934623B96E
:10DAD00012F0010F65D000F067F839460620FEF716
:10DAE00047FB4FEA600A2368BAFBF3F603FB16A66E
:10DAF00035464FF00008A16851F82590AA0001EBC7
:10DB00008503B9F1000F0CD11BF0010F49D06268F9
:10DB1000B8F1000F18BF4346013262601F60B9467A
:10DB200033E0B9F1040F17D1B8F1000F08BF9846E0
:10DB300023680135B5FBF3F203FB1255AE42DAD18F
:10DB40001BF0010F2DD0B8F1000F26D06368013310
:10DB50006360C8F80070E2E739464846019200F079
:10DB600053FB019A0028E3D01BF0020F0DD063682D
:10DB70002068A168013B63606B1CB3FBF0F400FB01
:10DB8000143351F8233023B98B50484603B0BDE815
:10DB9000F08F042341F82530F7E7204600F004F821
:10DBA000A1E74FF00009F0E7F8B50768866804467A
:10DBB000781CFFF7D7FD0025206065608000F2F734
:10DBC00070FBA060BD4204D13046BDE8F840F2F7DA
:10DBD00077BB56F8251029B1042903D0012220462D
:10DBE000FFF76FFF0135EDE770B5016802460023CE
:10DBF000994201D1002015E0946854F823009E005A
:10DC000001330028F4D00428F2D05568013D556056
:10DC1000B3FBF1F201FB123354F82330002B18BF91
:10DC20000423A35170BD10B504468068F2F748FB89
:10DC30000023C4E90033A36010BD704710B50C4643
:10DC4000F2F716FB046010BD10B50C46F2F71EFB90
:10DC5000046010BD83070FBF0068034B00F00F0086
:10DC600053F82000704700BF6812060808B5FFF798
:10DC7000F1FFBDE80840C088F3F71DBA70B50D4646
:10DC800004461646FFF7B8FC2846FFF7E3FF437A41
:10DC900043B100EB83033246294620461B69BDE8A9
:10DCA00070401847C28803492046BDE87040D5F748
:10DCB00063BF00BF7BBC05080A4601460148FFF769
:10DCC000DDBF00BF6C360608F7B5044608460E46B1
:10DCD00002F0E0F970B101AA6946304602F03CFA60
:10DCE000009B3BB116492046D5F78CFB009D033DB8
:10DCF000002D0BDA314620460222FFF7BFFF114903
:10DD0000204603B0BDE8F040D5F77CBB019A0E4930
:10DD100002EB850320465B6852F82520D5F72CFFDF
:10DD2000019BAF003B449A6822B906492046D5F7CB
:10DD300069FBDCE705492046D5F71EFFD7E700BFA2
:10DD400080BC0508EFD20508A4BC0508B9BC0508CD
:10DD500008B50246FFF77EFF837A53B100EB8303D9
:10DD600006491B698B4204D1BDE80840104608F003
:10DD700049BD181E18BF012008BD00BF2966030851
:10DD8000830710B5044603D10268084B9A4208D0B5
:10DD900021460820FEF7ECF910B92046FFF798F964
:10DDA00004462046BDE8104003F0D0BC141D060810
:10DDB000830713B5044603D102680D4B9A4208D07D
:10DDC00021460820FEF7D4F910B92046FFF780F964
:10DDD000044614F0010103D06010E11702B010BD39
:10DDE0006B460822204603F04BFADDE90001F5E717
:10DDF000141D06080E2838B503460C4604D100232E
:10DE000023600125284638BD1E2801D10123F7E7EC
:10DE100010F0010501D04310F2E7820707D1016835
:10DE2000064A914203D103F047FB2060E9E7194617
:10DE30000820FEF79DF90028F5D1E3E7141D060838
:10DE400013B501A90446FFF7D5FF10B92046FFF727
:10DE50003FF9019802B010BDC20705D4830705D170
:10DE60000268034B9A4201D103F01FBBFFF7E8BFE2
:10DE7000141D06080E2838B503460C4629D01E2866
:10DE80002AD010F0010508D0431000EE103AB8EE89
:10DE9000C00A84ED000A012519E081070CD102684F
:10DEA0000F498A4202D103F069FCF2E70D498A4228
:10DEB00002D102F06FFAECE719460920FEF758F993
:10DEC00028B1820703D10268064B9A42F1D0284656
:10DED00038BD9FED050ADCE7B7EE000AD9E700BFC1
:10DEE000141D0608BC1A06080000000013B501A99D
:10DEF0000446FFF7BFFF38B92046FFF7B7FE0449D5
:10DF000002460448FEF7E3F89DED010A02B010BD99
:10DF1000C2BC050820170608F8B504460F46164689
:10DF2000FFF7A8FF054620B10023336001252846EE
:10DF3000F8BDA10709D122680B4B9A4205D13246A0
:10DF40003946204601F08EF8F0E721460A20FEF718
:10DF50000FF90028EBD08207E9D10268024B9A4200
:10DF6000E5D132463946EDE72814060810B50446D7
:10DF7000FFF7D2FF38B92046FFF778FE0249024684
:10DF80000248FEF7A4F810BDCDBC0508201706080E
:10DF9000830710B50FD103680A4CA34204D143682C
:10DFA0000B600830106010BD074CA34203D183689A
:10DFB0000B60C068F6E7FFF759FE044902460448C3
:10DFC000FEF785F84C2806082C1E0608D4BC050868
:10DFD0002017060813B50C4601A9FFF7D9FF019BCE
:10DFE000A34204D0034904482246FEF770F802B069
:10DFF00010BD00BFDDBC0508D8160608F7B51F46E2
:10E00000D30706460D4614460DD5541001940198C9
:10E01000002823DA2844B7B100281DDBA84228BF16
:10E02000284603B0F0BD01A91046FFF7E3FE002823
:10E03000EDD12046F588FFF719FE0A4903462A4626
:10E040000948FEF744F8002801DBA842E9D3F2882A
:10E0500006490748FEF73BF80020E2E7002FDDD134
:10E06000F3E700BFEFBC05082017060806BD05084A
